:020000040800F2
:10000000005000201D2C0108BD2C01080516010818
:10001000BD2C0108BD2C0108BD2C0108000000000A
:10002000000000000000000000000000BD2C0108DE
:10003000BD2C010800000000BD2C0108D17800088B
:10004000BD2C0108BD2C0108BD2C0108BD2C0108E8
:10005000BD2C0108BD2C0108A9900008A59000083E
:10006000BD2C0108BD2C0108BD2C0108BD2C0108C8
:10007000BD2C0108BD2C0108C5900008BD2C01084D
:1000800075CA0008BD2C0108BD2C0108BD2C010853
:10009000BD2C0108BD2C0108BD2C0108A190000851
:1000A000BD2C0108918E0008BD2C0108A18E00080E
:1000B000818E0008718E0008618E00087F53000851
:1000C00083530008795300087D530008BD2C0108B4
:1000D000BD2C0108B9900008AD900008BD2C0108A6
:1000E000E1780008BD2C0108BD2C010800000000CB
:1000F0000000000000000000000000000000000000
:0C01000000000000000000005FF808F1A3
:100110002DE9F04F684B694EA1B033600023736046
:100120000FF0E2FB18B90FF001FC09F015FC09F023
:10013000DDFC634A634C1378634D43F00103137095
:100140000023089309930A934FF4E0130B93236859
:10015000287B43F480332360A36943F01003A36139
:10016000236803F400330993089B01330893099B28
:100170001BB9089BB3F5A06FF2D12368514913F462
:10018000003301D0022315E00A6842F001020A6040
:100190000893236803F002030993089B0133089333
:1001A000099B1BB9089BB3F5A06FF2D123689A078E
:1001B00039D501230A93454B45491A6842F010028C
:1001C0001A601A6822F003021A601A6842F00202EA
:1001D0001A606368636063686360636843F48063A4
:1001E00063603C4B1A68043B22F070425A603A4A02
:1001F0001160616821F47C116160596841F000412F
:100200005960D96821F40041D9609B681B0449BF3B
:10021000324B4FF4E01313604FF480130B930A9B9F
:10022000012B01D117E0FEE7022B18D168B10B9B1F
:10023000B3F5801F02D14FF4A01305E00B9BB3F57B
:10024000E01F02D14FF400130B930B9963680B432B
:1002500043F4803302E0636843F46013636023680F
:1002600043F0807323602168164B8F01FBD55968DA
:1002700021F003015960596841F002015960636837
:10028000104903F00C03082BF9D14B68DFF85480B8
:1002900003F00C03042B03D0082B03D00C4B29E0F4
:1002A000136827E04B684868C3F38343C00303F136
:1002B000020319D40A4A1CE0FB9100082809002017
:1002C0002C30002000100240541100200020024079
:1002D00000127A000410014020000020001BB7002B
:1002E00000093D003C00002049681268890348BFAE
:1002F00052085343C8F800306368DFF870A3C3F3B3
:10030000031353441A7BD8F80030DFF874B3D3409A
:10031000C8F80030C04B0DF18009CBF80C30A36950
:10032000002743F00103A361636ABC48B360636ABA
:1003300043F080736362A36943F01C03A3614FF62B
:10034000FF7329F82C3D49468DF856700CF088FC57
:10035000B34849460CF084FC4946B2480CF080FC96
:10036000B14A4846536843F0007353600DF02AF9D0
:10037000159BAE4A6420B3FBF2F3AD4A1360AD4B5C
:100380004FF47A721F60D8F80030DFF8F882B3FBC0
:10039000F2F3A94A013B5360F0238BF82330072383
:1003A00097601360AB68C8F8003007F05EFA394612
:1003B000A248A02214F00BFEE369394643F007037C
:1003C000E361A36943F4006343F00C03A361544663
:1003D0009B4B4FF0000A03F10C0201F802A001311F
:1003E0000E29F5D1FF229A76DA761A775A77954B4D
:1003F000954A51461A6095483022D8F8008014F08A
:10040000E6FD5146C8F380170423914ADFF83CE229
:10041000885C0C224A4302F80E0047B91E380128B6
:100420009FBFFF2003F1FF3302F80E00DBB2013162
:100430000429EAD1874A95F805B01370864B87499D
:1004400083F800B0864B7E4A3362C0330B60854B25
:1004500018F0200F03EBCB035B7818BF0123536226
:10046000002340F2DC51804A22F813100133082B9C
:10047000F7D10EA800211C2214F0A9FD18F4007A6F
:100480001DBF7A4BCDF850900493CDF810A0BBF16E
:100490000E0F03D00BF0EF03082B02D101238DF8D0
:1004A0004A30012006F0B6FF18B14088003018BF6E
:1004B0000120C8F340038DF83E30C8F340338DF877
:1004C0003830C8F3C03300F001008DF83B3018F429
:1004D00000638DF83D008DF8407004D095F88431AC
:1004E0005A1E534253418DF83C30C8F300438DF8F7
:1004F0004130736A1AF1000A18BF4FF0010A003345
:1005000018BF01238DF84330C8F300538DF84430F1
:10051000B5F84631B5F8440118F4805FADF84830BD
:10052000B5F85231ADF84E0018BF5148ADF846301D
:10053000C8F3804318BFB0F84C018DF83F30B5F8D0
:10054000503118BFADF84E00B3F5FA7FADF84C301E
:1005500084BF0023ADF84E3095F8D431454886F875
:100560002830002386F8293043709DF84A3008F07F
:100570000101002BC8F3C0028DF839108DF83A2024
:100580008DF842A00CBF0023022301B902B1013350
:1005900004EB8304E3694FF00009A3F1020A1A3364
:1005A00003934FF6FF733AF8026F9E4200F09B816F
:1005B0009DF83D20F3B21AB19A1E012A40F28F81B4
:1005C0009DF8402032B12C491A0189582B4A91429A
:1005D00000F085819DF8412032B127491A018958E0
:1005E000264A914200F07B819DF83E2052B1224A7A
:1005F0000A4802EB03125168814203D11289102A82
:1006000000F06D819DF83B20002A44D01A4A03482F
:1006100002EB031238E000BF0005FA0500080140B4
:10062000000C0140001001400000014040420F005A
:10063000441A0020481A002010E000E04C29002055
:100640002809002014280020461300201828002024
:10065000F99601082911002034040020682A00209E
:10066000641100201C8E010894100020306D0108D8
:100670005411002051090020C88B010800040040DB
:1006800000ED00E0342E00205168814203D1128930
:10069000022A00F024819DF83C2052B1C44AC5488A
:1006A00002EB03125168814203D11289022A00F041
:1006B0001681149A7AB1BE4C116804EB0314606879
:1006C000884208D121899088884200F00881D28828
:1006D0008A4200F00481360A022E02D19DF83820A9
:1006E00003E0012E04D19DF83920002A00F0F780A4
:1006F000AF4F9DF844104FEA031807EB08043A4641
:1007000031B19DF84A1019B9043B032B40F2CF8058
:10071000012EF0B246D1A84D4244FF23517B85F80B
:10072000703085F87130506802F1080312894FF07B
:10073000000BADF854208DF85610022215A985F84B
:1007400074B0C5F8804005938DF8572085F82CB01B
:10075000C5F830B0C5F834B0C5F838B0C5F86CB0DD
:1007600085F872B085F873B00CF07AFA059B57F8EB
:10077000080099785A460CF027F920465946324627
:1007800008F0EAFB8D4BC5F88CB0C5F884308C4B73
:100790002046C5F8883005F1840105F1880208F08B
:1007A00023FC9CE002284AD15FFA89F31C255D43B3
:1007B000DFF8FCC1DFF800B20CEB08010BEB05071A
:1007C000012391F80DE001F1080287F874304B68BD
:1007D0000989002687F87590ADF854108DF85700F8
:1007E00015A9184687F8766087F87E60C7F88040BC
:1007F0008DF856E0CDF818C005920CF031FADDF80E
:1008000018C0059A5CF80800917832460CF0DCF8C4
:1008100020463146012208F09FFB6A4A07F1840313
:10082000C7F88420684AC7F88C60C7F88820194642
:1008300020461A1D08F0D8FB09F101094FE00328F2
:1008400033D19DF83F305C4D604E3BB195F82A7036
:10085000204608214FF6FF7200231AE0BDF84C2015
:1008600095F82A70B2F5FA7FBDF84E300BD9584989
:100870002046B1FBF2F2082192B20CF0E5FA554B9A
:1008800046F827000AE054492046B1FBF2F2012164
:1008900092B20CF0D9FA514B46F82700C36095F894
:1008A0002A30013385F82A3019E0042817D1BDF821
:1008B0004620494B404D93FBF2F22046BDF84830AC
:1008C000012192B295F829600CF0BEFA95F8293012
:1008D00005EB86060133C6F8540185F82930039BE1
:1008E0009A457FF45EAE344F3D4E97F829200023A1
:1008F00087F874213B4A33701578A5F11702022A54
:1009000019D81C463B6A0021185903EB040811F062
:100910003DFB10B17B6A63BB26E0334B04EB030E57
:1009200098E80F008EE80F00337810340133C02CA4
:100930003370E7D1EEE72D4A12F835E002EBC5023D
:10094000D2F804C086F800E0BCF1000FE2D01C46EB
:100950007445DFDA244A230103EB020863440FCB1A
:10096000013488E80F00F3E7214F3B68DB044DD4E6
:1009700046E0204B204A13F8350003EBC5035C68C2
:100980001070002CF0D000238342EDDAC3EBC301DA
:100990006218D2F800C0DFF864E0013341F80EC0FD
:1009A00001EB0E079188B9809279BA71ECE700BF2C
:1009B000C88B0108000C014028090020B9C70008B5
:1009C00099C8000805CA000891C700081829002026
:1009D00000127A00B9C8000840420F00A9C80008F8
:1009E0004829002034040020700300201C8E0108D8
:1009F000342E0020BC760108F4290020F5290020BF
:100A000005F0EF03082B9E4B24D125E03378012B12
:100A1000F6D99C4C04EB031303F110061034B442D6
:100A2000EED054F8100C4FF07C5111F01BF94FF040
:100A30007C5144F8100C54F8140C11F013F94FF0D9
:100A40007C5144F8140C54F80C0C11F00BF944F8D8
:100A50000C0CE3E70E2D08D11A78182D42F0100285
:100A60001A7008D10DF04EFA05E01A78192D22F00F
:100A700010021A70F5E70DF029FA3B6801205C03BB
:100A80005EBF814B01221A70804A814C13784FF06F
:100A9000100943F00403137004F0F6F83D68204693
:100AA00000214A4614F093FA022305F4004805F4A5
:100AB000006700261D408DF836308DF837600CD069
:100AC00074480DA9ADF834900CF0F0FE04232370A7
:100AD000012507236670A570E37020236D480DA9DA
:100AE000ADF834304FF0010A0CF0E0FE4FF0070B88
:100AF0000523DFF89C9123726E1C657284F80AA0AE
:100B000084F80BB0B8F1000F0FD0022361480DA993
:100B1000ADF834300CF0CAFE89F8056089F804A0FD
:100B200089F806A089F807B0AE1C7FB102235A48A5
:100B30000DA9ADF834300CF0B9FE0923012223735E
:100B4000A273731C07226673E273DEB2534A5448E1
:100B50005368002543F4404353605369504F43F0BA
:100B600001035361936943F4007393610CF0B2FC89
:100B70004C4B012E15934C4B15A916930CBF2B46CD
:100B800080231A934FF480731B934FF480631C935C
:100B900020231D9338464FF400531E931795189643
:100BA00019951F950CF078FC3B68404943F0010310
:100BB0003B604A68012E22F4702294BF0023012377
:100BC00022F4807242EA03224A608B68384A1A4053
:100BD00042F4602242F002028A60CB6A23F470027F
:100BE000731EDBB242EA0353CB622946012362182B
:100BF000907800286CD0655C581C092DC0B2D27862
:100C00002A4F10D9A5F10A06D7F80CC006EB460604
:100C10004FF0070E0EFA06FE2CEA0E0EB2404EEA18
:100C20000202FA600CE03E6905EB450C4FF0070E3E
:100C30000EFA0CFE26EA0E0602FA0CF232433A6174
:100C4000062B1A4E0CD85A1E776B02EB82021F231A
:100C5000934027EA030705FA02F33B43736336E048
:100C60000C2B27D8DA1F376B02EB82021F2393402D
:100C700027EA030705FA02F33B43336327E000BF8B
:100C80004419002078030020A00800202C30002008
:100C90007428002000080140000C014000100240B0
:100CA000080002404C240140842800200024014018
:100CB000FDF7F1FFA3F10D02F76A02EB82021F2399
:100CC000934027EA030705FA02F33B43F362034626
:100CD000043110298BD1BE4B9A6842F480729A601D
:100CE0009A6842F001029A609A6842F008029A609B
:100CF0009968B74A0807FBD4936843F004039360EC
:100D0000B34B9A6812F004020392F9D19A6842F444
:100D1000A0029A60AF4BB3F85801002840F0BC879E
:100D2000B3F95A21002A40F0B787B3F95C31002BA0
:100D300040F0B287A84BA74C1B68A84FB3F85630B9
:100D400000210C22A648059394F85FA194F869B19C
:100D500094F86A5114F03BF914223846002114F03B
:100D600036F9A04EA04A00231370C6F8783104F07B
:100D700009FB002800F073879C4B9D4A3B609D4B0C
:100D80007B609D4BFB609D4B3B61012313709C4935
:100D90000B709C4B884699461A6842F001021A6013
:100DA0005246092A4FF0000101D90A46F9E74FF0EF
:100DB000010A0AFA02F313F04D0005D113F46C7323
:100DC00057D0914B18704AE08F4BC6F878111970C4
:100DD00004F0D8FA002842D006210A4615AB682054
:100DE00004F0A2F89DF8591001F001029DF8571087
:100DF00001F001014B0043EA82019DF8552002F009
:100E000001030B430AD05BB2012B01D1002302E0A6
:100E1000022B0ED1012386F87C3111E00DAB682046
:100E20000C21524604F080F89DF8343013F00F0383
:100E300003D1032006F023FD02E0042BEAD1E5E70D
:100E4000674B724A1A60724A5A6096F87C21002AEF
:100E50000CBF6F226E221A72032300F009BF604B91
:100E60006C4A1A606C4A5A6000221A72092300F018
:100E7000FFBE012A9A4693D8634A1370042D00F2EC
:100E80000F81DFE815F00500160105000500D70009
:100E900096F87D31534D002B40F08387142006F0E7
:100EA000E4FC7720D02101220DAB04F03DF80028AE
:100EB00000F0C0809DF834300322552B85F897311F
:100EC000A5F8A02140F0B680D12101220DAB7720FA
:100ED00004F02AF89DF83430772003F00F021B0944
:100EE00085F8982185F89931162215ABAA2104F0CE
:100EF0001BF89DF854209DF8553043EA0223A5F8CD
:100F000080319DF856209DF8573043EA0223A5F81A
:100F100082319DF858209DF8593043EA0223A5F804
:100F200084319DF85A209DF85B3043EA0223A5F8EE
:100F300086319DF85C209DF85D3043EA0223A5F8D8
:100F400088319DF85E209DF85F3043EA0223A5F8C2
:100F50008A319DF860209DF8613043EA0223A5F8AC
:100F60008C319DF862209DF8633043EA0223A5F896
:100F70008E319DF864209DF8653043EA0223A5F880
:100F800090319DF866209DF8673043EA0223A5F86A
:100F900092319DF868209DF8693043EA022341F2BE
:100FA0007072A5F894311D4B1A8046F678125A805B
:100FB0001B4A5A601B4A9A601B4ADA601B4A1A6134
:100FC0001B4A5A61012385F87D3100F0EABE00BF5B
:100FD0000024014054110020A4100020002E002005
:100FE000102C00202809002058020020115300086E
:100FF0000800002059500008ED4B000890C1793DD1
:101000003800002040190020543000205D4C0008BA
:101010009B50000825D1000841D10008F4000020B1
:101020000953000831500008F1520008F14F000840
:10103000114B000896F8A491534DB9F1000F40F000
:101040002186142006F011FC05F2A5137620D0218C
:10105000012203F069FF95F8A531582B29D105F538
:10106000D47388211822762003F05EFF3122762087
:10107000F42104F033F80123444A85F8A431444BA9
:101080009A60444AA3F800905A6045F6D8125A80F4
:10109000414ADA60414A1A61414A5A6100F0F2BDA0
:1010A000012D06D03F4A88F80250136843F004032C
:1010B00013603C4D2B68990702D53B4B1B68984742
:1010C000002386F8C431394B4FF47A721A603B68BA
:1010D0009847374A002313709246BBF1000F03D0A4
:1010E000BBF1020F40F0D1854FF0000920AB03F8AF
:1010F0002C9D1E200A210122C6F8C89103F014FF7E
:1011000088B19DF85430482B40F04E86294B2A4A2E
:101110001A602A4A5A60022388F803302B6843F089
:1011200008032B6002E0814600F03EBE94F8543183
:101130000BB1234A137094F855310BB1214A137047
:1011400094F856310BB18AF800302B681A073FD556
:10115000BDF914A04FF064099AFBF9F8404610F06D
:101160002DFD834609FB18A000B210F027FD16499B
:1011700010F078FD0146584610F06CFC134910F051
:1011800071FDC6F8CC0126E0280900200D4B0008AF
:10119000F40000200F4B0008E9520008A54F00089A
:1011A000A948000840190020102C00201821002018
:1011B00050300020D000002061510008DDC8000838
:1011C00058020020543000208988883C00002041CB
:1011D0000023C6F8CC31A94A0A26137843F002034B
:1011E0001370192006F041FB013E192006F03DFB6B
:1011F00016F0FF06F5D12B681B0705D5A04B1B6821
:101200009847A04B01221A709F4BDFF8B4821E68EA
:10121000307B10F0D3FC9D4910F024FD08F040FB1A
:101220009B4B18609B4B188810F0C8FC01464FF090
:101230007E5010F0CBFD984B94491860386910F03F
:1012400011FD964B00271860307810F0B7FC01466E
:101250004FF07E5010F0BAFD914B014618604FF0F0
:101260007E5010F0F5FB8F4B4FF07E5218608E4B86
:1012700038469A601F605F608C4B9A601F605F60A9
:1012800008F00EFB0646384608F098FA3146074645
:10129000304610F0E7FC39468246384610F0E2FC52
:1012A00031468146504610F0DDFC394683464846BB
:1012B00010F0D8FC0146584610F0CCFB3146C8F877
:1012C0000000384610F0CEFC3146059010F0CAFC04
:1012D000059B83463946184610F0C4FC0346584621
:1012E0001946059310F0B4FB059BC8F80400194695
:1012F000584610F0AFFB3946C8F80800504610F0C9
:10130000B1FC31460746484610F0ACFC0146384671
:1013100010F09EFB664E674B0027C8F80C00FF21BB
:101320001B2230461F7013F052FE2A68624B0121C7
:1013300012F0020F19701FBF717003211970022182
:1013400018BFB1703770570748BF1978304641BF92
:101350004D1C1D700325755412F00A0F0CD01A781D
:101360000421B154511CC9B205257554D11C023257
:101370001970D2B20621B154504D29688E0641BF72
:101380001A78561C1E70072648BF86540A0608D5D0
:101390001A7809268654961C01321E70D2B20A268B
:1013A00086546679082E01D00E2E04D11A78571C67
:1013B0001F700B2787541A7811F4803F4FF00C0EE2
:1013C00000F802E002F101071CBFDFF8ECE0023296
:1013D000FFB21F701FBF8EF80020354A4FF00E0E6F
:1013E00002F807E04A0748BF1A784FF0120E41BFD3
:1013F000571C1F70102787541A7811F4806F02F160
:101400000107FFB21F7000F802E00ED094F814E25A
:10141000BEF1000F09D0DFF8A0E002328EF8002004
:10142000234A4FF0130E02F807E01A7811F4007FF8
:101430004FF0140E00F802E002F101071CBFDFF8C4
:1014400078E00232FFB21F701FBF8EF80020184AEA
:101450004FF0150E02F807E0182E33D11A78162730
:101460008754571CFFB24FF0170E00F807E0D71C47
:101470000232D2B21F70865424E000BF2C3000200C
:10148000D0000020E8000020FC2A002035FA8E3C25
:10149000F82A00200A000020B02A0020B42A0020E8
:1014A000102B0020002B0020142B0020042B0020E8
:1014B0006D1000206C2A00206C100020342E0020BB
:1014C000E82A00200F0341BF1A78561C1E70192607
:1014D00048BF8654CE0541BF1A78511C19701A2393
:1014E00048BF8354002198229B4813F070FD0BF0F5
:1014F000BEFE9A4A9A4BB4F84E111A60994BB4F852
:1015000096011980984900230B808B7097490A60D7
:1015100081B2974A22F813100133122BF9D12B68AC
:10152000D9045EBF9349B1F89C1111801B0740F1AB
:10153000C280904B93F89041062C00F2B680DFE811
:1015400004F004070E395474740045F2F05201E0BF
:1015500042F6F822884B1A800BF023FFA4E042F6F3
:10156000F822854B1A8010F029FB844910F07AFB91
:10157000834910F06DFA10F061FD0023814A42F8B2
:1015800023000133122BF9D17F4A8049402011609A
:101590007F4A137006F018F8002800F086800123B7
:1015A0004FF0070890F9000040218DE80801794AC2
:1015B000794B74E042F6F8226F4B40201A80774A4C
:1015C000714B1A60724B10221A7005F0FDFF002853
:1015D0006BD001234FF0000C90F9000040218DE802
:1015E00008106F4A4FF4E13359E042F6F822624B9B
:1015F00040201A806B4A644B1A60654B08221A70AF
:1016000005F0E2FF002850D001234FF0000E90F9C2
:10161000000040218DE80840634A4FF4E13306F0B2
:101620006AF9624BC3F8D0013BE042F6F822524B14
:101630000C261A80564B5E485E4A5F49062CDFF83E
:10164000A8C11E704FF00003037013700B705B4F46
:101650001BBF1B238CF8003021230523DFF88CE10E
:1016600014BF3B708CF80030554A474B4FF0400098
:101670000DBF3C708EF800604FF4E1348EF80060CE
:1016800008BF504C1A6005F09FFF70B1012300277E
:1016900090F900008DE8880023464B4A402106F06F
:1016A0002AF9003018BF012028B9082008F022F9D3
:1016B000464A354B1A602A68354912F4804F1FBFDD
:1016C00008230B704248304B18BF186042F20103E8
:1016D00013409BB144F62060274B9604188041BF0D
:1016E00008230B703B48284B48BF1860D40741BF04
:1016F0000C230B703848244B48BF18600B78100639
:10170000A3F104034B7040F1AA802848334E002413
:10171000DFF8DC80C0F8D4612146152200F5EC70BA
:101720002F4F88F80140C8F80440C8F80840053E2B
:1017300013F04DFC20463E6007F026FA294B0220AC
:101740001B68C8F80C3005F03FFF002852D18020FC
:1017500008F0D0F87BE000BF70270020DC120020EA
:10176000100F0020140F002004300020F82F00205C
:101770002C2F002054110020DE020020CDCCCC3FC5
:101780000000B044E42E00201C0000209912010843
:101790000C28002041140108A086010085120108D0
:1017A0009513010871120108491301082809002046
:1017B000F42F002048270020492700206C27002014
:1017C0002DD1000890D003005DD10008F912010866
:1017D000C9120108E9120108D912010846130020B4
:1017E00054020020582E00206B270020F32F0020E9
:1017F00034020020447998F80130BD490C2202FBE4
:1018000003125278A24204D00133DBB2042BF4D984
:10181000002388F801303B6898F801201B7890F984
:101820000000002B4FF00C0303FB021314BF032432
:10183000012400225B7800940192022106F05BF8FB
:10184000AC4B1860002882D0012007F09DF9AA4B0C
:101850001868AA4B00F5C5721A6007F03DFA2B68AC
:1018600099056CD5A64AA74C049BA74823609369A9
:101870000DA943F001039361049B01261B88ADF879
:10188000343010238DF8363002238DF837300BF0CA
:10189000E7F923689C485B880DA9ADF83430042330
:1018A0008DF836300BF0DCF920680F21037A03F055
:1018B000030203F0FC0303F1804303F580339C68CB
:1018C0009200914024EA01019960996806FA02F2B7
:1018D0000A439A6043688D4AD943536114680C40A7
:1018E000146054680C40546014681C43146094687D
:1018F0000C409460D4682140D16091681943916094
:10190000D1680B43D360437A15A88DF85430032374
:101910008DF8553000238DF856308DF857600FF054
:10192000ADF87B4B7B4A1B683C3B13607A4A1368DB
:1019300043F010031360794B4FF0FF321A60784B7D
:10194000784A794C1360794A803313602B680026FB
:10195000DA03267040F1AD8040F22A38DFF8F891C2
:10196000DFF89CA10CF0F2FF0127424648463146C1
:10197000277013F02CFBDAF818306D4843F004039D
:10198000CAF818304023ADF8303018238DF83330C2
:101990000CA903238DF832300BF088FFDAF81C30E5
:1019A000644A43F00203CAF81C30634B634C1B6863
:1019B000AAF6947AB3FBF2F32288013B22F45C721C
:1019C0001204120C22809BB21D22A2852385A782BD
:1019D000238C23F001031B041B0C2384238CA1887C
:1019E000228B23F0020322F0730212041B04120C58
:1019F0001B0C89B242F060023B43A1802283A68681
:101A00002384238B23F008031B041B0C43F00803DF
:101A10002383B4F844306FEA43436FEA53439BB2E5
:101A2000A4F84430DAF8A83F3B43CAF8A83F504630
:101A30000BF050FD424BCDF85890159380231A932C
:101A40004FF480734FF010091B9350464FF400532E
:101A500015A91E9319961C961D961F96CDF85C909D
:101A6000CDF860800BF018FDA3890DA89BB243F45C
:101A70000073A381DAF8003043F00203CAF80030A3
:101A80008DF834908DF835708DF836608DF837709C
:101A90000EF0F4FF2B4B03991A682B4B43F82120CF
:101AA0000B460133202B0393F4D10AF0FBFF0AF01D
:101AB000F9FF2B685B0540F18D80DFF8A080234B98
:101AC000D8F818950420C3F8009005F07DFD042196
:101AD000C8F81C0505F054FD1D4B88F820050820AA
:101AE000C3F8009005F070FD1A4B0821186037E02C
:101AF00028690108AC1C0020A4100020640F0020FD
:101B00000010024030020020000C0140000401409F
:101B1000582E00202C02002040190020C410002064
:101B200078130020E81C0020A1080020E41C0020FD
:101B30000008014000366E013C0000200004004017
:101B4000340400405C6D0108A20800203419002014
:101B50008C190020D8190020150B0020280900201E
:101B600005F00EFD954C88F82105002120462C2219
:101B700013F02DFA8E2363707C27E0237D26E3701B
:101B8000277084F82B608E4C2C220021204613F005
:101B90001EFA8A2363701020A023E370277084F854
:101BA0002B60C8F8249505F00FFD1021C8F8280512
:101BB00005F0E6FC88F82C052020C8F8309505F0E3
:101BC00003FD2021C8F8340505F0DAFC88F8380553
:101BD0000FF03AFA2B687B4A13F4002318BF012355
:101BE000137005F01BFE784B1860784B5A79194634
:101BF000052A02BF764B4FF4C8721A80754B4FF41A
:101C00007A721A80744BC8221A80744A137843F08F
:101C100008031370724A137823F00203137040F61E
:101C200002032A6813406BB16E4A6F4B1A606F4B08
:101C300003221A706E4B01221A706E4A0023138021
:101C40006D4A13808B6801222B606C4B1A706C4AB2
:101C5000137863F07F03137021B0BDE8F08F694BF8
:101C60003B60694B7B60694BBB600823FFF78FB813
:101C700088F80130D9F8003043F00203C9F8003089
:101C8000FFF7FCB80425FFF70DBABBF1010F7FF693
:101C90004DAA9B46FFF71DBA5D4B00221A7000B299
:101CA0000FF08CFF5B490FF0DDFF484C0646B4F99E
:101CB0005A010FF083FF57490FF0D4FF0546B4F9DE
:101CC0005C010FF07BFF53490FF0CCFF0446304618
:101CD00007F0E6FD8046304607F070FD06462846D0
:101CE00007F0DEFD0746284607F068FD054620465A
:101CF00007F0D6FD8246204607F060FD414681464A
:101D000050460FF0AFFF4146834648460FF0AAFF0A
:101D10005146059030460FF0A5FF494606903046E3
:101D20000FF0A0FF3946079050460FF09BFF3A4C4A
:101D30004946206007F100400FF094FF294660609B
:101D4000A56006980FF08EFF014605980FF082FE01
:101D50002946E06007980FF085FF014658460FF0CE
:101D600077FE3946206106F100400FF07BFF2946DF
:101D7000606158460FF076FF014607980FF068FE45
:101D80002946A06105980FF06DFF014606980FF0F7
:101D900061FE4146E06138460FF064FF2062FEF7C5
:101DA000C9BF0225FFF77EB9BBF1010F7FF6BEA9BF
:101DB0004FF0000B8AF80090FFF796B95C190020ED
:101DC00091190020342C0020B00200205411002072
:101DD000822A00204A300020483000204419002088
:101DE00052300020CE1200202C1900209019002023
:101DF00030000020081000200A100020A008002059
:101E00002C3000202BD100084FD1000827D100082A
:101E10002400002035FA8E3C50280020954A2DE9F8
:101E2000F04F1568944C05F59C43944E2033236085
:101E3000336889B013F4804F059205D10FF0C8FBC9
:101E400010B92379013323718D4A13784BB18D4931
:101E500009688D4240F2E58003F1FF3882F8008086
:101E6000DFE09846884B5FFA88F51F78DFF83892F4
:101E7000AF4231D9D9F80030072D98BF595D834B57
:101E800088BF29461B6880489847032D1ED8D9F87B
:101E9000002005F10E0302EB83039988DA88A8B1CC
:101EA0004FF47A73401A5843531A90FBF3F040F6FC
:101EB000C90300F57A70984205DC40F2EE2398429F
:101EC000B8BF184601E040F6CA0080B204EB4505F1
:101ED000E88008F10108C5E794F804800325B8FB01
:101EE000F5F50F2384F82A3094F82B3005EB4505DF
:101EF000019394F82C30C5EB08050393D9F8003012
:101F0000DFF8ACA10293EBB204930025BD4255DA91
:101F10005F4B4FEA450933F815B0019B53B90FF0F9
:101F200057FB28B1039B002B08BF4FF0000B01E0CB
:101F3000DDF804B0029B988A584502D8D88A5845E3
:101F40000ED2E8B20FF0F0FA032D8346DFBF94F80B
:101F50002AE00120A8402EEA0000D8BF84F82A0019
:101F60000FF036FB18B14B4829F800B022E0049B73
:101F700094F876002AF813B030B9B8F1020F15D9E9
:101F80003D4B012083F87600BAF80000BAF8023021
:101F90000344BAF8040003443F489BB229F80030D8
:101FA0001BB2032093FBF0F39BB200E05B46394881
:101FB00029F8003001350AF1060AA7E794F82A202B
:101FC0003648A2F10F014A424A4184F89020344B2E
:101FD0006AB1344A1268520109D40268D9689A6019
:101FE000521AC82A1DD9012283F8212019E002685B
:101FF0009868DA605B68121A9A4288BF284B4FF0E3
:10200000000184F82B1088BF83F821100025BD4201
:1020100007DAE8B20FF088FA1E4B23F815000135F5
:10202000F5E73368DD0405D51E4B1B68D80701D4DE
:102030000EF064F9059B1F681B4B1A68907A002804
:1020400038D01449137B013831F810001BB1C0F5AA
:102050003B60083080B200B2A0F57A70B0F57A7FAC
:10206000A8BF4FF47A7020EAE0700FF0A7FD0F4987
:1020700055E000BF38300020640E0020342E0020D0
:1020800000300020FC2F00200C2800201C00002025
:102090006A0E00202C2F0020DC0E0020582E00207D
:1020A0000430002068100020F82F002000007A443F
:1020B000920E0020336819043AD5D4F89430934D29
:1020C000FB1A002B34DB07F59C432033C5F8943012
:1020D0008F4BD27A59798F4B33F8113095F898108D
:1020E0009BB293FBF2F3013101F00F0285F89820C7
:1020F0002A4482F899300346874A825C01301344AF
:1021000010289BB2F8D11BB293FBF0F000B2642808
:10211000A8BF642020EAE0700FF050FD7F490FF067
:1021200055FE7F490FF09EFD0FF088FF7D4B188014
:1021300033687D4D13F4807F00F00F817B4BDFF817
:10214000F0919F4205D999F8022012B9012289F82D
:10215000022099F80220002A00F0FF80744A95F8C6
:10216000008092F82170C8F380087A1E57425741C8
:10217000704A002F9246116818BF4FF0000BC1F350
:102180008063019308BF4FF0030B99F82020052AC4
:1021900000F2DD80DFE802F0034E537988A5B8F144
:1021A000000F3AD0D4F8AC00B4F8B01005F0A9FA9A
:1021B000012809D16049614A09681268C988642008
:1021C00000FB0122C9F81020019B6BB15A4A12682A
:1021D00012794AB10EF034FC032289F820204FF422
:1021E0007A72C9F81C20D0E7002F40F0B080534A23
:1021F000D9F8101010684E4A88420AD902920EF09F
:102200001FFC029A032182F8201040F6B831D161F8
:10221000BBE7012182F82010B7E7019B4FF48060F3
:1022200013B107F057FB01E007F044FB0022C9F8A7
:1022300010208CE0002F49D10EF002FCA5E727B159
:10224000052289F82020012000E03846B8F1000F6F
:102250000CD0D4F8AC204FF0020BD189384A118051
:1022600051809180344909684988D180334A116886
:10227000D9F81420914202D8B8F1000F64D147F286
:102280003052C9F81C20032221E02A7842F00202D1
:102290002A700EF033F8294AD9F81C1012680A4443
:1022A000C9F81820042212E0244A9FB11168D9F815
:1022B000182091424BD9234A12781AB9DAF8002033
:1022C000D30744D42A7822F002022A70052289F822
:1022D00020205AE71268D9F81C100A44C9F81820BF
:1022E00035E01549154A09681268C988642000FB61
:1022F00001224FF48060C9F81020002289F82020C4
:1023000089F8032007F0D6FA3FE700BF640E0020EB
:102310007428002084280020FD0E00200000C84200
:1023200000C07F44C810002052300020404B4C00B9
:102330000430002068100020202E0020582E00209D
:102340002C2F00200900002000287FF41EAFBBF1D5
:10235000000F02D0584605F027FA924F07F5C470D7
:10236000B7F84E1105F0CDF90197834668B90EF024
:1023700059FB8D4B0022C3F800B0C3F804B0C3F87A
:1023800008B08A4B1A605A609A602B785F0736D57E
:102390003368D80633D5864B1B78D9062FD4854BA6
:1023A0001B789BB1019B93F8E031BBF1000F15D175
:1023B0007BB1814B1A68D4F8B4309B1A002B08DA31
:1023C0000DF09CFF7D4B83F8B8B018E0BBF1000F17
:1023D0000DD1102005F0E8F901230EE03BB1764A5B
:1023E0004FF47A71126801FB0323C4F8B43094F8F7
:1023F000B83023B105F0C8F9002384F8B830019B48
:1024000093F8DEA193F8DF11B3F898E1B3F89AC11D
:10241000002318466A4F800837F9132001337245AC
:10242000C4BF60F07F00C0B26245B8BF40F040005A
:10243000042BB946EED194F8B930604A834205D1F5
:1024400092F8BA30F92B04D8013300E0002382F867
:10245000BA30584B84F8B9001A785A4F9846E2B906
:102460003B68DA0708D5BBF1000F16D12B78DB07E4
:1024700013D50DF09DFD10E02B7858070DD54F4B6F
:1024800093F82B304BB1504BDB7833B911B10DF0D1
:1024900035FF02E0BBF1000FF9D094F8BA30474A9B
:1024A000142BDFF840B140F0AF8098F800301AF1FB
:1024B000000A18BF4FF0010A6BB392F8B9305F2BD6
:1024C00011D12B7803F0040303F0FF0113B10DF0D9
:1024D00015FF08E00B200391029205F065F9029ABE
:1024E000039982F8BA10BAF1000F14D094F8B930F9
:1024F0007D2B10D12B7803F0040303F0FF0213B1FE
:102500000DF0FCFE07E00B20029205F04DF92B4B7D
:10251000029A83F8BA202B7803F0040303F0FF013A
:10252000002B71D194F8B930244A572B15D1274B81
:102530004FF47A721A803368190601D506F01CFC34
:10254000234B1B685A0742BF224A0A21118013F00D
:10255000080359D1204A138056E03068400716D549
:102560005A2B14D11D4B187820B119701C4B012225
:102570001A7049E092F8BB3083F0010382F8BB3057
:102580000BB10C2000E00D2005F00EF93CE05D2BB6
:1025900000F017855B2B00F016855E2B24D10320FD
:1025A00000F012BD541100201C21002098210020B1
:1025B0004419002009000020582E0020640E00203D
:1025C0002C2F002068100020043000204A3000200A
:1025D000401900204830002044110020AD2A00207E
:1025E000AE2A0020A4100020562B03D1029307F03E
:1025F0004DFC029B98F80020002A00F0FB846F2B12
:1026000040F0F2840DF0D4FC33685B0732D594F8C7
:10261000BB30A3B12B78580711D5019BB9F906201F
:10262000B3F898319A420ADD3B6813F0010301BF09
:10263000AC4A32211180AC4A08BF82F8BB303B68FB
:10264000D9030AD5A94B1A782AB9A94A127812B91E
:10265000A44A3221118001220BE0A54A13784BB124
:102660002B7803F0040303F0FF011BB9A14B117099
:1026700001221A70DBF8009000233B6009F17B080F
:1026800009F1CB0A98F8002098F8013018F8010CED
:102690009A420BD2414604F0FFFF38B118F8022CE1
:1026A000012303FA02F23B6813433B6008F104087C
:1026B000D045E7D1904B1B784BB1904BDFF854924B
:1026C0001A68984612F0020F40F037832FE309F1A1
:1026D000CA0709F589783A787B7817F8010C9A428D
:1026E00025D2394604F0D8FF08B397F804E00C214E
:1026F000BB7801FB0E41824A013B03EB43031344C9
:10270000D1F8C02097F803909A4277480FD0C1F8CB
:10271000C030002390F8EC20C1F8C430012303FA44
:102720000EF322EA030381F8BC9080F8EC30063700
:102730004745D0D1734BDFF8E0A1D3F80080724B4E
:102740004FF0000B1B68029394F82B300393DAF8D8
:102750000030002B00F0E28293F80090B9F1000FF6
:1027600000F0DC82DAF8042002998A1A002A0CDBD5
:1027700001F5FA72CAF8042094F8EC10012202FA6A
:102780000BF221EA020284F8EC20039A002A00F0FE
:10279000C5821AF8042C59780432D2B2002940F0CC
:1027A0007E825A4931F91210594AB2F8962102F143
:1027B000C800814201DD9F7814E0C83A914202DAF4
:1027C00099784F420EE094F8EC20012303FA0BF3C2
:1027D00022EA030384F8EC30029B03F5FA73CAF88B
:1027E00004309BE294F8EC3043FA0BF3DA0700F183
:1027F0009582002FCCBF0220012004F0F7FF09F1E1
:10280000FF32394B132A00F28182DFE812F0140004
:1028100023003200440061008700EC005101B60142
:10282000E90118027F02440055008700EC005101C5
:10283000BE002301880198F8001040460F44FA2F8B
:10284000A8BFFA2727EAE77788F8007004F00AFFA4
:1028500001201EE098F8011040460F44642FA8BFE5
:10286000642727EAE77788F8017004F0FBFE02206E
:102870000FE098F8031040460F44642FA8BF642768
:1028800027EAE77788F80370D3F8F01004F0A2FE87
:1028900003203946D0E198F805100D203944642909
:1028A000A8BF642121EAE17188F8051004F058FFFF
:1028B000B9F10D0F00F02A8298F804100E20394467
:1028C0006429A8BF642121EAE17188F80410B3E10A
:1028D00098F806100520394481F3080188F806109D
:1028E000AAE100BF942A0020640E0020AC2A002038
:1028F000AD2A0020AE2A00205330002068100020AE
:10290000CC6D0108CC100020582E00202C2F002068
:102910005411002040190020240F0020D3F8F43077
:102920001A78022A22D1384604930FF047F9A949B0
:102930000FF04CFA049B596A05930FF08BF80021B5
:1029400004900FF02DFB059B48B9049AA14910464D
:102950000FF044FB049A059B10B19E4A00E0002250
:102960005A620F20114604F0E7FE0AE099780F2022
:102970003944C829A8BFC82121EAE171997004F03F
:10298000EFFEB9F10F0F00F0C181934BD3F8F49033
:1029900099F80030022B1AD138460FF00FF98D4903
:1029A0000FF014FAD9F820100FF054F80021074660
:1029B0000FF0F6FA30B9384686490FF00FFB10B128
:1029C000844F00E00027C9F82070122057E199F8E1
:1029D000011012203944C829A8BFC82121EAE17199
:1029E00089F8011028E1D3F8F4301A78022A22D1AC
:1029F000384604930FF0E2F876490FF0E7F9049BAC
:102A0000196B05930FF026F8002104900FF0C8FA17
:102A1000059B48B9049A6F4910460FF0DFFA049AF3
:102A2000059B10B16B4A00E000221A63102011468A
:102A300004F082FE0AE0197B10203944C829A8BF9F
:102A4000C82121EAE171197304F08AFEB9F1100F6F
:102A500000F05C81604BD3F8F49099F80030022BC1
:102A60001AD138460FF0AAF85A490FF0AFF9D9F841
:102A70002C100EF0EFFF002107460FF091FA30B94D
:102A8000384654490FF0AAFA10B1524F00E000271F
:102A9000C9F82C701320F2E099F80B101320394478
:102AA000C829A8BFC82121EAE17189F80B10C3E049
:102AB000D3F8F4301A78022A22D1384604930FF062
:102AC0007DF846490FF082F9049BD96B05930EF00F
:102AD000C1FF002104900FF063FA059B48B9049AE6
:102AE0003C4910460FF07AFA049A059B10B1394A16
:102AF00000E00022DA631120114604F01DFE0AE016
:102B0000997D11203944C829A8BFC82121EAE17163
:102B1000997504F025FEB9F1110F00F0F7802E4BE6
:102B2000D3F8F49099F80030022B1AD138460FF000
:102B300045F82A490FF04AF9D9F838100EF08AFF03
:102B4000002107460FF02CFA30B9384621490FF022
:102B500045FA10B11F4F00E00027C9F83870142063
:102B60008DE099F8151014203944C829A8BFC82150
:102B700021EAE17189F815105EE0D3F8F49099F834
:102B80000030022B1AD138460FF018F811490FF017
:102B90001DF9D9F828100EF05DFF002107460FF04F
:102BA000FFF930B938460B490FF018FA10B1094F48
:102BB00000E00027C9F82870092060E099F80310A8
:102BC00009203944C829A8BFC82121EAE17189F840
:102BD000031031E00000C842640E002000007A4477
:102BE000D3F8F49099F80030022B1AD138460EF041
:102BF000E5FFBB490FF0EAF8D9F834100EF02AFFD0
:102C0000002107460FF0CCF930B93846B4490FF02F
:102C1000E5F910B1B24F00E00027C9F834700A207E
:102C20002DE099F80D100A203944C829A8BFC82101
:102C300021EAE17189F80D1004F092FD66E0D3F805
:102C4000F49099F80030022B1DD138460EF0B6FFF3
:102C5000A4490FF0BBF8D9F840100EF0FBFE00219C
:102C600007460FF09DF930B938469D490FF0B6F987
:102C700010B19B4F00E00027C9F840700B20394687
:102C800004F05AFD42E099F817100B203944C82986
:102C9000A8BFC82121EAE17189F81710CCE7012902
:102CA00034D19878904B33F91230B3F5617F05DB5E
:102CB00040F633029342A8BF134601E04FF461731C
:102CC000B9F10C0F22D14FF4966292FBF0F0A3F50C
:102CD000617393FBF0F3854ADFB21378BB4215D0E2
:102CE000042F34BF3B4602231370019A09FB0323D0
:102CF0007F4A03F2AE73136006F0D4FE48463946AD
:102D000004F02EFD781CC0B204F070FD94F8EC20A5
:102D1000012303FA0BF3134384F8EC300BF1010B9E
:102D2000BBF1040F0AF10C0A7FF411ADC5E433685E
:102D3000DB0511D56F4BDB7873B1D9F800309F07F5
:102D40000AD56D4B1B8813F001070AD10DF06AFEFE
:102D5000012006F0BFFD04E0012006F0ABFD0123D9
:102D600000E00023D8F8002050070DD563B1012002
:102D700006F0A0FD604B1B88990708D40DF052FEA9
:102D8000022006F0A7FD02E0022006F093FDD9F82C
:102D9000003013F00A0F29D0D8F80030DA060BD52E
:102DA000554B1B885B070AD4042006F093FD534B58
:102DB0001B88A4F8F83002E0042006F07BFDD8F868
:102DC00000309F0607D54C4B1B88580606D4402080
:102DD00006F080FD02E0402006F06CFDD8F80030DF
:102DE000590642BF454B1B88A4F8FA30D9F8003089
:102DF0009A0609D4D8F800301B0540F1B2804FF490
:102E0000807006F067FDB0E03D4BDFF8EC901B787A
:102E100013F0020F53D03B4B1B78042B4FD9D8F83B
:102E2000003013F4007A0FD0B9F80030DF063AD43E
:102E3000102006F04FFD202006F03CFD3248011D19
:102E400005F004FF02232AE0B9F8007007F010072C
:102E5000BFB22FB1102006F02DFD012784F8FCA091
:102E6000D8F80030580512D5D4F8003127495A89CE
:102E7000B1F90030002BB8BF5B42934207DAB1F9D9
:102E80000230002BB8BF5B429342C0F2F380B9F826
:102E90000030990608D5202006F00CFD002384F8A8
:102EA000FC30012700E0002794F8043193BB0E208A
:102EB00004F07AFC164B012283F804212AE0B9F8C9
:102EC000003003F03003002B94D0102006F0F2FC09
:102ED000202006F0EFFC002384F8FC301DE000BF4A
:102EE0000000C84200007A442C2F0020F02B002064
:102EF000CC10002004300020081A002044110020CB
:102F0000441900204A190020D41000204C11002040
:102F1000640E0020002F3FF46DAF00221446624B78
:102F2000002023F81400614B191D03F10A0721F852
:102F300014000021D15117447860B96023F81400BF
:102F400003F132075A33D151D150174413447860FA
:102F5000B960586099601432002C7FF44BAF0124A3
:102F6000DDE74FF4807006F0A5FC514B5A791C4602
:102F7000082A01D00E2A02D1402006F09BFC3368BB
:102F80005A0540F18D8094F814321BB92B7813F058
:102F9000040F03E0D8F8003013F4002F0AD0454B9B
:102FA00000221A703C200AF045FA002878D00CF074
:102FB000A1F9F7E70EF048F809B0BDE8F04F0AF0C4
:102FC00056B9012000E002205FFA80F8019A08F16A
:102FD000FF3382F8AC3706F0BFFC06F087FD4046B1
:102FE00004F004FCFFF710BBBAF1000F02D07E2BF7
:102FF0003FF408AB972B05D12F4B4FF4C8721A80C2
:10300000FFF702BBA72B06D12C4A137843F0040329
:103010001370FFF7F9BA0022BB2B079201D10223EC
:1030200003E0B72B04D14FF6FE73ADF81E300AE073
:10303000BE2B01D1022304E0BD2B7FF4E5AA4FF69D
:10304000FE73ADF81C30DBF80030BDF81C10B3F88F
:1030500058200A44A3F85820BDF81E10B3F85A208F
:103060000A44A3F85A2006F011FF002384F8BA306E
:10307000FFF7CABAB9F800309B063FF515AF20201C
:1030800006F028FC0E4B0F481A685B68011D436070
:10309000026005F0DBFD0C4B012783F8FC7003E7B1
:1030A00009B0BDE8F08F00BF4C3000206A0F00204F
:1030B0005411002011280020822A002044190020E9
:1030C0004C190020DC100020640E0020B54B2DE9C7
:1030D000F04FB3F90610B44B85B01F6801937A899D
:1030E00091420EDBB1F5FA6FFC79BFBF8B1A6343D7
:1030F000A2F5FA6493FBF4F4ACBFC4F16404643445
:1031000000E06424A94BAA4AB3F896B193F95E3162
:1031100012689BB2029215460393002240F2E630F9
:10312000A04B4FEA420C33F912E0CBEB0E0303F253
:10313000F316864203D8002BB8BF5B4201E04FF480
:10314000FA73022A2ED0029E96F811611EB1B34284
:10315000CCBF9B1B0023642093FBF0F8954E6FF0CF
:10316000630A36F818900AFB083A08F1010836F9A4
:1031700018600FFA89F8C8EB060606FB0AF696FBFC
:10318000F0F68D484E4420F80C60BE183679642065
:1031900073438A4E93FBF6F364339BB2634393FB12
:1031A000F0F02CE0029890F812611EB1B342CCBF4F
:1031B0009B1B0023642093FBF0F0DFF82C926FF050
:1031C000630808FB003A39F91060013039F9100042
:1031D000002BA0EB060000FB0AFA9AFBF8FA039812
:1031E000C6EB0A0A0AFB00FA7348B8BF5B42A0F8B4
:1031F00004A0B8794343714893FBF0F064306B78D6
:103200004FF06408434393FBF8F36D4E022AB35426
:10321000EB7A6C4E00FB03F393FBF8F3B3546B7D36
:10322000654E00FB03F090FBF8F0674B9854674B3A
:103230000ED1DE4583F802800DDB5C4CB4F898219A
:10324000914214DBB1F5FA6FA8BF4FF4FA610FE0B9
:10325000DE459C5404DA36F80C305B4226F80C301C
:103260000132032A05F101057FF458AFE5E7114665
:10327000891A4FF47A735943C2F5FA62B1FBF2F13D
:10328000642391FBF3F2DFF874E16FF063073EF81B
:10329000120007FB021101323EF9122007B2D21BC5
:1032A000514391FBF3F30344F380494B424D1B8898
:1032B0005F063BD5474A484B10881B88181A00B256
:1032C0000EF07CFC45490EF0CDFC074606F0E8FA0E
:1032D0008046384606F072FA0746B5F902000EF04D
:1032E0006DFC8146B5F900000EF068FC414682464F
:1032F0000EF0B8FC3946834648460EF0B3FC014652
:1033000058460EF0A5FB0EF073FE41462880484655
:103310000EF0A8FC3946804650460EF0A3FC01464C
:1033200040460EF097FB0EF063FE68802C4D2B6834
:10333000980740F19E8045F207212A4B2A4F1A68D0
:103340007B69D31A8B4240F394807A610AF0F6FBD2
:10335000264BDFF8AC901A789846032AB9F800306B
:1033600050D10A2B58D90023282088F8003004F0C7
:103370007CFA0AF0E3FB1E4B18880AF0C9FB1D4BD0
:103380001A68D37890FBF3F0013008281A4BA8BFD5
:1033900008201870537980B243433B831379584314
:1033A000788339E02C2F0020CC100020541100200D
:1033B000A4100020261A00204C1100200CFEFFFF54
:1033C00080210020FE0F00208821002008210020FD
:1033D000081A00205E0F00204411002035FA8E3CB0
:1033E000342E002038300020F00F002090190020EB
:1033F0008C2800202C190020300000200E1A0020FC
:10340000301900200A2B07D803238E4A88F8003091
:10341000002313703B837B8398F800308A4A012B8A
:103420000CD002D3022B1BD023E03A8BB9F800302A
:103430009A421EDD012388F800300FE0B9F8001031
:103440007B8B8B4202DD022313700FE07F4B1B8BC3
:103450000133994202DD002313700AE0082006E0E0
:103460007B8BB9F8002001339A42E3DC072004F09B
:103470009BF92D68290577D5754B744F1A68FB6940
:10348000C3EB020845F2072398456DDD714BB6F991
:1034900006B0D3F800904FF47A7099F80A30FA61C8
:1034A000012B98FBF0F8B4F84E11ABF57A7B6A4E1D
:1034B00003D042D3022B20D041E0684B396A5A7BBB
:1034C000674B4FF0080E33F8122091FBFEF392B2D7
:1034D000C91A8B183B6293FBFEF3BA8440F6E442B0
:1034E0009BB25343B9F80820C2EB13335843B9F9E0
:1034F000063090FBF3F0306021E05A4BB9F808A099
:103500001B78C6F800A05A0719D5574804F0F9F8F7
:1035100020B915F0100F18BF4FF0000B0BFB0BF389
:10352000322293FBF2F3B9F906205B445A434FF47D
:103530007A7392FBF3F3534400E000233360336863
:10354000D7E90A0103FB08F84FF47A7398FBF3F804
:1035500010EB080041EBE8710023C7E90A01434A78
:103560000EF08CFD424B1860424E3368DB0427D5C9
:103570002F0622D5404B1B789D071ED53F4B187850
:1035800004281AD900223E4B0521D718951C4FF06C
:103590000A0E122AD154E9B287F801E004D0B0EB48
:1035A000510F2A46EFD800E014215A18322002F8B1
:1035B000010CFF225A540F2000E00A2004F0F4F816
:1035C000304D2A68002A73D02F4B304F1868396865
:1035D000984681426CD82E4BDFF8C090187851681D
:1035E000B0B901221A70B9F80030CB5CD3B1294BC5
:1035F0001A700DF0F9FFB9F800309BB92B681B78F1
:10360000053B012B0ED804F009F9234B186009E0A3
:1036100000221A70B9F80030CB5C1BB11D4B1A7038
:103620000DF0E2FF2B68B9F800205B681B499B5C3A
:10363000FE2B02D100230B803AE0FF2B30D104F0A7
:10364000A3F835E03000002090190020F00F002092
:10365000383000202C190020381900207428002050
:103660008428002052300020DC120020407E05001B
:103670003C19002068100020441900204A1900203D
:103680001C2C0020401A0020582E0020381A002040
:10369000351A0020341A0020E82D00203C1A0020A2
:1036A000D8F800000A2505FB030301323B600A80BD
:1036B0009D4D2B7858073DD43268D1075CBF43F04D
:1036C00001032B70994B1B781F075EBF2B7823F0EB
:1036D00001032B70D60248BF2B78954A44BF23F0D4
:1036E00001032B70934B1B6813F0040F02D0924917
:1036F000098851B99149098809B1980705D4904BB7
:103700001B88003318BF012333B1022313702B78B9
:1037100023F001032B7004E02978C90758BF022366
:10372000137004F07BF8874B1B68C01A002801DB7C
:103730000DF05AFF0DF088FC834B1E789846002E42
:1037400000F0AA80814E3368002B00F0E3863068D9
:103750000AF011FA002800F0DD867C4B7C4C1868DA
:103760000AF006FA092801D03F2850D14FF0000A8C
:103770005746D4F80090774DB9F1000F05D0764840
:1037800029684A4611F070FC10B9AA4607B92F46BD
:10379000724B10359D42EFD3C7B1D7F800E0DAF88D
:1037A00000C023681EF803501CF80300A8420DD186
:1037B0005A1C694938B92D2B05D8654D2A6020253A
:1037C000CD54885402E0CD542260EAE723680BB15F
:1037D000574511D062480BF07DFE574507D857F882
:1037E000100B0BF077FE09200BF06CFEF5E75D483F
:1037F0000BF070FE4FF0000923689945A7D2564B95
:1038000013F809000BF05EFE09F10109F4E72368E3
:10381000002B40F06486042840F09D864E4806F058
:1038200065FC00F077BED9F80000DFF848A10AF087
:10383000A2F938B3DAF800000AF09AF9DBF80030A0
:10384000024693F84810002934D1242840F094808F
:10385000012283F84820DBF80030DFF814A193F848
:103860004820062ADFD193F8490001F0A1FD002885
:1038700000F0AD803B6898790BF079FD3B68002241
:1038800083F84820384B93F83530002B40F0FC8506
:103890004C36982E00F03E86344BF21892F84A10BF
:1038A0000129F5D1324FF3583A60324ABB461360D2
:1038B0009146B8E7012904D14D2814BF0022022205
:1038C000C7E7022904D13C2814BF00220322C0E725
:1038D00003290CD140284FF0000102D983F8481089
:1038E000B9E758711971D97198710422B1E70429A7
:1038F00006D1997983F849004A409A710522A8E7D0
:103900000529A8D1587919798842987906D9504063
:103910009871481C18710B441A729CE790420CBFB6
:103920000622002295E700BF5230002044190020F3
:10393000341A00204019002048300020822A00203C
:103940004A30002028300020533000200C2C00206A
:10395000E01C0020B4740108B01C0020647601084B
:10396000A88C0108AD8C0108F00F00207027002002
:10397000E8190020EC1900202B78D44958073FF5AE
:103980006AAF232ADAF8003014D1012088F8000049
:10399000CF4803910360CF4802920363CE480BF0F7
:1039A00099FDCE480BF096FD0399029A0B7843F0EF
:1039B00002030B70CA4B1B681B78934201BFC94AB4
:1039C000C94B1A60C94A04BFC94BDA6043E7DAF849
:1039D000002092F849304C2B00F0618450D8332BF2
:1039E00000F0988421D8292B00F0258409D8252BB4
:1039F00000F0FC83272B00F00084232B40F0A785E8
:103A000027E22D2B00F0288407D82B2B40F09F8530
:103A10000BF090FC607100F032BD2F2B00F0E784BA
:103A2000312B00F0F98400F092BD3C2B00F0E580D2
:103A300009D8372B00F0A384392B00F0EB83352B0A
:103A400040F085853EE2412B00F069840CD83E2B86
:103A500040F07D850BF06EFC84F8E0010BF06AFC11
:103A600084F8DF0100F00BBD432B00F06584442B8C
:103A700040F06D85974B012283F8352000F0FFBCA4
:103A8000D02B00F0168355D8CA2B00F0C58009D87A
:103A9000C82B00F0858000F243834E2B00F00C848D
:103AA00000F055BDCD2B00F00F8304D8CC2B00F0D7
:103AB000318200F04CBDCE2B00F00F83CF2B40F0B5
:103AC00046850BF041FC6FF4AF6283189BB2C62BA6
:103AD00098BFA4F896010BF037FCA4F840010BF056
:103AE00033FCA4F842010BF02FFCA4F844010BF0C6
:103AF0002BFCA4F8D8010BF01DFC84F8ED010BF0B1
:103B000019FC0BF017FC84F8EE010BF013FC84F8A1
:103B100085010BF00FFC84F892010BF00BFC754B48
:103B2000D3F800900BF010FC00EB80004000A9F8E7
:103B300056006FE3D62B00F040820AD8D22B19D062
:103B4000C0F01583D32B25D0D42B00F0428200F097
:103B5000FEBCEF2B41D005D8D82B40F0F8844FF0B5
:103B6000000909E1F22B00F07C82FA2B00F0BE8202
:103B700000F0EDBC2B78590700F181840BF0DAFBE3
:103B8000022884F8AC0740F29A825B4B002283F84B
:103B9000AC2794E20BF0D8FB584B188000F06FBCB8
:103BA00092F805904FEA5909B9F1120F03D909F0BB
:103BB0003DFC00F064BC4FF0000ACA4507D20BF090
:103BC000C3FB4F4B23F81A000AF1010AF5E7414BFA
:103BD000012283F8342000F052BCDFF81891D9F8A4
:103BE00000A00BF0B1FBAAF85A00D9F800900BF036
:103BF000ABFBA9F8580000F042BCDFF8F890D9F808
:103C000000A00BF097FB8AF80000D9F80030187874
:103C100008F09AFD00F033BC364B81461A689A468C
:103C20001278022A40F08D80DAF8003009F1080B92
:103C300002930BF07FFB0DF0BDFF32490EF0C6F88A
:103C4000029B43F82B00DAF800B00BF073FB09F18C
:103C50000A030BEB830B0DF0ADFF2B490EF0B6F80A
:103C6000DAF80030CBF8040002930BF063FB0DF0A0
:103C7000A1FF26490EF0AAF809F10E0B029B09F1EB
:103C80000109B9F1030F43F82B00CDD1B9F1070FAA
:103C9000DAF800B03CD10BF04DFB0DF08BFF194969
:103CA0000EF094F8CBF84400DAF800B00BF042FBC9
:103CB0000DF080FF13490EF089F8CBF84800DAF8D0
:103CC00000B00BF037FB8BF84C0034E05230002092
:103CD0000C2C0020F00F0020DD8C0108AD8C0108B9
:103CE00014280020EFBEADDEF04F00200400FA05DE
:103CF00000ED00E0A4100020541100205C0F002013
:103D00002C2F0020000020410000C84200007A440F
:103D10000BF010FBCB448BF80100DAF800B00BF08D
:103D200009FBCB448BF80B00DAF800B00BF002FB78
:103D3000CB448BF8150009F10109B9F10A0FA5D19F
:103D40009DE3DAF800B00BF0F5FACB448BF80100F4
:103D5000DAF800B00BF0EEFACB448BF80B00DAF88F
:103D600000B00BF0E7FACB4409F10109B9F10A0FF1
:103D70008BF81500E5D182E3DFF890A309F1080B79
:103D8000DAF8003002930BF0DFFA0DF013FFD94997
:103D90000EF01CF8029B43F82B00DAF800B00BF091
:103DA000D3FA09F10A030BEB830B0DF003FFD149A2
:103DB0000EF00CF8DAF80030CBF8040002930BF0A8
:103DC000C3FA0DF0F7FECB490EF000F809F10E0B27
:103DD000029B09F10109B9F1030F43F82B00CBD184
:103DE000B9F1070FDAF800B01AD10BF0ADFA0DF007
:103DF000E1FEC0490DF0EAFFCBF84400DAF800B06C
:103E00000BF0A2FA0DF0D6FEBA490DF0DFFFCBF8A9
:103E10004800DAF800B00BF097FA8BF84C0012E08B
:103E20000BF092FACB448BF80100DAF800B00BF0FB
:103E30008BFACB448BF80B00DAF800B00BF084FA65
:103E4000CB448BF8150009F10109B9F10A0FC7D16C
:103E500015E30BF06FFA132883463FF6A8AEDFF8A0
:103E6000ACA2DAF800900BF065FA0023A2490C220C
:103E700002FB0312117A814220D1137809EB8B09DE
:103E800089F879300BF056FA89F87A000BF052FA7B
:103E900089F87B000BF04EFA984A994B89F87C0020
:103EA0001A60DAF80000974B00211860793003F0AF
:103EB00017FC954B80F001001870E0E201331C2BD9
:103EC000D4D174E60BF036FA0B2882463FF66FAE7B
:103ED0008E4BD3F800900BF02DFA03283FF667AE17
:103EE000062303FB0A9989F8CE000BF023FA89F820
:103EF000C9000BF01FFA89F8CA000BF01BFA89F809
:103F0000CB000BF017FA89F8CC000BF013FA89F804
:103F1000CD00B4E25379092B7FF649AE019BD3F86B
:103F200000900BF007FA019B89F80000D3F800908D
:103F30000BF000FA89F801000BF0FCF9019B6428F2
:103F40001B68A8BF642018710BF0F4F9019B64286A
:103F50001B68A8BF642058710BF0ECF9019BFF2887
:103F60001B68A8BFFF2098710BF0E4F9019B64283F
:103F7000D3F8009028BF642089F807000BF0DAF925
:103F8000019B89F80200D3F800900BF0D3F9019B54
:103F900089F80300D3F800900BF0D6F93B68A9F834
:103FA0000A005B790A2B40F26A82594BD3F80090E1
:103FB0000BF0C0F989F8080061E281460BF0C4F902
:103FC000544B23F8190009F10109B9F1080FF5D193
:103FD00055E253790F2B7FF4EAAD0BF0ABF90728CC
:103FE00081463FF6E4ADDFF824A1DAF800B00BF02B
:103FF000ABF90E2303FB09F9CB44ABF81901DAF84E
:1040000000B00BF0A1F9CB44ABF81B01DAF800B01B
:104010000BF09AF9CB44ABF81D01DAF800B00BF0C5
:1040200089F9CB448BF81F01DAF800B00BF082F964
:10403000CB448BF82001DAF800B00BF07BF9CB44CD
:104040008BF82101DAF800B00BF074F9CB448BF84F
:104050002201DAF800A00BF081F9D144C9F823015C
:104060000DE20BF067F90F2881463FF6A0AD0BF08B
:1040700061F9C9EBC909A14489F8D0000BF05AF9DC
:1040800089F8D1000BF056F989F8D2000BF052F9FB
:1040900089F8D3000BF04EF989F8D4000BF04AF9F7
:1040A00089F8D5000BF046F989F8D60009F02AFF07
:1040B000E5E12B785B0700F1E2810BF037FC05F0BE
:1040C0004BFC05F013FDDAE12B78580700F1D7819E
:1040D000114B4FF4C8721A80D1E12B78590700F1C7
:1040E000CE810E4A137843F004033EE02B785A0742
:1040F000E5D52CE200007A44606E0108941200209D
:10410000540F0020580F002009000020A4100020A8
:10411000CC100020F22B0020822A0020441900201D
:104120000BF008F9DD4B1A7810B142F0020201E001
:1041300022F002021A700BF0FDF8D94BDFF88493DD
:1041400018700BF00BF9C9F800000BF007F9C9F86B
:1041500004000BF0F9F8D34B18800BF0F5F8D24BB4
:10416000D24A1880137843F00203137087E10BF0F2
:10417000E1F802900BF0F2F883460BF0EFF882467C
:104180000BF0ECF881460BF0DFF80BF0DDF80BF0EC
:10419000D1F8029BA3B9C64B1020C3F800B0C3F8F6
:1041A00004A005F087FBBD4A137843F001031370A8
:1041B000B9F1000F00F06381BE4BC3F800905EE1DF
:1041C000102B40F05C81BC4BC3F800B0C3F804A0D6
:1041D000B9F1000F02D0B74BC3F80090B648B74B07
:1041E0000222011D1A7004F031FD48E1A0600BF0BD
:1041F000B5F8A3681843A06041E10BF0A5F8A4F856
:1042000058010BF0A1F8A4F85A010BF09DF8A4F89E
:104210005C0134E10BF08EF884F87A010BF08AF837
:1042200084F87E010BF086F884F87D010BF082F8AB
:1042300084F87F0123E10BF087F8A4F880010BF0EC
:1042400083F8A4F882010BF075F884F884010BF070
:104250007BF8A4F8860112E10BF06CF884F8900169
:104260000BF072F8A4F89A010BF06EF8A4F896011E
:104270000BF06AF8A4F898010BF05CF8DAF800305B
:1042800084F891015B79082B40F2F9800BF05CF81F
:10429000A4F89C010BF058F8A4F89E01EFE00BF095
:1042A00049F884F8D6010BF045F884F8D7010BF0F3
:1042B0004BF8A4F8D801E2E092F805900323B9FB8B
:1042C000F3F9B9F1120F3FF672ACDFF8FCA14FF031
:1042D000000BCB4580F0D3800BF02CF88AF8A001BE
:1042E0000BF032F840F2ED23984205DD40F6CA03A8
:1042F0009842A8BF184601E040F2EE20A0F2EE205E
:10430000192390FBF3F00BF1010B8AF8A1010AF1DC
:10431000020ADEE70BF00EF884F89201AFE0814666
:104320000BF008F804EB090309F10109B9F1080FD2
:1043300083F88801F4D1A2E00AF0FCFF0023A36017
:1043400060710BF00BF8A3681843A0600AF0F2FF4D
:1043500084F890010AF0F8FFA4F858010AF0F4FF7D
:10436000A4F85A010AF0F0FFA4F85C010AF0ECFF8F
:10437000A4F880010AF0E8FFA4F882017FE05379F5
:104380004FF0070AB3FBFAF2C2EBC2029A1A12F01C
:10439000FF0F7FF40CACB3FBFAFA0AF1FF3A5FFAB5
:1043A0008AFABAF1FF0F6AD00AF0C4FF5FFA80FB05
:1043B0004FFA8BF003F02EF8814600283FF4F7AB5C
:1043C00080F800B00AF0C0FFA9F802000AF0B2FFBE
:1043D00089F804000AF0AEFF89F805000AF0AAFF88
:1043E00089F807000AF0A6FF89F80600D5E7DFF88C
:1043F000D89009F1400A0AF0A7FFA9F8A4020AF030
:1044000099FF89F8A6020AF095FF09F1040989F8D5
:10441000A302D145EFD132E00AF08CFF1F2881467C
:104420003FF6C5AB3B685B79082B7FF4C0AB0AF065
:104430008BFF09F1880904EB890900F03F00A9F816
:1044400006000AF081FFB9F80630800100F4FE5042
:104450001843A9F806000AF06DFF000189F804006E
:104460000AF068FF99F8043000F00F00184389F84B
:1044700004000AF05FFF89F805000AF067FA0020DF
:104480000AF0A4FFFFF7F6B90D4B985903F07CFA38
:10449000E0B9322003F0E9F9F6E700BF4419002043
:1044A0004A1900204819002046190020D210002087
:1044B000D4100020E4100020DC100020600F002049
:1044C000702700204C1900205411002009F0DAFC5C
:1044D00005F018FA524A534BDA60FFF7D9B90C28A5
:1044E0003BD00A2842D1504D50480AF0F3FF2846ED
:1044F000232110F0A2FD08B1401B20602368002B8F
:1045000057D1494800213022236010F060FD98F80F
:1045100000302BBB464B1B689B060FD5454B4649CD
:104520001B688A6B9A1A002A08DB444A1278042A0C
:1045300082BF03F5123303F5F8738B63404B9B681E
:10454000002B69D03F4805B0BDE8F04F184708F090
:104550006DFFFFF78FB90C2804D13B480AF0BAFF72
:104560003A480DE07F2812D1FFF7F1B80D28BAD0F4
:104570007F2809D12C4A013B002135482360D154C2
:104580000AF0A8FFFFF7E3B82F2B3FF6E0A8A0F151
:104590002002D2B25E2A3FF6DAA813B920283FF4EF
:1045A000D6A85A1C2260204AD0540AF08BFFFFF78D
:1045B000CEB85A1EA95C202901D113469FE71A4A9A
:1045C00000212360D154234B234DD3F800A0D5F80C
:1045D00000B0DFF85490584610F03DFD07465946AC
:1045E0003A46484610F040FD1C4A28B919F80730F1
:1045F00053445B785B0703D010359542E7D306E060
:10460000954204D2781CEB684844984702E014486D
:104610000AF060FF002374E705B0BDE8F08F00BF2B
:104620000400FA0500ED00E0B01C002055980108D8
:104630004019002038300020F00F00204A190020D7
:10464000002E00202C100020B28C0108AD8C010837
:10465000D98C010844000020B47401086476010874
:10466000BD8C01088F4A70B51368988A80B2C1B2B8
:10467000CE072ED5198821F400610904090C198090
:10468000198889B241F48061198000211171517932
:1046900099B1917911B9D179FF290ED10121917187
:1046A000117A022901BF198889B241F40061198089
:1046B000517A41F001011982DFE0517A01F0FE01E7
:1046C0001982D379FF2B00F0D880764BFF21197126
:1046D000D3E08D073AD5BFF35F8F107AC0B20128BF
:1046E00013D1517989B1917979B1198821F4806117
:1046F0000904090C1980BFF35F8F198B1988907218
:1047000089B241F4007119801BE0198BBFF35F8FF0
:10471000107A644902280AD1487940B1897931B1C7
:10472000198821F480610904090C19809FE0107A2E
:104730005C49032805D1487918B18979002940F0EE
:104740009680998889B241F4806195E04C0754D5F0
:10475000012191725179002936D09179002933D005
:10476000117A1888022911791CD920F4806000047C
:10477000000C18801C8AD568C8B2E4B249B26C54E7
:10478000198889B241F400711980811C1171198A4C
:104790000130C9B240B22954998889B241F480618C
:1047A000998026E080B240F4007018801C8AD56899
:1047B000C8B2E4B249B26C541C8A411C49B2E4B29A
:1047C00003306C54107114E09179364809B9017CBA
:1047D00041B1198889B241F4007119801179013110
:1047E000117106E0198889B241F4807119800121A4
:1047F00081711988C905FCD43FE001F0400101F046
:10480000FF04E1B110791E8AD568C4B2611C40B2C0
:10481000F6B22E54C9B2157A117149B2C81C85423C
:1048200001BF988820F480600004000C08BF9880C5
:10483000137A8B4221D11B4B02341C711DE00606FA
:104840001BD5117948B2451C0AD054690131205C4E
:10485000C9B21882107A117149B288420DD106E0AE
:10486000D17914711982517909B9117A29B99988C4
:1048700021F480610904090C9980117A92F90400ED
:1048800001318842074B0CD100219971997A31B1DD
:1048900019688B8823F440731B041B0C8B80002346
:1048A000137670BD301000202DE9F04FDFF85892DC
:1048B00085B00746D9F81C000E460DF07FF98E4CE6
:1048C000804620880DF076F94FF05C510546404651
:1048D0000DF0C8F94FF06451824628460DF0C2F938
:1048E000014650460DF0B4F84FF062518246404602
:1048F0000DF0B8F94FF06A51804628460DF0B2F934
:10490000014640460DF0A4F80546B4F902000DF04A
:1049100055F9014628460DF0A5F951460546504681
:104920000DF0A0F98046B4F904000DF047F90146F6
:1049300040460DF097F9014628460DF08BF8804669
:104940000DF056FB6D490546A06140460DF03EFA5C
:10495000D9F820308046284601930DF02FF94FF00A
:104960007C510DF07FF966490DF072F80546E38938
:10497000B4F90A0002930DF021F929460DF072F9FD
:1049800029460DF06FF94FF058510DF06BF9814643
:10499000B4F90800B4F810B0B4F80CA00DF00EF99A
:1049A00029460DF05FF9014648460DF053F84FF0E7
:1049B00058510DF057F94FF060510DF053F94FF089
:1049C0007E510DF047F88146E0880DF0F3F801467E
:1049D00048460DF047F9002181460DF0D7FA00282E
:1049E0007BD1294628460DF03DF903900FFA8BF054
:1049F0000DF0E4F8039B014618460DF033F94FF033
:104A000060510DF02FF98346BDF908000DF0D6F87E
:104A1000014628460DF026F901460DF01BF8014627
:104A200058460DF017F84FF07A510DF01BF98346F8
:104A300001980DF0C3F801464FF093400DF008F8CF
:104A400005460FFA8AF00DF0B9F84FF08F410DF0DE
:104A500009F9014658460CF0FDFF4FF066510DF084
:104A600001F9014628460CF0F3FF26490DF0FAF84B
:104A700049460DF0ABF90546B4F916000DF09EF865
:104A800029460DF0EFF829460DF0ECF84FF04051B3
:104A90000DF0E8F88146B4F914000DF08FF80146E6
:104AA00028460DF0DFF84FF060510DF0DBF80146BD
:104AB00048460CF0CFFF8146B4F912000DF07EF8A5
:104AC000014648460CF0C6FF4FF076510DF0CAF88B
:104AD000014628460CF0BEFF00E0002017B10DF0A3
:104AE00087FA38602EB140460DF082FA64235843AD
:104AF000306005B0BDE8F08FD00A00200000A0456E
:104B000000007A470050C3453010002070477047BE
:104B10002DE9F041324C334D6289AB8CB4F90480FD
:104B20009A1A2389B4F902E05A43B4F91230D61321
:104B3000B4F91420DB02324493FBF2F232440A2629
:104B4000E2615643A2F57A6202FB02F3B4F90EC0A9
:104B500002FB0EFE02FB08F2B4F90C801B130CFBE7
:104B600003FC03FB08F31B1403EB62320232E388FD
:104B7000921002F5004253434CF25032B4F92070C7
:104B80004FEAEE2EB4F900400EEBEC2C0CEB840453
:104B9000BC40AD6A0234A5EBA4043A4162434FEA3B
:104BA000D3384EBFB2FBF8F35400B4FBF8F340F631
:104BB000DE3448BF5B001A12524362430A4C083687
:104BC0005C43241404EB224202F6CF62361103EB5D
:104BD000221300B1036001B10E60BDE8F08100BF97
:104BE000A80A00203010002043E3FFFF064B93F893
:104BF0002C2002F0FF012AB101220270002283F86A
:104C00002C2070470170704730100020104B13B5F6
:104C100093F82D201C46CAB90E4B1B68B3B11A6815
:104C20001AB10D49886902438A619A889868ADF87B
:104C3000042002228DF8072004220DEB02018DF8DA
:104C4000062008F00DF8012384F82D3002B010BDC5
:104C500030100020A00A00200010024008B5FFF725
:104C6000D5FF074B1B7813B1012B03D008BD4FF4C0
:104C7000006201E04FF48052024B1A8008BD00BF71
:104C8000A40A00200A000020012828BF01202DE9E5
:104C9000F04F0646142000FB06F3704F89B0F91858
:104CA000FC586F4B0A691C6083F82E606D4BB1F89D
:104CB0000880DD69B1F80AA02A43DA61A2884D684C
:104CC00022F440721204120C4AEA0809A28003A9D5
:104CD000C5F8109002228DF80E0028460193ADF819
:104CE0000C908DF80F2007F0BBFF019B00971F462B
:104CF0004FF0080BAA6818EA020F03D10A2002F04D
:104D0000A9FDF7E70A20C5F8148002F0A3FDC5F855
:104D100010800A2002F09EFDBBF1010BEAD1C5F81C
:104D200014A00A2002F096FDC5F814800A2002F0B3
:104D300091FDC5F810800A2002F08CFD0222C5F812
:104D400010A0284603A98DF80F201C228DF80E20F4
:104D5000ADF80C9007F084FF434A03A894423A69E7
:104D60000BBF42F4001242F480023A613A610BBF79
:104D70003A693A6922F4001222F480023A61A38867
:104D800023F440731B041B0CA38023889BB243F0C5
:104D900001032380A58808F015FC0599334B25F005
:104DA0003F05B1FBF3F32D042D0C1D43ADB2A580DF
:104DB0002288002522F001021204120C22802C4AC3
:104DC00003A8B1FBF2F100298AB208BF012242F424
:104DD00000414FF4967253434FF47A7293FBF2F30F
:104DE00001339BB22384A1832388009A9BB243F0B2
:104DF00001032380238823F4816323F002031B042F
:104E00001B0C23804FF480432381142303FB0626CD
:104E1000737B01248DF80C308DF80D508DF80E50F9
:104E20008DF80F400BF02AFE337B9DF80F208DF894
:104E30000C308DF80D508DF80E501AB103A80BF000
:104E40001DFE08E05A0903F01F039C4002F12003F5
:104E5000084A42F8234009B0BDE8F08F086E010807
:104E600030100020001002400054004040420F006B
:104E7000804F120000E100E010B5214C2368998AB0
:104E800089B211F4706F1CBF012284F82F2011F435
:104E9000E06F2BD01A8B9A88890522F480624FEA42
:104EA00002424FEA12429A8020D41A8892051DD4F9
:104EB0001A88D0050FD51A88D105FCD41A8892B269
:104EC00042F400721A801A889205FCD494F82E00DD
:104ED000FFF7DAFE0AE01A8892B242F400721A80F2
:104EE0009A8822F440721204120C9A802268938AE3
:104EF00023F470631B041B0C93820023237610BDE4
:104F000030100020064A08B5138801339BB2138085
:104F1000044B93F82E00FFF7B7FE002008BD00BF3A
:104F2000661000203010002010B540001C4CC0B2AC
:104F30006072E1710120002121746071227220767B
:104F40002068E360636184F82F1040B383889B0579
:104F500015D40388D9050DD447F230530288920541
:104F600002D5013BFAD112E08BB103889BB243F426
:104F70008073038083889BB243F44073838047F23D
:104F80003053227E12B1013BFBD100E013B9BDE8E2
:104F90001040B7E7024B93F82F0080F0010010BDDE
:104FA0003010002007B5F7216B4606227620FFF768
:104FB000BBFF9DF800309DF801101B0343EA01136D
:104FC0009DF80210094A43EA111313629DF8033059
:104FD0009DF804101B0343EA01139DF8051043EAF2
:104FE0001113D36103B05DF804FB00BF3010002043
:104FF00007B5F62101AB03227720FFF795FF9DF857
:1050000005309DF804201B0243EA02439DF8062068
:105010001343054AB2F92020C2F10802D340034AE3
:10502000936203B05DF804FBA80A00203010002052
:1050300007B5F62101AB02227720FFF775FF9DF837
:1050400004209DF8053043EA0223024A938403B00A
:105050005DF804FB3010002013B5062204464321FE
:1050600068206B46FFF760FFA8B19DF800209DF80F
:105070000130012043EA022323809DF802209DF89D
:10508000033043EA022363809DF804209DF8053035
:1050900043EA0223A38002B010BD13B506220446E2
:1050A0003B2168206B46FFF73FFFA8B19DF8002029
:1050B0009DF80130012043EA022323809DF802205D
:1050C0009DF8033043EA022363809DF804209DF895
:1050D000053043EA0223A38002B010BD13B51F4B75
:1050E0004000C0B2587202AC1868D97104F8012DA2
:1050F000002101221A745C615971DC601A721A76FF
:1051000083F82F1040B38288920515D40288D40505
:105110000DD447F230520188890502D5013AFAD1FF
:1051200012E08AB1028892B242F4807202808288D0
:1051300092B242F44072828047F23052197E11B12D
:10514000013AFBD100E012B9FFF7DCFE04E0034BAB
:1051500093F82F0080F0010002B010BD3010002045
:105160002DE9FF415B4B1B689BB11A681AB15A4984
:10517000886902438A619A889868ADF804200222FF
:105180008DF8072004220DEB02018DF8062007F0B0
:1051900067FD322002F069FB002111221E20FFF77B
:1051A0009DFF012160221E20FFF798FF642002F07E
:1051B0005CFB002402A807F091FB274626460A253F
:1051C000022101221E20FFF789FF322002F04DFB51
:1051D00002A807F083FBBDF90820BDF90A101444AA
:1051E0008A42A8BF0A46BDF90C300F4493421E44C0
:1051F000A8BF134613F5805F04DD013DE0D14FF0F9
:10520000010801E04FF000081E2000211222FFF7E4
:1052100065FF0A25022101221E20FFF75FFF3220D1
:1052200002F023FB02A807F059FBBDF90820BDF9E5
:105230000A10A41A8A42A8BF0A46BDF90C307F1A88
:105240009342A6EB0306A8BF134613F5805F02DD69
:10525000013DDFD101E04FF0000820460CF0AEFC2C
:1052600001461E480CF0B2FD1D4D20F000402860A4
:1052700038460CF0A3FC014618480CF0A7FD20F0BE
:105280000040686030460CF099FC014615480CF06F
:105290009DFD20F00040A860002170221E20FFF735
:1052A0001DFF012120221E20FFF718FF1E200221D2
:1052B0000022FFF713FF642002F0D7FAB8F1000FC5
:1052C00004D14FF07E532B606B60AB6004B0BDE83F
:1052D000F08100BFF00A00200010024000406F463D
:1052E0001000002001C05E467620F4213122F5E650
:1052F000044B772093F82020F4219201343202F0FD
:10530000FC02EBE6A80A00207720F4212E22E5E635
:1053100008B5FFF77BFC6B2180226820FFF7DEFEDB
:10532000642002F0A2FA6B2103226820FFF7D6FE68
:105330000F4B19211A786820FFF7D0FE0F2002F0DA
:1053400094FA0C4B1A211A786820FFF7C7FE1B212C
:1053500018226820FFF7C2FE1C2110226820FFF7E8
:10536000BDFEBDE80840682037210022B6E600BF38
:10537000EC0A002008000020FFF774B97CE5FFF775
:1053800071B979E507B5232002F06FFA682075211D
:1053900001220DF10703FFF7C7FD28B19DF80700B3
:1053A000A0F168035842584103B05DF804FB00BF08
:1053B0004D282DE9F047044600F02A8600F2968039
:1053C000302800F0BD8651D8222800F0628423D80E
:1053D000032800F0CA8114D8012800F0BA810228FD
:1053E00040F0ED86042009F0F1FF432009F0BFFFF3
:1053F0004C2009F0BCFF462009F0B9FF4C2000F01A
:105400002CBE042800F0BA81052840F0D8861A2066
:1054100009F0DCFF0024D9E1282800F0B88515D870
:10542000242800F09B85262840F0C986DB4C062006
:1054300009F0CCFFB4F8580109F0CBFFB4F85A01D9
:1054400009F0C7FFB4F85C0100F085BD2C2800F01E
:10545000B1852E2800F048862A2840F0B086012029
:1054600009F0B4FFCD4B587900F0F7BD3B2800F0B0
:1054700009841CD8362800F01E860BD8322800F08C
:10548000E685342840F09B86482009F09FFF0025E0
:1054900000F021BC382800F067853A2840F08F865C
:1054A000042009F093FFBE4B186E00F083BE422823
:1054B00000F0E0850BD83D2800F0AB82402840F09A
:1054C0007E86082009F082FF002400F0C9BD46282E
:1054D00000F05B864B2800F08C85452840F06F86F5
:1054E000132009F073FF002400F059BE702800F06B
:1054F000E58200F2E180692800F0468200F2B28085
:10550000662800F0A08100F2A280642800F0778174
:10551000652840F05486A24C0B2009F057FF2088E4
:1055200009F057FF608880B209F053FF9D4B1B685C
:10553000C3F3C000C3F38002800040EA4200C3F31B
:1055400040021043C3F3401240EAC20003F01003CC
:10555000184309F03EFF944B1A88636802F0080173
:1055600003F4475949EA010903F4804149EA010972
:1055700003F4004149EA010903F4803149EA0109D1
:1055800003F4003149EA010903F4802149EA0109E1
:1055900003F4002149EA010903F4801149EA0109F1
:1055A00003F0007349EA0303DFF81C9212F0010FC5
:1055B00099F8009018BF4FF00208C9F3800908BF9E
:1055C0004FF0000843EA090312F0020F43EA080310
:1055D00014BF4FF0040C4FF0000C12F0040F43EA1C
:1055E0000C0C14BF4FF0100E4FF0000E12F0400FD5
:1055F00014BF202700274CEA0E0E12F0100F14BF24
:105600004FF4007600264EEA070712F0200F14BF71
:105610004FF4806500253E4312F4807F14BF4FF4A1
:1056200000600020354312F4007F14BF4FF40011D6
:105630000021284312F4806F41EA000114BF4FF0AB
:105640008063002300201943247A0346E7E067289B
:1056500000F02181682840F0B285102009F0B6FEE4
:10566000002488E16C2800F0A28117D86A2800F095
:10567000F8836B2840F0A385052009F0A7FE4B4B6B
:10568000188809F0A6FE4A4B188809F0A2FE444B80
:1056900093F86E0000F0010000F0DFBC6E28404D72
:1056A00000F0928100F2C081062009F08FFEE86DC3
:1056B00009F098FE3F4B85E1782800F0F98018D872
:1056C000742800F029830AD8722800F08A8373288E
:1056D00040F07585082009F079FE0124BAE37628A8
:1056E00000F0DF8300F251832F2009F06FFE324C6F
:1056F000C0E2A42800F0FB8314D87B2800F060826D
:10570000A02840F05C850C2009F060FE2B4B186847
:1057100009F068FE2A4B186809F064FE294B1868E6
:1057200000F048BDF12800F0FF80FE2800F006845C
:10573000F02840F044851A4C042009F047FE236C01
:10574000B3F85A0009F045FE236CB3F8580000F096
:1057500002BC032009F03AFE002009F008FE2046B2
:1057600009F005FE0D2000F078BC09F02FFE0120A5
:1057700009F0FDFD0A2009F0FAFDB6E3062009F064
:1057800025FE4F2009F0F3FD4C2009F0F0FD4920E3
:1057900009F0EDFD312009F0EAFDDBE354110020B2
:1057A0006410002040190020081A0020BE190020B3
:1057B000C01900203C1100202F6E0108E8F7FF1FE0
:1057C000ECF7FF1FF0F7FF1F52300020AA4B185DC7
:1057D000013409F0CCFD0B2CF8D10024A74B185D47
:1057E000013409F0C4FD082CF8D10024A44B185D45
:1057F000013409F0BCFD072CF8D100F0DDBC072016
:1058000009F0E4FDE72009F0B2FD9E4B587909F05C
:10581000AEFD002009F0ABFD042000F0CBBCA3429C
:105820000AD2994A9D5C012202FA05F50D421CBF7D
:105830009A4010430133F2E709F0D4FD914B93F8FD
:10584000AC0700F00ABC122009F0C0FD8F4B002409
:105850001B88B3F5806F8CBF082501258C4B33F96D
:105860001400013490FBF5F080B209F0B2FD032C76
:10587000F4D1884CA08C09F0ACFDE08C09F0A9FDB6
:10588000208D09F0A6FD608D09F0A3FDA08D09F023
:10589000A0FDE08D5FE3102009F098FD00247E4B11
:1058A000185D013409F063FD102CF8D100F084BCC0
:1058B000702009F08BFD00260E247443754D0136CF
:1058C0002B6C2344B3F8190109F083FD2B6C23449E
:1058D000B3F81B0109F07DFD2B6C2344B3F81D01C7
:1058E00009F077FD2B6C234493F81F0109F03FFD6D
:1058F0002B6C234493F8200109F039FD2B6C2344D1
:1059000093F8210109F033FD2B6C234493F8220115
:1059100009F02DFD2B6C1C44D4F8230109F062FD25
:10592000082EC9D100F048BC702009F04FFD554C3D
:1059300004F1700594F8D00009F019FD94F8D10035
:1059400009F015FD94F8D20009F011FD94F8D30088
:1059500009F00DFD94F8D40009F009FD94F8D50084
:1059600009F005FD073494F8CF0009F000FDAC42C2
:10597000E0D100F021BC494B185D013409F0F7FC7F
:10598000102CF8D100F018BC454D002428784000B8
:1059900000F0FE0009F01AFD2B789C4280F00C8488
:1059A000404B33F8140009F014FD0134F4E73E4C89
:1059B000062009F00BFD208809F00BFD608809F036
:1059C00008FD3A4B1888C6E2072009F0FFFC384B67
:1059D0001888FF28A8BFFF20C0B209F0C8FC354BCB
:1059E000186880F3100080B209F0F3FCB5F8640089
:1059F00009F0EFFC234B93F885212F4B186822B157
:105A00000A23584380F3100001E000F30F0080B236
:105A1000A1E21C4C022009F0D9FC94F8E00109F045
:105A2000A6FC94F8DF0118E30B2009F0CFFCAB6E65
:105A30000026187809F09BFCAB6E587809F097FCAB
:105A4000AB6E144C33441879013609F090FC032EE8
:105A5000F6D1A36ED87909F08AFCA36E987809F084
:105A600086FCA36ED87809F082FCA36E588909F0F1
:105A7000B0FCA36E187AF0E2F2880108FE880108F3
:105A8000D3880108541100206D1000200A00002066
:105A9000361100206410002094100020A81000206F
:105AA0000C2800202C2F00202A2E0020441100203A
:105AB000301900203C19002038190020C04C1E204D
:105AC00009F084FC236C00251B78022B65D1236C24
:105AD00005F1080253F82200BA490CF0C3F80FF0A0
:105AE00083FC80F30800C0B209F041FC236CB64986
:105AF00003EB8503D86A0CF0B5F80FF075FC80F362
:105B00000800C0B209F033FC236C05F10E0253F813
:105B10002200AE490CF0A6F80FF066FC80F30800F6
:105B2000C0B2013509F023FC032DD0D1072D236C21
:105B300021D1586CA3490CF095F80FF055FC80F377
:105B40000800C0B209F013FC236C9E49986C0CF05D
:105B500089F80FF049FC80F30800C0B209F007FC97
:105B6000236C93F84C000CF025F80FF03DFC80F30B
:105B70000800C0B20BE02B44587809F0F8FB236C06
:105B80002B44D87A09F0F3FB236C2B44587D013564
:105B900009F0EDFB0A2DC9D10EE3236C2B44587894
:105BA00009F0E5FB236C2B44D87A09F0E0FB236C69
:105BB0002B44587D013509F0DAFB0A2DEDD1FBE2CB
:105BC0003C2009F003FC00247D4D04F108022B6CFD
:105BD0007E4953F822000CF045F80FF005FC80B226
:105BE00009F0F7FB2B6C794903EB8403D86A0CF0BE
:105BF00039F80FF0F9FB80B209F0EBFB2B6C04F1E4
:105C00000E0253F8220071490CF02CF80FF0ECFB57
:105C1000013480B209F0DDFB032CD5D1072C2B6CAD
:105C200016D1586C69490CF01DF80FF0DDFB80B2FD
:105C300009F0CFFB2B6C6549986C0CF013F80FF052
:105C4000D3FB80B209F0C5FB2B6C93F84C000BE042
:105C50002344587809F0BDFB2B6C2344D87A09F013
:105C6000B8FB2B6C2344587D013409F0B2FB0A2C9D
:105C7000D4D1A1E214F8010F002800F09D8209F0B0
:105C800076FBF7E7012009F0A1FB4D4B1B6C187860
:105C9000E3E1502009F09AFB0025494B0C211C6CD4
:105CA0004B4B04EB850494F87920013501FB02335A
:105CB00093F8380009F05BFB94F87A0009F057FB81
:105CC00094F87B0009F053FB94F87C0009F04FFB3B
:105CD000142DE2D170E23A4B1C6C062303FB054401
:105CE00094F8CE0009F043FB94F8C90009F03FFB9B
:105CF00094F8CA0009F03BFB94F8CB0009F037FB9D
:105D000094F8CC0009F033FB013594F8CD0009F08C
:105D10002EFB0C2DDFD14FE24FF0000801260027AB
:105D2000274B1A7A974227DA0933FA5C00240C23AE
:105D30006343274D05F13001595C914207D12B4453
:105D4000586B0FF088F982462EB9B14605E0013450
:105D50001C2CECD10EE080440CE0D1450ADA0C2377
:105D600003FB04535B6B13F8090009F000FB09F116
:105D70000109F2E70137D3E7002E00F01D825FFA38
:105D800088F009F023FB0026C9E70D4D0024287A8E
:105D900009F01CFB2B7A9C4280F00E820D4B0021F7
:105DA000E65C0C2202FB01F3094800F13007DA5DE2
:105DB000B24211D1034493F8380009F0D8FA0EE04A
:105DC00064100020000020410000C84200007A4416
:105DD000306E01086D10002001311C29E1D1013421
:105DE000D8E7CC4C162009F0F1FAB4F8960109F086
:105DF000F0FAB4F8400109F0ECFAB4F8420109F005
:105E0000E8FAB4F8440109F0E4FAB4F8D80109F06A
:105E1000E0FA94F8ED0109F0AAFA002009F0A7FAD7
:105E200094F8EE0109F0A3FA94F8850109F09FFABD
:105E300094F8920109F09BFA002009F098FAB64B09
:105E40000A201B6CB3F9563093FBF0F080B209F0D6
:105E5000C0FA8DE0E0B2013409F089FA092CF9D1D9
:105E6000AAE1102009F0B2FAAC4BAD4C187800F062
:105E7000020009F07CFAAB4B187809F078FA206838
:105E800009F0B0FA606809F0ADFAA74B188809F07C
:105E9000A0FAA64B188809F09CFA9F4BB3F86C0047
:105EA00059E009F047FA0746122009F08FFA9A4C98
:105EB00017B9266F656F05E0102F19BF00252E4614
:105EC000A66FE56F384609F052FA304609F08AFAB3
:105ED000284609F087FAD4F8800009F083FA0020F8
:105EE00009F077FA002009F074FA0020B5E08A4D35
:105EF000002495F884002E4680000130C0B209F0DD
:105F000065FA95F8840009F032FA96F884309C42DC
:105F100080F05281864D285D09F029FA05F11003C1
:105F2000185D09F024FA05F12003185D303509F0F9
:105F30001EFA285D09F01BFA0134E6E7082009F093
:105F400045FA002009F045FA002009F042FA002045
:105F500009F03FFA002009F03CFA2DE1042009F095
:105F600035FA6C4B986825E1042009F02FFA694C4A
:105F700094F87A0109F0FBF994F87E0109F0F7F939
:105F800094F87D0109F0F3F994F87F0165E0614C24
:105F9000072009F01BFAB4F8800109F01AFAB4F8E6
:105FA000820109F016FA94F8840109F0E0F9B4F8D6
:105FB0008601D0E7574C0C2009F008FA94F89001BC
:105FC00009F0D5F9B4F89A0109F003FAB4F896018A
:105FD00009F0FFF9B4F8980109F0FBF994F8910180
:105FE00009F0C5F9B4F89C0109F0F3F9B4F89E0181
:105FF000B1E7484C042009F0E9F994F8D60109F01A
:10600000B6F994F8D70109F0B2F9B4F8D801A2E7CB
:10601000484C494D2078002600EB4000C0B209F002
:10602000D5F9237802359E4280F0C68015F8020C1F
:1060300009F09DF915F8010C013600EB800000EB2A
:10604000800000F2EE2080B209F0C3F9E9E70120F8
:1060500009F0BCF92F4B93F8920109F088F9ABE0F5
:106060002C4B234493F88801013409F080F9082C63
:10607000F6D1A1E0274C102009F0A8F9607909F0C9
:1060800076F9A06809F0AEF994F8900109F06FF97B
:10609000B4F8580109F09DF9B4F85A0109F099F9DA
:1060A000B4F85C0109F095F9B4F8800109F091F9B0
:1060B000B4F882014FE7184B164C93F8C50004F171
:1060C0002005C0EBC000C0B209F080F994F8F401DB
:1060D00000231A4AD25C904274D00C33302BF8D192
:1060E0000834AC42F2D167E0402009F06FF9094C66
:1060F00004F14005B4F8A40209F06BF994F8A60283
:1061000009F035F9043494F8A30209F030F9AC42EF
:10611000F0D151E0541100206410002044190020F7
:106120004C1900204A190020481900204619002067
:10613000E91000200C280020F4120020182800206C
:10614000E02009F043F92B4C04F18005B4F8260255
:10615000043400F03F0009F03CF9B4F82202C0F327
:10616000861009F036F994F82002000909F0FFF8CA
:1061700094F8200200F00F0009F0F9F894F82102D9
:1061800009F0F5F8AC42E1D116E00D2009F01EF956
:10619000002009F0ECF8002009F024F906E0164B85
:1061A000185D013409F0E3F80B2CF8D1002009F058
:1061B00019F9002009F016F90120BDE8F087002048
:1061C000BDE8F08709F0D3F8B4F8F60109F001F959
:1061D00094F8F80109F0CBF894F8F90109F0C7F840
:1061E00094F8FB0109F0C3F894F8FA0109F0BFF83C
:1061F00076E700BF54110020F28801082DE9FF471F
:10620000CC4C07462378CC4E002B00F0018232683C
:106210006368D31A7C2B40F2FB81237A62600133DE
:1062200023724FF0000808F12400C24DC0B20AF0FA
:10623000BFFE05F10A0333F918000BF0BFFCBF4B9A
:10624000814618880BF0BAFC014648460BF0BEFDAB
:10625000BB490BF007FD0BF0CBFE08F1010800B2C3
:106260000AF094FEB8F1030FDDD130200AF0A0FE51
:10627000B5F910000AF08AFE0AF092FE2B7A9A070E
:106280002CD141F288336A689A4218D910200AF05A
:106290008FFE68694FF0640890FBF8F000B20AF0D6
:1062A00075FE21200AF084FE686990FBF8F308FB74
:1062B00013000028B8BF404200B20AF067FE142065
:1062C0000AF076FEB4F918000AF060FE1C200AF00D
:1062D0006FFE00200AF05AFE0AF062FE237ADFF811
:1062E00054825B0740F0718102200AF061FED8F809
:1062F0001C006423323090FBF3F000B20AF046FE3B
:10630000B8F926504FF0050A95FBFAF503200AF07C
:106310004FFE8C4BADB21B78DFF83C9213F0040FAC
:106320000DD008F5D870394601F0EBF928B9D9F845
:10633000003013F0100F18BF002528B205E0D8F880
:1063400000389889B0FBFAF000B20AF01FFED9F8C5
:1063500000309F0740F18780DFF80092B4F80428EE
:1063600099F800304FF0640808FB02325B00B2FB82
:10637000F3F3B4F8067806203F01BFB247EA0327DB
:10638000BFB2C3F303231F430AF012FE38B20AF070
:10639000FDFDB4F8063899F8001001339BB293FB69
:1063A000F1F201FB1233A4F80638D4F80838614D35
:1063B0009B7B012B05D139200AF0FAFDB5F90408C1
:1063C0001AE0B5F804586E235D43152795FBF7F5E1
:1063D0003A20AFB20AF0ECFDB7FBF8F528B208FBA3
:1063E00015750AF0D3FD3B200AF0E2FDA8B2451D69
:1063F0000A2095FBF0F000B20AF0C8FD28200AF050
:10640000D7FDD4F80C380A2093FBF0F000B20AF064
:10641000BDFD04200AF0CCFDD4F80038454F9D891D
:106420004FF6FF73D7F810089842A8BF1846ADB1D1
:106430000028ACBF281A28460BF0C0FB42490BF0DD
:1064400011FC074628460BF0B9FB014638460BF015
:10645000BDFC0BF0CDFD6428A8BF642020EAE070ED
:1064600000B20AF093FDD4F81438324F9D0640F183
:10647000A18097F8183898071DD511200AF098FDCB
:10648000B7F81A084FF4F3656843304B90FBF3F00C
:1064900000B20AF07BFD19200AF08AFDB7F81A084D
:1064A0004543642095FBF0F595FBF0F300FB13509A
:1064B00000B20AF06BFD94F81838B4F81C5813F0C9
:1064C000020F08BF002501200AF072FD28B20AF071
:1064D0005DFD09200AF06CFD00200AF057FD1C4B01
:1064E00094F81E581A88B2F5967F0AD9114B1B7A78
:1064F00003F00F03072B04D842F20F75954228BF13
:10650000154605200AF054FDD4F808385B7B0BB91A
:1065100028B22DE0A5F120000BF050FB0D490BF047
:1065200055FC002105460BF03BFDC8B94FF07C51EE
:1065300018E000BF2C110020582E00200A00002077
:1065400000007A44523000200000C842A0860100BA
:10655000320000206666E63F342E00203000002026
:106560004FF03F4128460BF075FA0BF041FD00B2A9
:106570000AF00CFD94F81828C74B910703D493F840
:106580001F28012A04D1012384F81F38C34818E0CA
:10659000D3F80858C24968680BF064FB0BF028FD7B
:1065A000BF490290A8680BF05DFB0BF021FD039042
:1065B00002A806E0BB4A02AB92E8030083E80300AE
:1065C00018460AF005FD0AF0EBFC237A282B1FD1B0
:1065D000B14B00221A7233684FF47A70B3FBF0F8B3
:1065E0003C2717200AF0E4FCB8FBF7F5B5FBF7F001
:1065F00007FB1050000200B20AF0C8FC18200AF095
:10660000D7FC07FB158000B20AF0C0FC0AF0C8FCFA
:1066100094F82838A04D002B00F0638101F0FEF8BB
:10662000D5F82C38A04AC31A9342074640F2C780D7
:10663000002385F8323885F83438B5F80438DAB2F2
:106640001B0A85F84E2885F84F3885F8442885F8C8
:106650004538D5F85C2833689A1AD5F86038D97B64
:106660004FF47A734B439A420ED3904B1B68C5F894
:106670005C3895F86438013B012B9FBF102385F8E7
:106680003238022385F83438D4F80C280A20D4F89C
:10669000103892FBF0F293FBF0F384F84C281212BE
:1066A00084F84D2884F8503894F818281B1284F880
:1066B000513894F81E389207774984F87F3803D40C
:1066C0002D2381F8803878E0D4F820987848DFF8D6
:1066D000ECC199FBF0FA0CFB0A924FF0060E042B6A
:1066E0000EFB02F28CBF3323322381F88038714BCA
:1066F000D4F8246892FBF3F196FBF0F003FB11222F
:10670000642592FBF5F20CFB006C0EFB0CFE84F88A
:106710007128121284F872289EFBF3F203FB12E335
:1067200093FBF5F30AEB8A0A4FFA81F80AEB8A0A1F
:1067300008EB8A0189B284F86F1800EB8000090A1F
:1067400084F8701800EB800051B201EB800292B225
:1067500084F87428120A84F8752884F87638B4F816
:106760001A281B1284F877382423534393FBF5F53A
:10677000B4F892380A2284F878381B0A84F87938F9
:10678000B4F81C384FEAD979B3FBF2F303F5FA7386
:106790009BB284F87A381B0A84F87B38B4F89438B2
:1067A000F60F84F86C58C5F3072584F86E9884F8C2
:1067B000736884F86D5884F88138C4F82C7894F89C
:1067C0009688354DB8F1000F0DD1D5F89C0807F02B
:1067D000D2F9012807D90228374E00F0608201F073
:1067E00049FE0123B370D4F8A0282B4D002A78D09D
:1067F00095F896683EB140F6B731D5F8A838FB1A3F
:106800008B4219D86DE00123D5F89C0885F896389D
:1068100000F0ECFDD5F8AC38082193F90000022314
:106820008DE8480032464FF4964301F064F885F84D
:10683000B068C5F89C0852E095F8A468CEB9D5F8C0
:106840009C08C5F8A06885F8966800F0CFFDD5F8DB
:10685000AC38082193F9000001238DE84800324646
:106860004FF4964301F047F8C5F89C0801F002FE8A
:1068700035E0013EF6B285F8A46895F8B01895F8B1
:10688000B138EEB94A1C013385F8B02885F8B13823
:10689000D5F89C0821E000BF2C1100204C190020E5
:1068A0008096184BBC6F01083F0D0300582E002046
:1068B0008096980040420F000A000020806967FF20
:1068C00012F8016B01337018314685F8B008D5F81D
:1068D0009C08C5F8A02885F8B13807F04FF9C4F82E
:1068E000A87894F8B238A14DF3B1D5F8B438DBB13B
:1068F000D5F8B838C3B1C5F8BC381B689C4AC5F890
:10690000C038D5F8C4381344187AFEF751FDD5F8CD
:10691000BC38987908F02BFDD5F8C4380133092B21
:1069200088BF0023C5F8C438924D94F8C8282E6853
:106930008E4B002A00F0EE81D3F8CC28002A00F01C
:10694000E98193F8D038013B012B00F2E381D4F8C0
:10695000CC08864F07F00FF9E0B1D7F8CC0807F064
:1069600007F997F8D13880467E2BD5F800900ED1E4
:1069700002231B2887F8D03809D1D7F8CC0807F0B4
:10698000FAF820B90123C7F8D49887F8D83884F8E2
:10699000D188DCE7D7F8D4282B689B1A41F6583207
:1069A00093421ED9032387F8D038B3E1724A32F8F4
:1069B000130010B903464FF403600133B0F5C06F04
:1069C000DBB279D01ED9B0F5006F7FD032D9B0F5E7
:1069D000036F3FD184F8D938D4F81438634F99063F
:1069E0003FD494F8D81894F8D938002900F054818D
:1069F0002A68921B012AD9D984F8D938002384F84F
:106A0000D83887E1B0F5007F43D007D8B0F5807F54
:106A100049D0B0F5887F00F08B80E6E7B0F5806F55
:106A200000F0AE80B0F5826F00F0F380B0F5047F27
:106A3000DBD123E0B0F5E26F00F08B80B0F5E46FBE
:106A400000F08C80B0F5E06FCFD184F8D938B4F97C
:106A50000A1087E0B0F5046F74D0B0F5026FC4D1AE
:106A600003E197F818389A07BBD5B7F81A1824230A
:106A70004B436421123393FBF1F107E184F8D938D9
:106A80003E4B3A4F1B689B07ABD5B7F804380A2139
:106A9000FBE084F8D938394B344F1B681905A0D571
:106AA000D7F80C18F2E084F8D938D4F814382F4FFE
:106AB0005A0796D57969E9E084F8D9382F4B2B4FDE
:106AC0001B681B058DD5D7F81018DFE0D4F8141813
:106AD000264A8F0684F8D93883D592F81818880783
:106AE0007FF57FAFD90711D5D2F82438192283EA70
:106AF000E371A1EBE37101EB5101B1FBF2F1002B6A
:106B0000ACBF41F0004141F040410EE0D2F82038E6
:106B1000192283EAE371A1EBE37101EB5101B1FBAF
:106B2000F2F1002BB8BF41F080414FF400608BE0E0
:106B300084F8D938D4F814380C4F5B077FF551AF7F
:106B40003969A3E084F8D938B4F91830642159437D
:106B50007AE084F8D938B4F90C1003E0B4F90E10D7
:106B600084F8D9382C2391FBF3F16DE02C1100202F
:106B7000BC6F0108582E0020FA8D0108342E002029
:106B800084F8D93894F8DA38644A0133DBB2032B3D
:106B900088BF012382F8DA3842F2107394F8DA18C9
:106BA00059435F4B1B78D80748BF01319A0748BF4C
:106BB00002315F07B4F8DC3848BF0431D80748BF5A
:106BC0000A319A0748BF14311F0648BF2831D8053B
:106BD00048BF28315A0748BF64311F0748BFC83132
:106BE000980548BF01F5C8719A0648BF01F57A714A
:106BF000DF0648BF01F5FA61580648BF01F57A6122
:106C00004FF4806001F002FC444B002283F8D82846
:106C1000E7E6D4F81418DFF8048111F0200784F8AF
:106C2000D93817D098F8182812F0020F14BF4FF473
:106C30007A71002112F0010F14BF4FF4FA630023A0
:106C40000B4494F81E18194401F0E0FB002384F86B
:106C5000D838C6E6334B1B6819067FF5C2AE3946F5
:106C600001F0D4FB88F8D878BBE684F8D938D4F89A
:106C700014382A4F9A067FF5B4AE97F818389B0758
:106C80007FF5AFAEB7F81C386421594301F0BEFB65
:106C9000002387F8D838A4E684F8D9383AE0B378E6
:106CA00023B1C5F8987886F802809CE5D5F8983825
:106CB000FB1AB3F57A6FFFF496AD0123D5F89C0863
:106CC000B37006F055FF0646D5F89C0806F050FF55
:106CD00076067FF488AD8A2802D08E280DD082E512
:106CE000D5F8143898067FF57EAD95F89638002BC8
:106CF0007FF479AD05F6650306E095F89638002B2C
:106D00007FF471AD05F50363C5F8A0382D2385F830
:106D1000A43868E504B0BDE8F08700BF2C1100205E
:106D200052300020342E0020F8B504460E46174697
:106D30000025204620210EF080F90446D0B1013410
:106D400020460EF0DDF9B0F5617F05DB40F6340337
:106D50009842A8BF184601E04FF46170A0F5617039
:106D6000192390FBF3F00DB9307000E070703B78A0
:106D700001333B700DB90125DBE72046F8BD30B586
:106D800005460C46134629462246BDE830400148D8
:106D900002F065BCEC8E01087FB504780646E4B9C4
:106DA000354B1921186800EB840090F87B5090F85F
:106DB00079204D4305F5617590F87A30009590F88B
:106DC0007C00414301F5617101912C482146013459
:106DD00002F045FC142CE3D14BE00EF091F913289E
:106DE000054641DC244B701C1C68202100238DF8D3
:106DF0000F300EF022F91E35064670B101363046CE
:106E00000EF07EF91A289FBF04EB850358709DF899
:106E10000F30013398BF8DF80F30304620210EF02F
:106E20000CF9064670B1013630460EF069F90D28AE
:106E30009FBF04EB850398709DF80F30013398BF16
:106E40008DF80F3004EB85043046E11C0DF10F0284
:106E5000FFF76AFF9DF80F30042B0AD0601C002159
:106E600004220EF0B4F804E0054800211322FFF7D5
:106E700086FF04B070BD00BFA41000200B8F010876
:106E8000208F0108014808F025BB00BF268F0108AC
:106E9000F8B50478064674B9304D2146B5F8C421DA
:106EA000B5F8C6312E48013402F0D9FB042C05F1A7
:106EB0000405F2D1F8BD2B490EF092F8A8B9274B82
:106EC0004FF47A714FF4FA62A3F8C411A3F8C62103
:106ED000A3F8C811A3F8CA21A3F8CC11A3F8CE21B6
:106EE000A3F8D011A3F8D221F8BD30460EF008F96E
:106EF000032805462BD8304620210EF09EF8044684
:106F000030B1013420460EF0FBF80126074600E0C0
:106F10000646204620210EF090F810B9BDE8F84052
:106F2000B0E701300EF0ECF8012EF7D140F2DC535F
:106F3000A7F2EE229A42F1D8A0F2EE229A42EDD8C0
:106F4000064B703503EB85039F80D880F8BD06485B
:106F500000210322BDE8F84011E700BF54110020D2
:106F6000348F0108478F01085B9A01082DE9FF4122
:106F700004780546002C34D16D4808F0ABFA6D4D0D
:106F8000286900210BF002F8002840F0CE8021464D
:106F9000694802F064FB2869694602F0FBF9014682
:106FA000664802F05CFB6869694602F0F3F9014645
:106FB000624802F054FBA869694602F0EBF9014609
:106FC0005E4802F04CFBE869694602F0E3F90134DF
:106FD00001465B4802F043FB0C2C05F11005CFD1B4
:106FE000A3E0584905220EF03FF838B9514B002272
:106FF00003441030C0281A61F8D196E0284652495F
:1070000004220EF031F804462846002C3FD12021FE
:107010000EF013F8002800F08880451C28460EF07A
:107020001AF80746494B53F824601EB9484808F03F
:1070300051FA7AE028463146FAB20EF015F80134DA
:107040000028EFD13B4B0021C2181030C02811613D
:107050009E46F7D13F4B03EBC402D2F804C09846DA
:10706000BCF1000F04D131463B4802F0F8FA53E07E
:10707000002718F834309F42F5DA3B010EEB030588
:10708000103563440FCB013785E80F00F1E70EF0B0
:1070900037F80B28064643DC284620210DF0CDFFAB
:1070A000054648B10135284602F0DEF8214B01249F
:1070B00003EB0613186100E00446284620210DF07A
:1070C000BCFF054640B10135284602F0CDF8194B0A
:1070D000013403EB06135861284620210DF0ADFF63
:1070E000054640B10135284602F0BEF8114B013487
:1070F00003EB06139861284620210DF09EFF10B97E
:10710000FFF7C0FE11E0013002F0AEF8094B032C8E
:1071100003EB0616F061F3D11048FFF727FF04E0F8
:107120000F4801210C22FFF72AFE04B0BDE8F081D0
:107130004D8F010854110020688F01086E8F0108DF
:1071400097970108478F0108728F0108FC86010894
:10715000778F01081C8E0108868F0108DC8C0108DE
:10716000208F0108F0B5047887B0064614BB514B58
:1071700019201968062303FB041191F8CA5091F8ED
:10718000CE20454305F5617591F8C930009591F819
:10719000CB50C831684300F56170019008790290C6
:1071A0004979454803912146013402F058FA0C2CE4
:1071B000DDD17CE00DF0A4FF0B28044672DC3D4BD2
:1071C000701C1D68202100238DF817300DF035FF4D
:1071D000064680B1013630460DF092FF03289FBF6E
:1071E000062303FB045383F8CE009DF817309CBFA1
:1071F00001338DF81730304620210DF01EFF074671
:1072000080B1013738460DF07BFF0D289FBF062364
:1072100003FB045383F8C9009DF817309CBF01336A
:107220008DF8173006266643A9193846CA310DF184
:107230001702FFF779FD20210DF0FFFE074670B120
:10724000013738460DF05CFF14289FBF9DF81730BA
:107250007619013386F8CC0098BF8DF81730384680
:1072600020210DF0EAFE78B101300DF049FF0D2824
:107270009FBF062303FB045383F8CD009DF817300E
:107280009CBF01338DF817309DF81730062B0ED0B8
:10729000062202FB04500021C9300DF098FEFFF7D2
:1072A000F1FD04E0054800210B22FFF768FD07B05F
:1072B000F0BD00BFA4100020928F0108208F0108AC
:1072C0002DE9F347047807464CB9204601A906F09A
:1072D00057F80134FFF7F4FF122CF6D178E00DF0E7
:1072E0000FFFC5B2112D6ED8781C20210DF0A5FE20
:1072F000394C05F1D00614F816800346374F30B9E3
:10730000A8F10202D2F1000848EB020843E000F1C4
:10731000010A597838460DF090FE60B1032D8CBFFC
:1073200003230023C01BC0B23B44184490F80490D0
:10733000B9F1030F02D1FFF7A5FD49E0A9F102035E
:10734000D3F1000850464FF0200148EB03080DF040
:1073500074FED8B1B8F1000FEDD001300DF0D0FEC1
:1073600040F2ED2380B2984205DD40F6CA03984210
:10737000A8BF184601E040F2EE20A0F2EE2019224C
:1073800090FBF2F004EB4603587002E0B8F1000FF6
:10739000D1D104F8169014F81630FA5CB8F1000F49
:1073A0000CD00D4B0E4803EB4606717819234B4366
:1073B000294603F2EE2302F052F909E02946094872
:1073C00002F04DF904E0084800211122FFF7D7FC34
:1073D00002B0BDE8F08700BF54110020D06F010853
:1073E000B28F0108C48F01085B9A01080022084986
:1073F0000C2303FB02135968814204D10022C262AC
:107400001A725A6070470132042AF0D1704700BFE7
:107410001828002010B5084B0022196801EBC203A0
:1074200093F90240844201D1981C10BD0132042A14
:10743000F4D1002010BD00BF14280020F0B5027860
:1074400087B08AB94A4C04F1200694F8F42100234D
:10745000484950B2595681426DD00C33302BF7D188
:107460000834B442F1D180E0002204920592451C18
:107470000DF046FEC4B260B2FFF7CCFF074618B16C
:107480008DF81040012400E00446284620210DF02C
:10749000D4FD054638B1013528460DF031FE0134E2
:1074A000ADF81200E4B20026284620210DF0C5FDFB
:1074B000B0B3451C28460DF023FE00222E495FFA8A
:1074C00082FE51F82230834204D00132082AF5D1DD
:1074D000002300E0734651F82320824220D1022E7F
:1074E0000FD0032E12D05A1E012ED2B204D0042A7D
:1074F00013D88DF814300EE0042A0ED88DF815300C
:1075000009E0052B09D88DF8173004E09A1E052AEA
:1075100003D88DF816300134E4B20136042EC3D1FD
:10752000052C03D807B0BDE8F040ABE404AB03CBB7
:107530003860796019E094F8F9010F4B94F8F8512C
:1075400053F82000B4F8F621009094F8FB0153F8AA
:107550002000019094F8FA0153F8200053F82530E8
:107560000290064802F07BF87AE707B0F0BD00BF52
:107570005411002018280020D8780108D38F010862
:1075800038B1438811EA030003D08B420CBF0120BD
:107590000220704730B50A4B0A491C680A78032A52
:1075A0000AD81346551C04EBC303EAB29D8828424F
:1075B000F5D00A70981C30BD0A70002030BD00BFA5
:1075C000142800200C1A0020014B00221A70E1E759
:1075D0000C1A00202DE9F047877890F803C0BBB261
:1075E000C7F1640E03EB83065C42C3F178001C4DC7
:1075F0005FFA8EFE7600CCF16408A4B280B2A3B22A
:107600000FFA83F9B9F1000F04DC002B14BF3B46DD
:10761000012300E0734609FB09F25B4302FB0CF215
:1076200092FBF3F3434403FB09F30A2293FBF2F3C7
:1076300033449BB225F8023FB1F800904A880A34DF
:10764000C9EB020A1AB202FB0AF24FF47A7392FBF8
:10765000F3F3A4B24B4484422B80D0D1BDE8F08731
:107660000C1A002010B544780078002240F6C411AE
:1076700002FB02F3193B634303F6C4135343434332
:1076800093FBF1F3034921F812300132072AEDD1BF
:1076900010BD00BF261A0020104B043033F9100033
:1076A000B0F5617F05DB40F633039842A8BF18466A
:1076B00001E04FF461700A7819235A4302F28332D1
:1076C000824208DA4A78534303F283338342B4BFD9
:1076D0000020012070470020704700BF2C2F0020A1
:1076E00010B500F1500302788A4203D18478C27841
:1076F000944204D304309842F5D1002010BD0120FB
:1077000010BD0B4B1B6813F4805F0A4BB3F90630B6
:1077100005D0C089421A934207DD084400E0008A80
:107720008342B4BF0020012070470120704700BF92
:10773000342E00202C2F00201FB5084B1B681B0384
:1077400009D58DF80400039101230D2001A98DF8BE
:10775000053000F0B7FA05B05DF804FB342E0020C8
:107760001FB5084B1B681B0309D58DF80400029157
:1077700000230D2001A98DF8053000F0A3FA05B013
:107780005DF804FB342E002038B5064C002584F843
:10779000285009F029FF84F82950E56225866563A1
:1077A00038BD00BF0C1A002010B510B9BDE810405C
:1077B000EAE700230C225A430A4C1119125D824257
:1077C00003D00133102BF5D110BD074B586B18B106
:1077D0004A784078824203D2002259631A86DA62DC
:1077E00010BD00BF187901080C1A002010B5400028
:1077F0001428A8BF14200023074A022199540B44DF
:1078000099181424834201F8014CF5DBFF21D1546F
:107810000F20BDE81040C7E71C2C002010B50A4A15
:107820000A4B11689B6800BF12689142F7D1084A61
:107830004FF47A70946B00FB04F2D31AB3FBF4F3A9
:1078400000FB013010BD00BF582E002010E000E00A
:107850000C1A002038B50446FFF7E0FF0546FFF795
:10786000DDFF401BA042FAD338BD10B504462CB151
:107870004FF47A70FFF7EEFF013CF8E710BD2DE9F9
:10788000F04180460B25013D19D008F10106322751
:1078900005243846FFF7E9FF3846FFF7E6FF3CB11D
:1078A000013CF6D14FF4FA70FFF7DFFFFA27F0E75B
:1078B000013EEED14FF47A70FFF7D7FFE3E7024ABB
:1078C000024BDA60BDE8F0810400FA0500ED00E04B
:1078D000024A136801331360704700BF582E00201E
:1078E000024BDB6B03B11847704700BF0C1A002036
:1078F00003685B6918472DE9F743064689469DF8FA
:10790000288011461A469DF82C3000250C2068432B
:107910001A4FC419C057B04202D1207A20B126E0D4
:107920000135042DF2D122E0012E0AD003DCF6B994
:107930000093134807E01E2E0AD01F2E17D10120F6
:1079400006E010480093434603F0A1FB044605E01F
:1079500005F0B8F941460446FFF7CAFF4CB10C23C5
:1079600003FB0575267185F808906C6001E0002026
:1079700000E0204603B0BDE8F08300BF18280020D7
:10798000003801400044004003681B69184710B5E7
:1079900004462046FFF7F8FF18B90A20FFF765FFF5
:1079A000F7E710BD0368DB68184700BF344B354A62
:1079B0001B68126810B51A60334A11685960516823
:1079C00092689960DA60314A116819615168926869
:1079D00059619A612E4A1168D96151689268196299
:1079E0005A622C4A11881985518859859188D28804
:1079F0009985DA85284A118819865188598692888E
:107A00009A86264A1188D9865188928819871946FC
:107A100021F83A2F224A10780022824206DA214CBD
:107A200034F81240013221F8024FF6E71E4A12885C
:107A3000A3F864201D4A1288A3F866201C4A118806
:107A4000A3F86C1051889288A3F86E10A3F87020E8
:107A5000184A3B2112689A66174A126892FBF1F2A3
:107A6000B2F5967FC8BF4FF0FF325A67134A1288AB
:107A7000A3F87820124A5289A3F85E2010BD00BFF7
:107A8000502C00203830002054210020602100209C
:107A90006C2100204C11002088100020361100209D
:107AA00048290020A81000208C2800201410002055
:107AB0008E1000204011002000000020C81000207F
:107AC000941000202DE9F84305460E460D4B002486
:107AD00093E88003B44213DA7B1933F9140008EBFE
:107AE000050333F9142009EB050333F9143001348D
:107AF0001344022293FBF2F3C01A08F053FAE9E7A9
:107B0000BDE8F883502C002070B5472008F09AF9A2
:107B1000174B1B681B0307D5164B174A5B68106889
:107B20001B68C01A08F02FFA144E154C154D30780A
:107B300008F029FA23682868C01A08F033FA636845
:107B40006868C01A08F02EFA0F4B188808F01BFA64
:107B50000E4B188808F017FA0D4B188808F013FA26
:107B6000337823742B68A3606B68E36070BD00BF3B
:107B7000D42D0020502C0020383000204A1900203D
:107B80003C2C00204C1900204819002046190020E8
:107B9000D01000207FB5264C264E274D2749284A75
:107BA000284B20B128480088B0F5805F31D230885A
:107BB00091F820101278ADF8040028781C4D1B783D
:107BC0008DF806008DF807108DF8082001A82946C9
:107BD00006228DF809300DF0DFF930B30198BDF8B9
:107BE00008302860AB80532008F02CF9208808F07A
:107BF000CAF9A07808F0C7F9E37801A801932379BE
:107C000002936379039308F025F90F4B00221A8041
:107C10000BE0308891F820102080127828781B78AB
:107C2000A070E17022716371DDE704B070BD00BF28
:107C30004C1A0020081A00204419002004300020AB
:107C40008F0E0020F40E0020F42D0020A0F17D0303
:107C5000012B70B504460D460A4E05D830687D21CB
:107C600005F08CFF84F020043068214605F086FF83
:107C700035B12B881C4404EB142404F0FF042C8041
:107C800070BD00BFF81900200A4A13880133138021
:107C9000094A136801331360084A138801339BB201
:107CA000202B01BF00231380054A138808BF01332E
:107CB00013807047F42D0020DC2D0020E02D0020E3
:107CC000E22D002038B53A4B05461B780C46083BA0
:107CD000012B6BD8452008F0B5F8284608F0B2F81B
:107CE0000C2D23D004D80A2D0AD014D835B138BDB4
:107CF0000E2D4BD02ED3FF2D50D038BD206849E03B
:107D0000207808F09FF862796378002A14BF8020F9
:107D10000020184300E0207808F094F8A07808F0DC
:107D200091F8E07808F08EF820793BE0B4F9000093
:107D300008F01FF9A07808F085F8E07808F082F8DC
:107D4000B4F9040008F015F9B4F90600BDE83840AC
:107D500008F00FB9637820788BB180F0800008F0CC
:107D600071F8A468E0B208F06DF8C4F3072008F0D9
:107D700069F8C4F3074008F065F8200E12E008F037
:107D800061F86068BDE8384008F00CB9206808F078
:107D9000FAF86068BDE8384008F0F5B8054808F022
:107DA0002FF80020BDE8384008F04CB838BD00BFBF
:107DB000342C0020F28F01082DE9F04FBE4B8BB020
:107DC0001A880193BD4F002A40F0A98042F20103B6
:107DD000B7F8D207BA4EC21A50425041FFF7DAFE46
:107DE000FFF7E4FD34684920254608F02BF8B54B31
:107DF00004F11C09186808F0C6F855F8040B08F0DF
:107E0000C2F8284605F026FA04F1100005F022FA1F
:107E10004FF01008AC4D01232A6803FA08F313420F
:107E200003D0D9F8000008F0BDF808F10108B8F156
:107E3000130F09F10409EDD104F1280005F0FAF956
:107E4000B7F84031B4F92E00C01A08F09CF82B683E
:107E5000DB0408D59D4BB4F864001B88181AC0F3E6
:107E60000D0008F090F82B68980403D5B4F866006C
:107E700008F089F82B68590503D504F16C0005F06A
:107E8000D9F92B681A0502D5A06E08F08BF82B687B
:107E90005B0402D5606F08F085F82B68180403D5E1
:107EA000B4F8780008F06FF8A04604F1300005F04F
:107EB000C1F904F1360005F0BDF9B7F8403138F9E1
:107EC0003C0F0127C01A08F05EF8814B1B789F42D7
:107ED00008DA38F9020FB4F93C300137C01A08F05B
:107EE00061F8F2E72B68990505D5B4F95E00A0F2B8
:107EF000DC5008F057F8326876487260B260121AA7
:107F00009110754A4A43531C032293FBF2F202EB91
:107F100042029A1A7C2303FB02033360D6E16F4BC3
:107F20006F4A1B6811688B4206D00AA941F8203DB0
:107F300000201360FFF7C6FE019B97F8D2171B883D
:107F400097F8D3070B44013BB3FBF0F200FB12336D
:107F50008B4280F086815A4F0120FFF71BFEFFF70E
:107F600025FD50203E687D6807F06CFFBA683B68CD
:107F700010681B687A680344106806F11C0BA3EBB9
:107F8000400008F00FF86A68736802A89B1A029311
:107F9000AA68B36805F11C089B1A0393EA68F368A2
:107FA00010249B1A049305F055F92A69336902A835
:107FB0009B1A02936A6973699B1A0393B369AA694E
:107FC0009B1A049307F046FF3F4901220B68A24029
:107FD0001A428A4606D0DBF80000D8F80030C01AF2
:107FE00007F0E0FF0134132C0BF1040B08F1040837
:107FF000EAD106F1260005F12601002331F9024FEE
:1080000030F9022F121B02AC44F823200133042B59
:10801000F4D103214FF000094FEA89035FFA83F995
:1080200002AB53F821206AB102F108000F2802D8F0
:1080300049F0010906E08032FF2A94BF49F00209A5
:1080400049F0030911F1FF31E6D24846002407F058
:10805000F9FEA0460DF1080B09F00302022A16D022
:10806000032A1DD0012A4ED1B8F1000F05D1DBF84B
:10807000004090462401E4B245E0DBF800004FF0F8
:10808000000800F00F00204307F0DCFE3BE0B8F1F1
:10809000000F0CD0DBF80000C0F3031020432CE0ED
:1080A000B8F1000F1ED19BF8010007F0CBFE9BF842
:1080B000000007F0C7FE26E0E02D0020541100204C
:1080C000502C0020DC2D0020D42D0020D02D0020AD
:1080D000482900205C2C0020DF7BEFBDE82D00202C
:1080E000E42D0020DBF80000C0F30330204307F04C
:1080F000A9FEDBF80000C0F3071007F0A3FEDBF8D1
:1081000000402401E4B20BF1040B06AB9B454FEA9F
:108110009909A1D1B8F1010F02D1204607F092FED2
:10812000DAF8003013F480541FBFB6F86420B5F8B5
:1081300064100124521A18BF02929A040AD50AAA9E
:1081400002EB8401B5F86600B6F866200134121A15
:1081500041F8202C580513D502AA02EB840C06F135
:108160006A0E05F16A0000223EF9021F30F9028F03
:10817000C8EB01014CF822100132032AF4D1033478
:10818000190508D50AAA02EB8400A96EB26E013463
:10819000521A40F8202C5A0408D50AAA02EB84008F
:1081A000696F726F0134521A40F8202C18040BD5F5
:1081B0000AAB03EB8402B5F87810B6F878300134D6
:1081C0005B1A42F8203C00E0FCB1012C03D102987C
:1081D00007F0E8FE19E0631E002002AA52F82320EF
:1081E0004000C0B20AB140F00100013BF5D507F0F4
:1081F00029FE4FF0000802AB53F8280008B107F041
:10820000D1FE08F10108A045F5DB30200321FFF77E
:1082100059FC36200321FFF755FC2F4B3C201978E1
:10822000FFF750FCDAF80030990506D5B6F95E0084
:10823000B5F95E30C01A07F0B5FE3A6827487B688A
:108240007A60121A9110264ABB604A43531C0322DB
:1082500093FBF2F202EB42029A1A7C2303FB020325
:108260003B60204B1B681A0630D51F4C1F4D2268FF
:108270002B689A420BD162686B689A4207D1019BC6
:108280001B88102B11D11A4B1B885B060DD148207F
:1082900007F0D8FD206807F085FE606807F082FED1
:1082A00023682B6063686B600EE0124A0F4B1178F5
:1082B0002A7C914208D1104A99681068884203D1FB
:1082C0005268DB689A4201D0FFF71EFC07F08AFD76
:1082D0000BB0BDE8F08F00BF482900205C2C0020C7
:1082E000DF7BEFBD342E0020D41000203C2C00207A
:1082F000E22D00204A1900204C1900202DE9F84FEA
:108300000C9EC2EB030B394C0B9B002914BF4FF0A2
:10831000060A4FF0040AF61A6368054601339046D0
:1083200013D1236853455ED2314A032B98BF2946A7
:1083300052F823202F4807F073FD636800220133B1
:1083400063602D4B05469A7113E0002511E02B4A1E
:108350001278954240DA0B9BE3B109FB06F2995C77
:1083600001228A40264909680A4213D16368013311
:108370006360D4F804900A9B1C4F9945E7DB2BD12E
:108380000A2007F05FFD3B6801333B604FF0FF338D
:108390007B6021E0184A917921B12C2007F052FD31
:1083A000013501E00121917109FB0BF3226808EB13
:1083B000030752B958F8030007F022FD97F904109B
:1083C00005444B1CD2D00F4802E03A440E481179C4
:1083D00007F026FD0544C9E7206850452CBF002062
:1083E0000120BDE8F88F0020BDE8F88FEC2D0020BB
:1083F0009C740108FD8F01084C1A002040000020E9
:10840000D42D00200C900108AF97010830B585B03D
:1084100004AC002524F8025D0091ADF80600214669
:108420001020FFF713FC9DF806002146FFF70EFC15
:108430009DF807002146FFF709FC9DF80000214642
:10844000FFF704FC9DF801002146FFF7FFFB9DF8B4
:1084500002002146FFF7FAFB9DF803002146FFF7D3
:10846000F5FB9DF80E002946C043C0B2FFF7EEFBB6
:1084700005B030BD10B5054C206805F07CFB18B187
:10848000206805F075FBF6E710BD00BFC819002095
:1084900010B509F093FB0021044609F09FFD08B1D7
:1084A000204601E004F10040054909F08FFC054930
:1084B00009F0D8FB01F0F4F9034B186010BD00BFC0
:1084C0008096184B35FA8E3C280000202DE9F041AB
:1084D00005460E46078A83899BB21F40002F37D07E
:1084E000B7FA87F24FF00043D340DB4399B21F4005
:1084F000A2F11B032982042BF0D8DFE803F0221F2E
:108500001C190300746A24B1013C0023A4B27362F5
:1085100001E0AC8DA4B2D6F82080B8F1000FDDD018
:10852000D8F80030404621469847D8F80480F4E750
:108530003068A98E08E07068298F05E0B068A98FBF
:1085400002E0F068B5F84010036889B29847C5E7C3
:10855000BDE8F08138B50D4B0D4D99680D4B1A688B
:108560001C465288114203D0FFF758F9286007E0F3
:10857000FFF754F92B68984282BFC01A064B186067
:1085800023685A68054B5A6138BD00BF000C014092
:10859000541A002030020020000000200004014096
:1085A000F8B59C4B05461B68187818B1012800F0F7
:1085B0006781DCE2242D984C0CD006D80A2D00F0FF
:1085C000D8800D2D00F0D58044E12A2D06D02C2D29
:1085D00004D03FE120716071A0714DE18F4B617952
:1085E000277900208C4A58542FBB1978D771472916
:1085F00021D1597850291ED19978472907D1D978A6
:10860000472904D11979412901D10121D1719978E2
:10861000824A522903D1D1784D2900F0AA82997853
:108620007E4A472907D1D178532904D11279562A95
:1086300004BF0322E271E279774E022A38D0032A7E
:108640004BD0012A40F08380BA1E072A7FD8DFE88A
:1086500002F004080F131A257E2A08F09FFBA06081
:1086600075E01B78532B72D1A3685B42A3606EE068
:1086700008F094FBE0606AE01B78572B67D1E36851
:108680005B42E36063E01B78302B654B1A788CBF4C
:1086900042F0020222F002021A7058E0002008F0B4
:1086A000DDFB207453E0002008F0D8FB60824EE030
:1086B000072F06D0082F4AD1012008F0CFFBF08207
:1086C00045E0012008F0CAFB41F2184358434FF43B
:1086D0007A73B0FBF3F0B08239E0022F07D0032F9A
:1086E0000AD1002008F0BAFB4E4B18702FE0002092
:1086F00008F0B4FB30762AE029D93A1F9210337E75
:108700000132D2B2013B02EB8303DBB2102B1ED845
:10871000F91EC2F1010201EB8202D2B2012A0BD092
:10872000042A11D100205E1E08F098FB3E4B002267
:1087300098553E4B9A5507E03D4A5E1E00209355E2
:1087400008F08CFB3B4B9855E3690133E361324BF6
:108750002A2D18BF9A7907F101074FF000000CBFCE
:1087600001225540277160710CBF83F820209D7154
:1087700082E094F82000002847D02F4B13F8012DF9
:108780002E495A708B42F9D1244A234D13785278DE
:10879000402B85BF373B1B011B01DBB298BF03F0A9
:1087A000F003402A8CBF373A303AD2B21344A27950
:1087B000DBB29A4226D121230B70E8796B6A01283B
:1087C00003F101031D4A6B620AD002281CD17223F7
:1087D0001370AA8A1A4B1A80EA8A1A4B1A8013E07D
:1087E000672313700E4B1B789F070ED5164BAA6894
:1087F0001A60EA685A602A7C144B1A706A8A144B11
:108800001A8002E03F230B700020002384F8203000
:1088100032E000BF54020020541A0020602E0020D5
:1088200044190020E810002019110020091100202F
:10883000E9100020F9100020140B0020000B00208C
:1088400046190020D01000204C1900204A190020A1
:1088500048190020637994F820000E2B9FBFA94A85
:10886000591C5171A84A98BFD554A64A18B9937992
:108870005D40957100E00020003018BF0120F8BD78
:10888000A04B002293F82810082900F27081DFE83D
:1088900001F0050C101A2B3B5E788500B52D40F0D9
:1088A000668183F8292001224EE0622D08BF022252
:1088B0004AE0032283F8282083F82A5083F82B50BB
:1088C00083F82C5053E1042283F8282093F82B20BE
:1088D00093F82C102A44D2B283F82B200A4483F850
:1088E0002C2083F82D5042E1052283F8282093F8AC
:1088F0002B2093F82C102A44D2B283F82B200A4460
:1089000083F82C20DD8532E1062283F8282093F8B5
:108910002B2093F82C102A44D2B283F82B200A443F
:1089200083F82C20DA8D02EB0525ADB2B5F5AC7FCE
:1089300082BF744A012182F829100022DD851A863F
:10894000002D40F01481072283F828200FE193F8CE
:108950002B2093F82C102A44D2B283F82B200A44FF
:1089600083F82C201A8EB2F5AC7F3EBF654989187A
:1089700081F834500132D98D92B291421A86E2D9EF
:10898000F5E0082283F8282093F82B30AB4200F062
:10899000EE805C4B012283F829200FE05B4C83F8CA
:1089A000282014F8012D6270594A9442F9D193F8A5
:1089B0002C10544AA94206D03F232370554A5368CD
:1089C00001335360D3E0516A92F8290001315162BA
:1089D00010B13E232370CAE02121217092F82D109E
:1089E000062941D004D8022907D0032923D0F8BD95
:1089F000122959D0302967D0F8BD5021217046493D
:108A0000946B4C60D46B0C60516C4FF47A7491FB96
:108A1000F4F1424C218092F88C11414A19B111783D
:108A200041F0020102E0117821F0020111700122EF
:108A300083F88D218DE05321217092F83910CE07F3
:108A400005D592F83820D51E6A426A4100E00246F8
:108A500002F0010183F88C11002A7AD130490A789A
:108A600022F002020A7074E04F21217092F83F1048
:108A7000CC0705D592F83E20D11E4A424A4100E07B
:108A8000024602F0010183F88C1122B924490A78C8
:108A900022F002020A7093F86310224A1170B3F8B0
:108AA0006010214A118054E056212170946C1F49B6
:108AB0000C8042F21074D16C91FBF4F11C4C2180BB
:108AC000012182F88E1144E04921217092F838107A
:108AD000184A102988BF10211170174914780022F4
:108AE000A24233D20E7A154D56554E7A144D565534
:108AF000CE7A144D565511F80C6F134D5655013260
:108B0000EEE700BF541A0020602E0020140B002056
:108B1000000B0020340200204C19002048190020CE
:108B2000441900204A190020320000204619002074
:108B3000D0100020E8100020881A0020E910002042
:108B4000F91000200911002019110020DA69013202
:108B5000DA6193F88D310B4A93B192F88E317BB183
:108B6000002182F88D1182F88E111846F8BD002080
:108B7000F8BD1279432A7FF452AD0222E2714EE52C
:108B8000F8BD00BF541A00200449054B09680022B3
:108B900018705A6199611A77704700BF582E0020EB
:108BA00034020020F8B5101A0D461F4609F006F8E9
:108BB0000446781B09F002F8174B079E196809F064
:108BC00051F821460546204609F04CF8294607464B
:108BD000284609F047F80146384608F03BFF0CF0FC
:108BE00041FE0E4909F03EF809F028FA069B294695
:108BF000186004F1004000F060FD094909F032F806
:108C0000084908F027FF09F0F3F90028BCBF00F578
:108C10000C40A0303060F8BD280000202C7D8E3F35
:108C2000A00CB34500A00C4644F25063984203DD0B
:108C3000A0F50C40A0387047034B9842BCBF00F52C
:108C40000C40A030704700BFB0B9FFFFF7B5036814
:108C5000174C184D23600B68174E63600068FFF7D0
:108C600017FC95E80300154B0196009394E80C005F
:108C7000FFF798FF3668124B60681E606B68114FF3
:108C8000C01A08F09BFF104B196808F0EBFF09F0C1
:108C9000AFF92A68236878609B1A3B600B4B1E6013
:108CA0000B4B1B68DA880B4B1A8003B0F0BD00BF7A
:108CB000902B00204C1900209C2B0020982B00208A
:108CC000D82B0020A02B002028000020D02B002033
:108CD000640F0020CC2B002070B50446407908F0CA
:108CE00069FF1E4909F072F81D4D1E4E2860E07B99
:108CF00008F060FF194909F069F8EE606860A07932
:108D000008F058FF184909F061F8184D2860207CD8
:108D100008F050FF114909F059F86860A07E08F08A
:108D200049FF134909F052F8EE60A860E07908F0B5
:108D300041FF0D4909F04AF80E4D2860607C08F0AB
:108D400039FF064909F042F86860E07E08F032FF1A
:108D5000074909F03BF8EE60A86070BD0000C8420A
:108D6000A82B00200000FA4400002041B82B00206E
:108D700000007A44DC2B002010B50C4C23789B07B4
:108D800013D50B4B1B78042B0FD90A4A0A4B1068DA
:108D9000526818605A60FFF77BFB084B1A88084B33
:108DA0001A80237843F00103237010BD441900207A
:108DB0004A1900204C190020D41000204411002032
:108DC000EC2B0020164B13B51B681B0325D5154B48
:108DD000154C1B7815498DF80030154B20681B7811
:108DE0008DF8013008F03EFF09F028F911498DF89F
:108DF0000200606808F036FF09F020F98DF80300E2
:108E0000A06809F01BF90C4B8DF804001B780A20B0
:108E100069468DF80530FEF755FF02B010BD00BF62
:108E2000342E0020242E0020482E00200000204157
:108E3000442E002000007A44282E0020054A137892
:108E400083F001031370044A00231360034A136084
:108E5000B8E700BF282E0020402E00203C2E002026
:108E600001480249FFF732BB00080040C429002036
:108E700001480249FFF72ABB000400409C2900205A
:108E80004FF080400149FFF721BB00BF742900204B
:108E900001480249FFF71ABB002C01404C29002071
:108EA00001480249FFF712BB002C01404C29002069
:108EB000254B10B55A43254B254C1B680139B3FB94
:108EC000F2F20388013AA04289B292B29BB212D068
:108ED00004F50064A0420ED0B0F1804F0BD0A4F591
:108EE0009834A04207D004F58064A04203D004F572
:108EF0008064A04202D123F070039BB2154CA042C3
:108F000006D004F58064A0421CBF23F440739BB2DA
:108F100003800F4B8185984202850FD003F50063D3
:108F200098420BD003F54063984207D003F5806365
:108F3000984203D003F58063984201D10023038651
:108F40000123838210BD00BF40420F003C0000207F
:108F5000002C01400010004073B505460068FFF783
:108F6000A7FF2A680124138800269BB243F001035F
:108F70001380EB7A01A88DF804308DF805408DF848
:108F800006608DF8074007F079FDEB7A1B2B0BD1BB
:108F9000192301A88DF804308DF805408DF806607E
:108FA0008DF8074007F06AFD02B070BD0C4B800AD7
:108FB00098420CD004D8B0F5801F0CD10120704726
:108FC000084B984205D04933984206D003E002206E
:108FD000704703207047FE2070470020704700BF95
:108FE00001001000020010002DE9F8430468074654
:108FF000204688469146FFF7D9FF03284BD8BA7A16
:109000009108B8F1000F06D1A589AEB202258D40B6
:1090100026EA0505A5810A2303FB00131F4A42F82F
:109020002380043342F82390B8F1000F07D0BD7AB3
:10903000A189AD080223AB400B439BB2A381282337
:10904000434303F120011144EFF31286502585F3C9
:10905000128803F10C051C331544134455F8047FA2
:1090600017B10F60296804319D42F7D100230B60CE
:10907000F3B283F31188282303FB0020036A23B192
:10908000A3899BB243F0010304E0A38923F0010309
:109090001B041B0CA381BDE8F88300BF4C290020F2
:1090A000FFF758BAFFF756BAFFF754BA014801F074
:1090B0008BBF00BFE41B0020014801F085BF00BF4B
:1090C000381C00200C4B4FF400525A604FF6FE73D0
:1090D0000A48D0F8182211680B401360D0F8082213
:1090E000D0F80C329A4203D000F5F27001F09EBF26
:1090F000012380F82832704700000240541A0020F3
:10910000F0B50124B0FBF4F58D4201D34C43F9E7EF
:109110000026D4B1B0FBF4F504FB1500B4FBF1F468
:109120001EB9002D01DC002CF3D1092D03F1010E35
:10913000EFB204DD002A14BF3725572500E03025A3
:109140003D441D7001367346E3E71C70F0BDF0B579
:109150000124B0FBF4F58D4201D34C43F9E700261E
:10916000D4B1B0FBF4F504FB1500B4FBF1F41EB967
:10917000002D01DC002CF3D1092D03F1010EEFB21B
:1091800004DD002A14BF3725572500E030253D4473
:109190001D7001367346E3E71C70F0BD03685A1C6E
:1091A0000260197070472DE9F843089E002B0746AE
:1091B00088461446334614BF4FF030094FF020095B
:1091C00013F8012B0AB9254603E0002CFBDD013C16
:1091D000F6E7002D04DD38464946C047013DF8E773
:1091E000354624EAE474A01B284415F8011B11B18C
:1091F0003846C047F7E7BDE8F883024B186804F02B
:10920000BDBC00BF20100020F8B507460C464868DA
:10921000002115461E4608F0B9FE58B1284608F050
:10922000CDFC104908F01EFD01464FF07E5008F0BD
:10923000CDFD60606168304608F00CFC01463046A8
:1092400008F0C4FD256806462946384608F000FCAB
:109250000146304608F006FD0146284608F0FAFBB4
:109260002060F8BDDB0FC9402DE9F04102780346CC
:10927000202A00F10100F9D0092AF7D02D2A02D1C5
:109280000346414D04E02B2A08BF03464FF07E55AC
:109290001C460026234614F8012BA2F13007F9B230
:1092A00009290DD83949304608F0DCFC0646384615
:1092B00008F084FC0146304608F0CCFB0646E9E79E
:1092C0002E2A17D1314F234614F8010B3038C2B281
:1092D000092A0FD808F072FC394608F077FD0146DC
:1092E000304608F0B7FB29490646384608F0BAFC74
:1092F0000746E8E71A7802F0DF02452A39D15A78A2
:109300002D2A02D10233012704E02B2A14BF013396
:1093100002330027013B002413F8012F303AD1B269
:10932000092903D80A2101FB0424F5E7B4F59A7F43
:1093300028BF4FF49A74A0464FF07E53B8F1070F40
:1093400007D91846124908F08DFCA8F10808034611
:10935000F4E704F0070434B118460C4908F082FC25
:10936000013C0346F7E719462FB1304608F02EFDC1
:1093700004E04FF07E51304608F074FC0146284668
:1093800008F070FCBDE8F081000080BF00002041C3
:1093900020BCBE4C30B5054687B00C4603A8002162
:1093A0000C220BF014FE2846002108F017FE20B115
:1093B0002846284908F04EFB03E02846254908F0D6
:1093C00047FB254908F04EFC08F012FE054680EAEE
:1093D000E0706946A0EBE57003F0D2FF002DACBF52
:1093E00020232D2368468DF80C300BF034FE012825
:1093F00007D130238DF80D308DF80E308DF80F30F9
:109400000CE0022805D130238DF80D308DF80E3098
:1094100004E0032804BF30238DF80D30694603A80B
:109420000BF0FCFD03A80BF016FE0338C5B22A466C
:1094300003A920460BF03AFE002363552046074956
:109440000BF0ECFD03AB204659190BF0E7FD20466D
:1094500007B030BD6F12033A00007A443090010823
:1094600070B50646B6FBF2F40846154614B1204620
:10947000FFF7F6FF05FB1464024B1B5D00F8013B90
:1094800070BD00BF329001082DE9F04F81468A4639
:1094900016461C4689B000253178002900F0DB8093
:1094A000252902D00136484674E072784FF0000852
:1094B000302A0CBFB278B71CA2F1300312BF4FF0B4
:1094C000000BF71C4FF0010B092B19D8A2F1300348
:1094D000D9B2092905D80A2202FB083817F8012B4E
:1094E000F4E7A2F16103052B02D8A2F1570305E0CE
:1094F000A2F14103052B03D8A2F137030A2BEADDC1
:109500006C2A30D13A787E1C642A00F083800BD814
:10951000252A3DD003D8002A00F09D80BCE7582AB8
:109520000CD0632A19D0B7E7732A22D002D86E2A4A
:1095300037D0B1E7752A5CD0782AADD1271D2068D5
:10954000A2F1580462424FF01001624155E02CD95B
:10955000582A32D0632A2AD13E4648462178271D10
:10956000D04701350FE0642A63D00ED9732A14D195
:109570003E46236848460093514642460023FFF783
:1095800012FE271D05443C4686E7252ADFD13E46CC
:1095900048462521D04701357EE70AD86E2A06D1F4
:1095A0003E46236804341D6076E7002A53D03E46C9
:1095B00072E7752A26D0782AF9D1A2F1580304F16E
:1095C000040C5A422068CDF80CC04FF010015A41EB
:1095D00005ABFFF795FDDDF80CC03E46644605ABD4
:1095E00000934846514642465B46FFF7DCFD054482
:1095F00052E72068271D0A21002205ABFFF7A7FDCF
:109600003C46ECE704F1040CCDF80CC020680A21BC
:109610000022DDE72068271D002808DA2D238DF8B9
:10962000143040420DF115030A210022E6E705AB94
:10963000FAE7206804F1040C00280ADA2D238DF8DB
:10964000143040420DF11503CDF80CC00A21002260
:10965000BFE705ABF8E7284609B0BDE8F08F0FB4C7
:1096600013B50B4904AB08680A4953F8042B096881
:109670000193FFF709FF0446074B1868FEF784F9CA
:109680000028F9D0204602B0BDE8104004B0704771
:109690002C090020280900202010002080EAE07317
:1096A000A3EBE0738B4206DB002801DD401A704714
:1096B00002D008447047002070472DE9F84321F09C
:1096C000004520F00046074688462846314608F007
:1096D00085FC08B9344600E02C462046002108F0FD
:1096E00055FC60B92846314608F05AFC08B93046A6
:1096F00000E02846214608F069FB044600E000240B
:109700002046254908F0AEFA244908F0A1F921467F
:1097100008F0A8FA224908F09BF9214608F0A2FABD
:10972000204908F095F9214608F09CFA1E4908F0F6
:109730008FF91E4900F10049204608F093FA1C49B0
:1097400008F088F9214608F08DFA4FF07E5108F0B4
:1097500081F90146484608F039FB2946044630465F
:1097600008F03CFC20B12146124808F071F904468B
:109770004046002108F014FC20B121460E4808F0B4
:1097800067F904463846002108F00AFC08B104F1E4
:1097900000442046BDE8F88339094E3DE3B59E3EBE
:1097A00088FA163E45FE7F3FA7DFA83499FB243F89
:1097B00069A2163EDB0FC93FDB0F494070B5044676
:1097C00008F016FC2030402857D820462C4908F0D5
:1097D00005FC28B120462B4908F03AF90446F4E785
:1097E0002046294908F0DCFB28B12046254908F02D
:1097F00031F90446F4E72046244908F0EFFB30B184
:109800002249204608F024F9014620480AE0204673
:109810001F4908F0C5FB40B11C49204608F01AF961
:1098200001461B4808F014F904462146204608F07A
:1098300019FA05462046294608F014FA0021064682
:10984000284608F00FFA134908F002F901462846A5
:1098500008F008FA104908F0FDF80146284608F01B
:1098600001FA0E4908F0F4F80146304608F0FAF91A
:109870000146204608F0EEF870BD002070BD00BF24
:10988000DB0F4940DB0FC940DB0F49C0DB0FC93F8D
:10989000DB0FC9BF92E741399730083C15A82A3E33
:1098A00008B5034908F0D6F8BDE8084086E700BFD0
:1098B000DB0FC93F064B10B51A881C4622EA000090
:1098C0009042188002D00120FDF790FF208810BD43
:1098D000081A0020064B10B51A881C461043904207
:1098E000188002D00120FDF781FF208810BD00BF45
:1098F000081A0020024A936823EA0000906070472B
:109900005411002008B5104B1A780023D9B29142A7
:1099100007D20E49002051F823100133096808804E
:10992000F4E73220FDF7A1FF094B1B685A0309D564
:10993000084B9B685B0305D4BDE8084040F2DC504F
:10994000FDF793BF08BD00BF48290020182900205B
:10995000342E0020541100202DE9F34107F022FE9F
:109960004B4A6C2313704FF4FB635380BE23137177
:10997000EF2382F8D53700231946164682F8D637EA
:10998000F25C0133B3F5FB6F81EA0201F8D1404B81
:10999000404A83F8D617404B04275A6002F18832B8
:1099A0005A600020013F17F0FF075ED03A4B342287
:1099B0003A4CDA6004F17848A8F5FC38C8F309039A
:1099C00053B100234FF4005056F80880019303F080
:1099D00049FE0428E6D11CE04FF4302003F042FE9B
:1099E0000428DFD12C4D4FF430202B6943F00203C3
:1099F0002B616C612B6943F040032B6103F032FE55
:109A000041F6FD732A69042803EA02032B61D8D0CA
:109A1000C8E7214D4FF400502B6943F001032B613F
:109A20001FFA88F3238003F01DFE042813D1A31C22
:109A30000193019B4FEA1848A3F800804FF40050AF
:109A400003F010FE41F6FE732A69042803EA0203BC
:109A50002B6106D0A6E741F6FE732A6913402B61FD
:109A6000A0E70F4B04349C42A4D10B4A042813698D
:109A700043F08003136102D105F036FF10B90520D1
:109A8000FDF7FDFE07F078FD02B0BDE8F08100BFF4
:109A900054110020230167450020024000F801080E
:109AA000D8FF010810B50E4C2068FDF7DBFD2068DB
:109AB0000022047A02FB02F3193B634303F6C4134A
:109AC0005343192193FBF1F3064921F81230013277
:109AD000072AEFD1BDE810400349FDF77BBD00BF69
:109AE000CC100020F00F0020941200202DE9F0414E
:109AF00005F0FAFE10B90420FDF7C1FEBF4C07F0D7
:109B000051FDBF494FF4FB6220460BF055FA94F823
:109B1000AC374FF4CC71022B84BF002384F8AC37F0
:109B200094F8AC27B74D01FB02F3E01800F539704B
:109B30002344286093F8380301FB0242022803F50E
:109B40004C7384BF0020187292F83833AE4A1370F9
:109B50000C2202FB0343AD4A03F2AE73136046F2DC
:109B60000902A3681A401AB9A44A43F40053936047
:109B7000A368DE0703D54FF40050FFF7BBFEA368D0
:109B8000580409D50820FFF7B5FE4FF40050FFF741
:109B9000B1FE0120FFF7AEFEA368190706D54FF40A
:109BA0000050FFF7A7FE0120FFF7A4FEA3689A0468
:109BB00013D54FF40040FFF79DFE904B93F884318E
:109BC000012B03D14FF40060FFF794FE4FF4803077
:109BD000FFF790FE4020FFF78DFEA3685B0603D5DC
:109BE0004FF48030FFF786FE894B1B6803F4206337
:109BF000B3F5206F07D194F88431012B03D14FF4D2
:109C00000060FFF777FE94F8DE217C4B2AB193F8D1
:109C1000E22112B1002283F8E2214FF0000C6746E6
:109C20007C4E7D4B1E6004EB0C03B3F8F6E14FEA6B
:109C30005E0101F077314FEA9E0303F03333C1EB4D
:109C40000E00C11A4FEADE0303F01133CB1A03EB07
:109C5000231303F00F32FF2392FBF3F31EF00108EE
:109C6000C3EB032318BF0137A2EB030318BFFFB2F6
:109C7000012B0ADD022B40F0BE80B8F1000F00F08E
:109C8000BA801EF0BC0F00F0B6800CF1080CBCF1DD
:109C9000200FC8D1013F012F00F2AD80FFF702FF76
:109CA000302200215D480BF092F95D4F5D4BD5F8F5
:109CB00000801F605C4B002108F17900C3F8008030
:109CC000FDF70EFD594B80F001001870584B07F15D
:109CD00028021A60574B07F1D4021A6098F8000066
:109CE00002F032FD2868544B00F5C5721A60FEF789
:109CF000F3FF524B94F8D61107F196021A606422D2
:109D00004A434F4BC8325A6000229A60DA601A61A7
:109D10005A619A61DA6183F8202083F82120494B47
:109D20002D6807F12E021A60474B05F219121A60CE
:109D3000464B05F289121A60454B07F108021A607A
:109D4000444BDFF844811F60434B07F1A2021A60C5
:109D500007F1AC03C8F80030404BB4F864011E6052
:109D600007F028FFC8F80800B4F8660107F022FFE2
:109D700095F85C3008F1040288F8043095F87830E2
:109D8000C8F80C0088F8053094F8E131286E88F89E
:109D90001030334BC8F814501A6005F16403C8F84A
:109DA0001830304907F05EFF01464FF07C5008F054
:109DB0000DF8B5F81641C8F81C00204607F0FEFE65
:109DC0000146294808F002F8284907F04BFF284AC5
:109DD000284B1560284A186005F168031360274A6C
:109DE00005F211151560264A1760264ABDE8F041B4
:109DF000136007F0C1BB03F07BFA4FE7541100205A
:109E000000F80108A4100020F02B0020CC10002046
:109E1000342E0020DC120020F82F0020200F00201C
:109E200094120020540F0020580F00200900002039
:109E30005C020020400E0020640F0020202E002035
:109E400004300020842A0020EC1C0020580400204C
:109E5000EC290020F02900206C03002030040020B1
:109E6000FC2A0020DB0F4940000061444C3D0F44B8
:109E700028020020680300201C0200205803002054
:109E800060030020180100208C1C002008B5FFF79B
:109E900063FDFFF72BFEBDE808400120FDF7A6BCDF
:109EA00038B500240B4D6059254405F013FB696853
:109EB00011B10948FFF7D3FBA96811B10748FFF7B3
:109EC000CEFB0748103405F005FBB4F5D87FE9D187
:109ED00038BD00BFB4740108579001085D900108B7
:109EE00055980108F0B585B004460BF0B4F8082881
:109EF00026D1621EE01D1F4912F8013F096819446E
:109F0000497801F00301022908BF203B8242137007
:109F1000F1D1254604F1080715F8016B16483146C2
:109F20000BF08BF820B1284631460BF086F810B1C3
:109F3000FCF7A8FF1CE0BD42EED1204603F002FA78
:109F40000E4805F0C7FA00230D4A04A91A4492F8F6
:109F500088210A440849595C0133082B02F80C1C7B
:109F6000F2D10023074801A98DF80C30FFF777FBE9
:109F700005B0F0BD44000020FD9601086390010883
:109F8000541100209797010808B5184B184C1D680C
:109F90002068FDF7FCFC2846FDF7F9FC20684179B4
:109FA0008B0703D441F00201FDF7A2FC206803F007
:109FB000E2FD68B10E4B186803F0DAFD0646FEF7C5
:109FC000EFFA08B104F01CFD2846314603F0D6FD37
:109FD000284603F0D0FD0028E8D02846266803F084
:109FE000C7FD0146304603F0C9FDDFE70C2C002019
:109FF000AC1C00202DE9F04705460BF02CF82F4E45
:10A000000446D6F8088090B92D4805F063FA2D4B28
:10A0100053F8241049B10123A34013EA080F02D0DA
:10A020002948FFF71CFB0134F1E7284822E02846C5
:10A03000274922460BF018F858B9264805F04AFA85
:10A04000254C54F8041F0029EFD01F48FFF707FBE9
:10A05000F7E72B784FF000092D2B03BF013504F1F2
:10A06000FF344FF0010A4FF0000A164B53F82970E5
:10A0700027B91A48BDE8F04705F02CBA28463946FA
:10A0800022460AF0F1FFA8B9012000FA09F0BAF15E
:10A09000000F03D0FFF72EFC114803E040EA080050
:10A0A000B060104805F016FA3946BDE8F0470E4892
:10A0B000FFF7D5BA09F10109D7E700BF5411002015
:10A0C00069900108647601087390010855980108A9
:10A0D000779001087C90010860760108778F01086D
:10A0E00088900108919001089697010810B50848DA
:10A0F00005F0F0F9074B00241C715C63064B1C70E3
:10A1000003F0E4FE05F0BEFB044B1C6010BD00BF75
:10A1100099900108AC1C0020533000200C2C00202A
:10A1200070B5064600240B4BE518AA8816420AD0E3
:10A13000E1580948FFF793FA2846002105F05BF93A
:10A14000064805F0C7F940F6444314349C42EAD16E
:10A1500070BD00BFB87A0108C59001085598010884
:10A16000F0B504788BB005460CB1002436E04B4BBB
:10A1700019680E2303FB0411B1F91D51B1F919211E
:10A18000B1F91B31009591F8205101F58C700195C2
:10A1900091F8215101F59071029590F90700039013
:10A1A00091F902103E48049121460134FFF757FA15
:10A1B000082CDCD170E02D2B14D1072C1BDC284699
:10A1C0000AF09EFF0AAB661C03EB440424F8100C53
:10A1D00015F8013F303B092BFAD934462B78002B78
:10A1E000E9D104E0A3F13002092A09D8E5E7082CF7
:10A1F000BDF8182009D00BB0BDE8F040FCF742BE16
:10A20000202BF8D101352646E7E7072AF3D840F29C
:10A21000DC55BDF81A00214BA0F2EE2189B2A9420B
:10A220001B68E8D8BDF81C10A1F2EE24A4B2AC4221
:10A23000E1D8BDF81E6004B237B2A742DBDB0DB235
:10A24000AF42D8DCA542D6DBBDF8247007F1640428
:10A25000A4B2C82CCFD8BDF826E00FFA8EF4112C8A
:10A26000C9DCBDF82050B42DC5D8BDF82240B42CAF
:10A27000C1D812B24FF00E0C0CFB0233A3F8190137
:10A28000A3F81B11A3F81D6183F8205183F8214125
:10A2900083F81F7183F822E10BB0F0BDA4100020F9
:10A2A000CF900108F0B504468FB020460AF0D3FEE7
:10A2B000C5B21DBBAE4805F00DF9AE4C94F8D210F6
:10A2C00009B9AD4853E049B294F8D02094F8D130A0
:10A2D000009194F8D310A948019194F9D41007344F
:10A2E000029194F9CE10039194F8CF10049129466D
:10A2F0000135FFF7B4F9102DE0D1E2E72046A0497F
:10A3000005220AF0B1FE0546B8B929469D487022DB
:10A310000AF05DFE28469C4B19680E2303FB0013D0
:10A3200001300022082883F8232183F8242183F8B0
:10A33000252183F82621F0D118E1204693490422F3
:10A340000AF092FE05462046002D4AD120210AF04F
:10A3500074FE002800F00A81461C30460AF07BFE9D
:10A360002C4607468A4B53F824502DB989480FB024
:10A37000BDE8F040FFF773B930462946FAB20AF05B
:10A3800073FE01340028EDD17A4A164602F17001BD
:10A39000002382F8D63082F8D23082F8D13082F8A9
:10A3A000D03007328A42F3D17B4901EBC40191F8E6
:10A3B0000822934210DAD1F80C72C3EBC302B01832
:10A3C0003A44176800F1D001C0F8D070908801338A
:10A3D000888092798A71E7E729467048FFF73FF94C
:10A3E00095E06F4907220AF03FFE05462046002D02
:10A3F00049D120210AF021FE06460AF02CFEC4B203
:10A400006CBB6848FFF72BF9214667480134FFF71A
:10A4100026F90E2CF8D15848FFF721F9002463489B
:10A420002146FFF71CF90025574A012311680E2227
:10A4300002FB0412D2F82321AB4013425C4B5D496E
:10A440005D4808BF19460135FFF709F90E2DEBD11C
:10A4500049480134FFF703F9082CE0D186E0304683
:10A4600056490AF051FE2C46002852D0022C55D0F5
:10A470000AF046FE06AB43F82400504900200AF0DB
:10A4800043FE0134F0E74D490AF03EFE002460B17E
:10A49000082C3ED00AF034FE06AB43F824004749AE
:10A4A00000200AF031FE0134F1E7082C31D1069B7F
:10A4B0000F2B2ED8DDF81CE0BEF1070F29D8089F1E
:10A4C0000D2F26D8099E06F16402C82A21D80A9DBC
:10A4D000FF2D1ED80B9864281BD80C99642918D816
:10A4E000884216DA0D9C032C13D8224AC3EBC3030F
:10A4F000134483F8D0E083F8D17083F8D26083F8F6
:10A50000D35083F8D40083F8D51083F8D6402C4C70
:10A51000CBE60FB0BDE8F040FCF7B4BC069B072BC0
:10A5200020D807990D291DD80278722A0DD06E2ADD
:10A5300018D1154A0E20126800FB032301228A401D
:10A54000D3F8231121EA020209E00F4A0E20126813
:10A5500000FB032301228A40D3F823110A43C3F8E6
:10A56000232101E0FCF78EFC0D4C9EE60FB0F0BD00
:10A57000F790010854110020559801082291010814
:10A58000478F010824120020A4100020728F0108B8
:10A59000FC860108778F0108B4740108868F0108D2
:10A5A000EF900108619001083E910108AF97010802
:10A5B000489C01088E9B01084391010847910108BE
:10A5C000DC8C01082DE9F743047805468CB9324D3F
:10A5D00095F8A712B5F8A42295F8A6322F48009155
:10A5E00021460134FFF73BF8102C05F10405EFD1AB
:10A5F0004EE00AF085FD0F28044636DC284620216F
:10A600000AF01BFD264EE4B2D6F83880451CA400A3
:10A61000002728460AF074FD5FFA87F9B9F1010FA7
:10A6200083B208D0B9F1020F0BD0B3F5B47F24D2B6
:10A63000B26B13530AE0FF2B1FD8B36B23449870FF
:10A6400004E0FF2B19D8B36B2344D87028462C2183
:10A650000AF0F3FC054608B1013502E0B9F1020F3A
:10A660000BD10137032FD4D112E00E4800210F2265
:10A6700003B0BDE8F043FCF782BB08EB0400002107
:10A6800004220AF0A4FC03B0BDE8F043FCF7FABBD7
:10A6900003B0BDE8F08300BF5411002049910108C8
:10A6A000AC1C0020208F01082DE9F04304788FB006
:10A6B0000546002C59D17C4B0021142209A807AE75
:10A6C000D3F83C800AF083FC0722304600210AF0D0
:10A6D0007EFC00231A46A70005A8059308EB070592
:10A6E00083807249B5F802E031F813C01CEA0E0FFE
:10A6F0000AD00E310DF1380C595C02F1010E6244A2
:10A7000002F81C1C5FFA8EF20133072BE9D10021FD
:10A710000B46674AB5F802E011F802C01CEA0E0FBA
:10A720000AD006320DF1380C8A5C03F1010E634445
:10A7300003F8242C5FFA8EF301310629E9D118F8C9
:10A7400007308DE841006A785A49029209A81A092F
:10A7500003F00F0306F0A8FB2146574809AA01346D
:10A76000FEF77DFF202CA6D19BE00AF0C9FC1F2834
:10A77000044600F3898028462021E4B20AF05DFCFB
:10A780001F2C02D9FCF77EFB8BE0474B451CDB6B93
:10A79000002103EB8404204604220AF018FC002761
:10A7A000464B09AE304600210A2217F803905FFAA3
:10A7B00087F80AF00CFC002315F8012B32B10A2BA4
:10A7C00004D04A4502D0F2540133F5E74A4561D13D
:10A7D00008F1FF33032B09D8DFE803F0100502422C
:10A7E0000DF1230037E00DF123011FE030460AF0A0
:10A7F00087FC2378C0B243EA001006E030460AF036
:10A800007FFC237800F00F001843207034E0013300
:10A81000062B0BD02A4800F2F3269E5D9642F6D115
:10A82000034493F8ED2263881343638011F8012FEA
:10A8300012B30023EEE70133072B0CD0204A02F2BB
:10A84000E6269E5D8E42F6D102EB4303B3F8D82292
:10A8500063881343638010F8011F69B10023EDE79B
:10A8600030460AF04DFC0F2804DC30460AF048FC64
:10A87000607001E0002363700137052F90D101243F
:10A8800004F064F86CB97DE70E4800211F22FCF744
:10A8900076FA06E02046002104220AF098FB002404
:10A8A000EEE70FB0BDE8F083AC1C00208C77010808
:10A8B000A17701085D9101086C910108AD7701084D
:10A8C000B4740108208F01082DE9F04FAB498BB01B
:10A8D00004460AF085FBAA49002820460CBF012542
:10A8E00007250AF07DFBA7490028204608BF02255E
:10A8F0000AF076FB002808BF0425E90740F1E6804E
:10A90000A14804F0E7FD002004F0F4FB9F4CA048B0
:10A9100004F0E0FD9F4804F0DDFD63799E4A013BB1
:10A9200052F823109D48FEF79AFE9D48FEF797FEC9
:10A9300026460027D6F810800021404607F026FB67
:10A9400020B19848FEF78BFE002669E0394696480C
:10A95000D6F814B0D6F818A0D6F81C90FEF77FFEF3
:10A960004046002107F01CFB10B1202004F0AAFD96
:10A9700006A94046FEF70EFD01468C48FEF76FFE25
:10A980005846002107F00CFB10B1202004F09AFD7E
:10A9900006A95846FEF7FEFC01468448FEF75FFE16
:10A9A0005046002107F0FCFA10B1202004F08AFD87
:10A9B00006A95046FEF7EEFC01467C48FEF74FFE26
:10A9C0004846002107F0ECFA10B1202004F07AFD8F
:10A9D00006A94846FEF7DEFC013701467448FEF73B
:10A9E0003EFE0C2F06F11006A4D1AAE749B294F856
:10A9F000D02094F8D130009194F8D3106D48019193
:10AA000094F9D4100734029194F9CE10039194F87C
:10AA1000CF10049131460136FEF721FE102E03D0EF
:10AA200094F8D2100029E1D1634804F053FD574B4C
:10AA3000624C9F6854F8041F19B16148FEF70FFE7D
:10AA4000F8E70E465F4B53F826404CB10123B34064
:10AA50003B4203D05C482146FEF701FE0136F1E798
:10AA60005A4804F037FD2146484B0AAA0B4493F894
:10AA700088311344564A8A5C0131082903F8102CA6
:10AA8000F2D1002306A953488DF82030FEF7E7FDE8
:10AA9000514804F01FFD5148FCF7D0FC504804F029
:10AAA00019FD4E48FFF700FE4E4804F013FD4B48D9
:10AAB000FFF788FD4C48FEF7D2FD4020FFF730FB42
:10AAC0004A4804F007FD4548FCF7FAFBAA0739D5C8
:10AAD000474804F0FFFC474804F0FCFC3F4804F002
:10AAE00049FB454804F0F6FC3C48FCF755F943485F
:10AAF00004F0F0FC3948FCF735FB4148FEF7AFFDA8
:10AB00003648FCF7C5F93F4804F0E4FC3348FFF74A
:10AB100027FB00260E27774300243B4A0123126CB3
:10AB2000A3403A44D2F80A2013421ED101340E2C1D
:10AB3000F3D10136082EEDD12B48FEF790FD802091
:10AB4000FFF7EEFA6B0716D5304804F0C3FC304827
:10AB500004F0C0FC214804F0E7FA2348FEF77FFD2B
:10AB60004FF48070FFF7DCFA05E0314622462948B1
:10AB7000FEF775FDDAE70BB0BDE8F08F78910108BC
:10AB8000889501087F9101088591010854110020E2
:10AB900093910108A5910108FC860108B191010873
:10ABA000BC910108C9910108D69101086090010883
:10ABB00097970108EE910108DE910108607601087F
:10ABC0000D920108647601081B9201082892010881
:10ABD000FD960108349201083D920108DC8C0108C1
:10ABE0004C92010858920108559801086692010894
:10ABF0007392010886920108949201089E920108BE
:10AC0000AD920108BB920108AC1C0020C79201085C
:10AC1000D8920108EA920108026B0346C16810B598
:10AC2000406942B11A6C8C1A013A08BF0A46005DAD
:10AC30001A64C0B210BD1A6A805C01328A4228BF11
:10AC40000022C0B21A6210BD436B13B190F84400E9
:10AC50007047836A406A1B1A584258417047036B19
:10AC600013B15B68016C01E0C369016A8B423CBFB0
:10AC7000C2689B18581AC0B27047426A806A131A99
:10AC80005842584170474171704743799B070AD534
:10AC9000436A8269D154436A01690133B3FBF1F21B
:10ACA00001FB123343627047437913F001031FBF66
:10ACB000C36803F1FF32C369006A1DBF181A104050
:10ACC000C0B218467047437910B513F0010304462B
:10ACD0000DD0FFF7E9FF58B1236A6269E168D05CE3
:10ACE0000133B3FBF1F201FB1233236210BD1846AE
:10ACF00010BDF0B5046D8279A389467923F4005321
:10AD000012F0020F4FEA03434FEA13430CBF002136
:10AD10004FF4005112F0040FA38114BF4FF4806E62
:10AD20004FF0000E16F0010F8768054614BF04208F
:10AD30000020B307238A48BF40F008029BB223F4E7
:10AD4000405343EA01032382A18948BF90B289B2EC
:10AD500021F4B05121F00C014EEA010140EA010258
:10AD6000A281A38A87B023F440731B041B0CA38227
:10AD700001A802F027FC049E039B204A944218BFBE
:10AD80001E46A389192272431BB2002BB4BF7E005A
:10AD9000BE00B2FBF6F66427B6FBF7F0000101092E
:10ADA00007FB1163A28912B2002AADBF1A01D900B4
:10ADB00032313232ABBFB2FBF7F3B1FBF7F203F043
:10ADC0000F0302F00702B4BF104318432A6DAB799A
:10ADD00080B2208113F0080F938A0BBF23F0080381
:10ADE0009BB21B0443F0080308BF1B0C938293899A
:10ADF0009BB243F40053938107B0F0BD003801408B
:10AE0000417176E7816074E703460A4690F846028E
:10AE1000D96A9B7901F056BF38B5A0F513746379F0
:10AE2000A579DB0746D594F8383205F00105F3B172
:10AE3000226B1068838DC3F34E03838494F83C32F5
:10AE400023B1B4F842320133A4F84232917A6A0055
:10AE500001F097FD012384F83B32002384F8393256
:10AE600084F83A3284F83832A4F8403238BD94F885
:10AE70003B322046012B04BF94F8393284F83A3231
:10AE800001F06AFD94F83B22236B3AB9012284F861
:10AE90003B221868997A05FA02F207E0002284F84A
:10AEA0003B2295421868997A08BF0222BDE83840D3
:10AEB00001F067BD38BD10B5A0F5127494F83C22BE
:10AEC000BAB9A36A616A994228D0591CA069A162E3
:10AED000C35C2069DBB25B0043F400738142A4F8D9
:10AEE0003E324FF00A0384F83D3228BFA2620123AC
:10AEF00012E094F93D327BB1B4F83E1220464B0883
:10AF0000A4F83E3201F0010101F04EFD94F83D320B
:10AF1000013B84F83D3201E084F83C3294F8383249
:10AF2000002B50D194F839320133DBB2092B84F86D
:10AF3000393204D12046BDE8104001F00DBD0A2B86
:10AF400041D194F83B322BB9B4F8403243F00103BD
:10AF5000A4F840326379D9071CD5B4F840028205C1
:10AF600001D4C30705D4B4F844320133A4F8443201
:10AF700010E0E36AC0F347000BB198470AE0E369C9
:10AF80006269D054E369E1680133B3FBF1F201FB7C
:10AF90001233E361012284F8382294F83B22002323
:10AFA000012A84F839320ED1A27984F83B32236B1E
:10AFB00012F0010F1868997A0CBF02220022BDE836
:10AFC000104001F0DEBC10BD026D70B5158804465E
:10AFD000ADB2A90613D5036B8BB9C36A1BB19088B8
:10AFE00080B298470BE0E169928840694E1CD2B26A
:10AFF000E6614254E169E268914228BFE3612B06B1
:10B0000013D5636AA26A9A42236D0AD0511CA069C3
:10B01000A162825C9A802369994206D30023A362CD
:10B0200070BDDA6822F08002DA6070BD836A8169DF
:10B03000426B1944D160416A994297BF0169CB1AAA
:10B04000CB1A536096BF0023536083624FF0000316
:10B0500080F84430136888BF816243F001031360B5
:10B060007047436A8269D154436A0269013393424B
:10B0700028BF00234362436B1BB11B68DB0705D469
:10B08000D4E7026DD36843F08003D36070472DE9A5
:10B09000F0431E46944B8DB09842894690469DF8E9
:10B0A000507051D1914B924A92491A60924AC3F81A
:10B0B00008805A6102F580729A614FF48072DA60FA
:10B0C0001A618E4A18651A63A2F54842543ADA6446
:10B0D0009A6459638A4B9A6942F480429A615A6928
:10B0E00042F001025A6102238DF803303A074FF40F
:10B0F0000073ADF8003001D51C230FE0B30706D56F
:10B100001823804869468DF8023001F0A9FDF50743
:10B110000AD54FF48063ADF800304823794869467A
:10B120008DF8023001F09CFD0E238DF804300022D2
:10B13000012301A88DF805308DF806208DF8073021
:10B140006A4C05F09BFC4EE06F4B984240F0C78084
:10B150006E4B674AC3F808801A604FF48072DA6059
:10B160001A616B4A18655A6102F580729A61694AE0
:10B170003C079A64DA64624BDA6942F40032DA61BD
:10B180005A6942F001025A614FF002038DF8033010
:10B190004FF00403ADF8003001D51C230EE0B007DA
:10B1A00006D51823574869468DF8023001F058FD3E
:10B1B000F10709D50823ADF8003048235148694606
:10B1C0008DF8023001F04CFD26238DF8043000226A
:10B1D000012301A88DF805308DF806208DF8073081
:10B1E00005F04CFC494C0025012384F844302562CD
:10B1F000E561A5626562C4F82C906671C4F80880A8
:10B20000A7712046FFF775FDF20731D5206B0028A6
:10B2100026D0E36C039501934FF480530A93802367
:10B220000693E368059504932023099363690795C2
:10B23000029308950B9502F04DF901A9206B02F0DD
:10B240002BF9226B216D136843F0010313608B8A85
:10B250009BB243F040038B8253689BB2236407E0A8
:10B260004FF6DF72236D1A80DA6842F02002DA604E
:10B27000B3072CD5606B28B3A36C002501934FF462
:10B2800080530A9380230693236902950493102325
:10B29000039305950795089509950B9502F01AF902
:10B2A000606B01A902F0F8F8636B1A6842F00202C1
:10B2B0001A60226D5D605D60938A9BB243F08003EB
:10B2C000938204E0226DD36843F08003D360226D43
:10B2D000204693899BB243F40053938100E0002001
:10B2E0000DB0BDE8F08300BF00380140381C0020DD
:10B2F0007078010844000240F01C00205800024011
:10B30000001002400008014000440040E41B0020FF
:10B31000F01E0020044400402DE9F74FFCF77EFAB0
:10B32000A64C804626686568A768861BF643451BC1
:10B33000C71BED43FF43F60FED0FFF0F2EB93FB9CB
:10B34000002D00F08782B9462CE04FF0000929E07B
:10B35000B14627E003EB8A0BBBF802301A050ED486
:10B3600013F4805F1DBF964A9BF801101268954A3E
:10B37000954B14BF52F82120126843F82A20BBF8DD
:10B380000230D80516D499050AD5904B1B7813F0D6
:10B39000040F0CBF8E4A8F4A8B4B126843F82A2049
:10B3A00009F10109207B5FFA89FA8B4982450B6814
:10B3B000D0D326E0894A5046594603F057FA884BC5
:10B3C0001B885A0603D550465946864A16E0580748
:10B3D00003D550465946844A10E0190703D5504614
:10B3E0005946824A0AE09A0703D550465946804A90
:10B3F00004E0DB07D4D5504659467E4A03F036FABE
:10B40000CEE7DFF808E20093BEF906307822A3F514
:10B410007A7353434FF47A7293FBF2F3F34603F2D9
:10B420002B13019300225FFA82FE864517D2009B00
:10B4300003EB820EBEF802E01EF4806F0DD040F2E6
:10B44000671ADFF88491019B39F822E09E449EFB45
:10B45000FAFC0AFB1CEE29F822E00132E3E74DB3C7
:10B4600008F5C333A0336360637B544A13BB937303
:10B47000614B1B6813F0020F0AD0DFF894E19EF8CD
:10B4800000E0BEF1000F03D04FF0010E82F80EE095
:10B49000DA0506D5594BDB781BB1A37B43F00203D9
:10B4A000A3734A4B1B7813F0050F02BFA37B43F035
:10B4B0000403A37394F80EE0BEF1000F03D13F4BD9
:10B4C0005B7B002B4FD094F80DC01CF0010FACF14A
:10B4D0000C031DD1BCF1030F07D8DFF8E8901EF074
:10B4E000040F3B4A08BF4A4600E0364AACF1040C60
:10B4F000BCF1070F05D8DFF81CC11EF0010F18BF03
:10B500006246DBB2032B0ED81EF0020F3C4B06E066
:10B51000DBB2032B06D82F4B2A4A1EF0020F18BFAE
:10B520001A4600E0274A4FF0000C5FFA8CF3834282
:10B530000DD20B6803EB8C035B881B0642BFD2F86D
:10B540000090214B43F82C900CF1010CEDE785B1F4
:10B55000BEF1000F08D0637B184A0133DBB2142B15
:10B5600006D1002304E025B1637B002BF3D100E07A
:10B570005373002E52D0234A3223B2F90250B2F94B
:10B580000020002DB8BF6D42002AB8BF524295FB83
:10B59000F3F592FBF3F2EDB2D3B2AB4238BF2B46D8
:10B5A000194A13B192FBF3F300E0134643442360BE
:10B5B000E37B024A83BB01232FE000BFF020002081
:10B5C000E41C00209A880108A208002052300020C4
:10B5D0008488010874880108E81C0020907801081C
:10B5E000081A0020967801089C780108A2780108C2
:10B5F000A8780108AE780108342E0020043000201D
:10B600008C8801084C110020400D03002C2F0020D5
:10B6100090190020948801080023D3738F4D904B1C
:10B620002D78E27BADB9002F00F00F818D4B267B8A
:10B630001A788D4B02F0040293F800C08B4BD2B203
:10B64000D3F800E00B680021894D03EB86060F4616
:10B65000B5E01AB9874A1A61002508E0864AFAE778
:10B660000A68AB00D6187688760604D40135EBB2AA
:10B670008342F5D3D7E7814EB6F90060192E25DD58
:10B6800012F803E094F814C00EF00F09E1452669A2
:10B690000CDCDFF8CCC19CF815C0BCEB1E1FDEBF74
:10B6A000D6F800C0DFF8D8E143F80EC012F803E086
:10B6B00094F816C00EF00F09E14533DBDFF8A0C1A6
:10B6C0009CF815C0BCEB1E1F2CDC26E0193629DACD
:10B6D00012F803E094F814C00EF00F09E145266952
:10B6E0000CDCDFF87CC19CF817C0BCEB1E1FA2BFAE
:10B6F000D6F800C0DFF888E143F80EC012F803E086
:10B7000094F816C00EF00F09E1450BDBDFF850C1CD
:10B710009CF817C0BCEB1E1F04DBD6F800E0584EA7
:10B7200043F806E0554EB6F90260192E1BDD12F8FB
:10B7300003C094F814E00CF00F09F14526690CDC05
:10B74000DFF81C9199F81590B9EB1C1FDEBFD6F8F5
:10B750000090DFF82CC143F80C90D25C02F00F0C83
:10B76000F4451EDD82E7193680DA12F803C094F83A
:10B7700016E00CF00F09F14526690CDBDFF8E090CC
:10B7800099F81590B9EB1C1FDEBFD6F80090DFF8D2
:10B79000F0C043F80C90D25C02F00F0CF445FFF6B9
:10B7A00065AF94F817E0BEEB121FA2BF3668344AAB
:10B7B0009E505BE75888000504D404330435B34237
:10B7C000F8D122E04AB101EB0C0A06209AFBF0F90D
:10B7D00000FB19A001280DDC01E057B9012793F8FF
:10B7E00001900EEB89003EF829A090F80290C078F5
:10B7F00003E01746002081468246013125F802AC5D
:10B8000085F800906870C9B2D7E7174A1378013BF2
:10B8100013F0FF0308BF06231370124B1B785B075E
:10B8200041BFBBF906304FF47A72A3F57A7303EB8C
:10B83000C30348BF93FBF2F3124A46BF0133DBB2A6
:10B84000012392FBF3F34344A36003B0BDE8F04F40
:10B8500001F028B903B0BDE8F08F00BF8F0E0020C3
:10B86000F0200020523000200E000020E41C0020B8
:10B87000A4080020908801089A8801084C11002033
:10B88000A2080020400D03002DE9F04F87B003937C
:10B89000904B81461B889346980737D540F2E63295
:10B8A000109B8D48DC89B0F900301B1B03F2F315A7
:10B8B000954203D8002BB8BF5B4201E04FF4FA7306
:10B8C000B0F9022040F2E630121B02F2F314844277
:10B8D00003D8002AB8BF524201E04FF4FA729342F3
:10B8E000B8BF13460522C3F5FA7393FBF2F30A229D
:10B8F000643B534399F81C20D2105343642293FBBA
:10B90000F2F3134423EAE373DBB200E06423C84696
:10B910000093CB1C02930025029B022D13F8016FAC
:10B920006E4F02934FEA450A05D1B7F904301B3632
:10B930005E43761149E06A4B37F9152033F915302B
:10B9400003EB4202CBF100039A4203DB5A45134654
:10B95000A8BF5B46634A32F90A40039A1B1B32F9BF
:10B9600015402344019304F0FDFC019B88B15E4A1D
:10B970001846545D06F022F95C4906F027FA0146A4
:10B98000204605F099F8594906F06CF906F030FBAD
:10B990000346504A1288D10713D437F90A401B36A0
:10B9A000664392074FEA26160FD599F812409DF983
:10B9B000002063435343642293FBF2F306EB231608
:10B9C00003E099F808405C432611494B042433F9FD
:10B9D0000A3098F8017093FBF4F4341B6743454E2A
:10B9E000022DAB5D03FB07F701934FF0640397FB58
:10B9F000F3F74FEAE7170AD1384606F0DFF8311DB2
:10BA00001E22F368FDF700FC06F0F2FA0746394BF8
:10BA100098F80B60198A03F1140E01FB04F25EF82A
:10BA20002500D21206FB0206334AB6F5001FA8BF56
:10BA30004FF400169642B8BF164603F1200252F8A2
:10BA4000250042F825404FF6FF720909B2FBF1F1DB
:10BA5000201A484399F850404EF825604FEA850C6B
:10BA6000761380118CB1CDF810C0059306F0A6F8BE
:10BA7000059B224603F12C0101EBC501DB68FDF7B4
:10BA8000C3FB06F0B5FADDF810C098F815301B4A74
:10BA90005843019BB91943431846642390FBF3F3C1
:10BAA0001B12194422F80A10013502F108014CF862
:10BAB0000170032D02F1140102F120024CF8016023
:10BAC0004CF8023008F101087FF426AF07B0BDE85A
:10BAD000F08F00BF081A00202C2F00204C110020EE
:10BAE0004C3000202A2E0020B478010800002041AC
:10BAF00088100020082100200000E0FF4C210020D9
:10BB00002DE9F04F87B00393A64B80461C88029125
:10BB100004F00204A4B2019294B1A34BB3F9024021
:10BB2000B3F90030002CB8BF6442002BB8BF5B42B1
:10BB30009C42B8BF1C46B4F5007FA8BF4FF4007408
:10BB4000C2460025984B994933F91520984B4FEA86
:10BB5000450B33F91530520083EAE376A6EBE37622
:10BB6000B6F5206F4FEA850951F8250011DC04264F
:10BB700093FBF6F3D31A0344B3F57A5F8D48A8BF5D
:10BB80004FF47A538342ACBF41F8253041F8250089
:10BB900002E0002341F8253051F809709AF80B3083
:10BBA000FF119AF801605F437E4B56431B88BF111B
:10BBB0009B074FEAA61656D07F4B3BF903301A4439
:10BBC000019B5B429A4203DB019B9342A8BF134651
:10BBD0007A4A3BF902209B1A039A32F915201A443B
:10BBE000049204F0BFFB049A98B1754B10465B5D5C
:10BBF000049305F0E3FF734906F0E8F8049B01465F
:10BC0000184604F059FF6F4906F02CF806F0F0F9D9
:10BC1000024642F210706C4959F8013013448342D5
:10BC2000A8BF034669488342B8BF034649F80130BC
:10BC300098F8081098F81C004A4300EB8000D211D5
:10BC400041428A4203DB8242A8BF0246114698F86D
:10BC50001220761A53431B13FF1A6743664303EB04
:10BC6000672701EB6626524B4FF0040C3BF803E0CC
:10BC7000574B0FFA8EF292FBFCF003F17801495D0D
:10BC80004143A6EBA11603F17C013BF901002BF81F
:10BC900001E0101A98F8502090FBFCF072B1059367
:10BCA000049205F08BFF059B049A03F12C0101EB34
:10BCB000C501DB68FDF7A8FA06F09AF9444B0AF1D2
:10BCC000010A03F1800212F805C0F2190CFB00F022
:10BCD0004011121A03F144012BF8012003F14C0228
:10BCE00049F8026003F1580249F80270404203F13A
:10BCF000640249F802000DB9012523E72A4A04200D
:10BD0000B2F90410029ADC6992790F3252004A4368
:10BD100027495211B1F90410002A91FBF0F0A2EB6F
:10BD20000000B8BF5242322A98F80D100BDC01FB1C
:10BD30000041284A8A42A8BF0A4627498A42ACBF26
:10BD4000DA61D96101E00022DA6198F8031001FBA1
:10BD500000F222499211097803290CD9B8F84E1043
:10BD6000B1F5FA7F07D24842824203DB8A42A8BF7C
:10BD70000A4600E00246D9696FF0FF0041F34F31F7
:10BD8000B1F5807FA8BF4FF480718142B8BF0146F2
:10BD90005A6550180022A3F848001966DA6607B001
:10BDA000BDE8F08F081A00204C1100201C21002053
:10BDB0008810002080C1FFFF4C3000202A2E002078
:10BDC000B47801080000204178210020F0D8FFFF5E
:10BDD00008210020FEFFFF0F020000F0482900208C
:10BDE0002DE9F04F89B00593BD4B0026B3F90270E1
:10BDF000B3F90030002FB8BF7F42002BB8BF5B42C1
:10BE00009F42B8BF1F468046B246B3463446B7F598
:10BE1000FA7F04910292A8BF4FF4FA77009001963E
:10BE2000B04D2B88990758D0AD4B610033F91420E1
:10BE3000AD4B33F9143003EB4202029B5B429A4252
:10BE400003DB029B9342A8BF1346A84A31F9029034
:10BE5000059AC9EB030332F9140003EB000904F05F
:10BE600081FA90B1A24B484613F804B005F0A6FE43
:10BE7000A04905F0ABFF0146584604F01DFE9D4960
:10BE800005F0F0FE06F0B4F8814698F80830642218
:10BE900003FB09F393FBF2F398F81C206FF0040BFB
:10BEA0000BFB02FB5B4504DB02EB820B9B45A8BF4F
:10BEB0009B4642F21072904B53F824004844904243
:10BEC000A8BF10468D4A9042B8BF104643F82400E0
:10BED00098F812305843031301932D8805F003039B
:10BEE000012B37D07E4B864933F914A0009BA60066
:10BEF00093F801C0834B51F824E033F9140080EA31
:10BF0000E073A3EBE073B3F5206F16DC502303FB63
:10BF10000AF292FBFCF3042290FBF2F0181A86441A
:10BF2000BEF57A5F784BA8BF4FF47A5E9E45ACBFF2
:10BF300041F824E041F8243002E0002341F82430A5
:10BF40008B597D2693FBF6F6009BDB7A73434026E4
:10BF500093FBF6F6AA0711D507FB06F507FB0AF9CE
:10BF60000198C7F5FA7303FB0B9903FB00534FF4D9
:10BF7000FA7199FBF1F293FBF1F505E0EB0759BF7C
:10BF8000354652465A46019D630003935D4B04209B
:10BF900033F814E0DFF874C10FFA8EF393FBF0F975
:10BFA0000CF17801615C01FB09F16FF04F0991FB25
:10BFB000F9F991440CF1840232F9141022F814E0DA
:10BFC00098F850205B1A93FBF0F08AB1CDF81CC0B2
:10BFD000069205F0F3FDDDF81CC0069A0CF12C0169
:10BFE00001EBC401DCF80C30FDF70EF906F000F8A7
:10BFF000464B03F18002115D09EB05024843202105
:10C0000090FBF1F00399121A03F1440E21F80E206F
:10C0100003F14C0242F8249003F1580242F82450F4
:10C02000404203F1640242F82400009A0132009277
:10C030000CB90124F4E62A4A0420B2F90410049A47
:10C04000DC6992790F3252004A432E495211B1F9FC
:10C050000410002A91FBF0F0A2EB0000B8BF52429E
:10C06000322A98F80D100BDC01FB0041284A8A4265
:10C07000A8BF0A4627498A42ACBFDA61D96101E00C
:10C080000022DA6198F8031001FB00F222499211B4
:10C09000097803290CD9B8F84E10B1F5FA7F07D208
:10C0A0004842824203DB8A42A8BF0A4600E00246B9
:10C0B000D9696FF0FF0041F34F31B1F5807FA8BF20
:10C0C0004FF480718142B8BF01465A655018002272
:10C0D000A3F848001966DA6609B0BDE8F08F00BF22
:10C0E0004C110020081A00204C3000202A2E00207D
:10C0F000B47801080000204178210020F0D8FFFF2B
:10C100001C2100208810002080C1FFFF0821002092
:10C11000FEFFFF0F020000F0482900202DE9F04F3C
:10C12000054690F850008DB0099106920A9318B117
:10C130003228A8BF322000E0012005F03FFD014673
:10C14000A94805F043FEA94B04461888002808BFFB
:10C15000012005F033FDA649079005F083FD01900D
:10C160000199204605F076FC0146019805F02EFE67
:10C17000A04B08901B889A0724D59F49B1F900303D
:10C18000B1F9020083EAE37280EAE071A2EBE372A4
:10C19000A1EBE07191420C46B8BF1446B4F5E17FC3
:10C1A00012DA914203DD0028D8BF404203E0002BA1
:10C1B000CCBF1846584205F001FD904905F006FE37
:10C1C000064603E0002601E04FF07E564FF00008DF
:10C1D00004950024CDF8088063000593884B33F95B
:10C1E000140005F0EBFC874905F03CFD05F000FF6D
:10C1F00005F0E4FC844905F035FD7F4B039033F9ED
:10C20000140005F0DBFC7B4B07461B889B077ED0A8
:10C21000014605F01FFC7D4B804633F9140005F004
:10C22000CDFC0146404605F015FC05F0E1FE069BFD
:10C230005B42984203DB069B8342A8BF0346744AD5
:10C240000599885E0A9A1B1A32F91400184405F001
:10C25000B5FC804604F086F870B16E4B40466E49DE
:10C2600014F8039005F0B2FD0146484604F024FCA2
:10C27000694905F0F7FC8046287F05F09BFC67497B
:10C2800005F0F0FC8246287A05F094FC0146404611
:10C2900005F0E8FC624905F0E5FC05F0A9FE8146E1
:10C2A0000AF1004005F0A4FE814505DB504605F08B
:10C2B0009FFE4845A8BF484605F080FCDFF884A1F2
:10C2C00002900199404605F0CDFC5AF8241005F083
:10C2D000C1FB54494FEA840B804605F061FE38B932
:10C2E0004046514905F07AFE20B1DFF83C8101E07B
:10C2F000DFF830814AF80B80A87C05F05BFC014632
:10C30000404605F0AFFC494905F0ACFC8046394B8E
:10C31000B3F800A01AF0010F40F09680384B059A50
:10C320004FEA840BD35EDFF81491002BB8BF5B4259
:10C33000B3F5206F03DD002349F8243029E03C49A0
:10C34000384605F08FFC049B0B90587805F032FCC2
:10C350000B9A0146104605F039FD039905F078FB6C
:10C36000019905F07FFC59F8241005F073FB314961
:10C37000814605F015FE38B948462F4905F02EFED6
:10C3800020B1DFF8B49001E0DFF8A8902B4A42F822
:10C390000B90049BD87A05F00DFC284B53F8241021
:10C3A00005F060FC264905F05DFC1AF0020F81469D
:10C3B0004CD03846029905F04BFB0146304605F05B
:10C3C00051FC0146029805F045FB414607464846A8
:10C3D00005F03EFB0146304605F044FC0146404670
:10C3E00005F038FB814631E083F9223E64100020DD
:10C3F000BD378635081A00204C1100200000E143AB
:10C40000881000200000A03ECDCC4C404C300020D5
:10C410002A2E0020B4780108000020410000A0402E
:10C420006F12033C0000F0C10000F0410AD7A33DA9
:10C430000000A043000040C30000404398210020BA
:10C440000AD7233C90210020C146029FDFF820A29A
:10C450000AF17802105D05F0B1FB0146039805F082
:10C4600001FC7B4905F0FEFB0146384605F0F0FA79
:10C470000AF19C0B5BF824100746039805F0E8FAD4
:10C48000019905F0A3FC039B0AF1A4024BF82430A8
:10C4900052F824B00392594605F0DAFA014608989A
:10C4A00005F0E0FB0146584605F0D4FA039A8346AE
:10C4B00042F824000AF18002105D05F07FFB01467E
:10C4C000584605F0CFFB634905F0CCFB834649464F
:10C4D000384605F0BFFA594605F0BAFA08F084FF6D
:10C4E000059B0AF14402D0520AF14C0238460392ED
:10C4F00005F07EFD039A0AF1580742F824004846E9
:10C5000005F076FD47F824000BF1004005F070FDC2
:10C51000049B0AF16407013347F8240004930CB923
:10C52000012459E6099A4C4B9479B3F9043064001C
:10C5300028345C43494B6411B3F9040005F03EFB19
:10C540004FF07A5105F08EFB08F04EFF201A05F0EF
:10C5500035FB002CB8BF6442322C064603DD0023B5
:10C56000CAF81C3027E0079805F042FD20F00300D0
:10C5700005F024FB0746687B05F01CFB01463046AE
:10C5800005F070FB36490446384605F01FFC0146AD
:10C59000204605F067FB05F02BFDDAF81C30184447
:10C5A000304B9842A8BF18462F4B9842ACBFCAF8F0
:10C5B0001C00CAF81C30DAF81C306FF0FF005B1367
:10C5C000B3F5807FA8BF4FF480739842B8BF184678
:10C5D00005F0F4FA0746304605F00AFDEB785843BB
:10C5E000801105F0EBFA214B04461B78032B11D97F
:10C5F000B5F84E50B5F5FA7F0CD205F0F9FC6B4258
:10C60000984203DBA8420346A8BF2B46184605F014
:10C61000D5FA04463946204605F01CFA05F0E8FC38
:10C6200000B205F0CBFA08F0DFFEAAF84800204679
:10C6300005F0DEFCCAF85400384605F0D9FC0023AA
:10C64000CAF86000CAF86C300DB0BDE8F08F00BFCA
:10C65000A69B443BF7CC92384C1100208810002058
:10C6600000803B45FEFFFF0F020000F0482900203C
:10C67000082100202DE9F84F4668D1F808A0D0F82D
:10C6800008904F680D68D0F8008051463046144637
:10C6900005F0E8FA39468346484605F0E3FA0146D4
:10C6A000584605F0D5F929462060484605F0DAFAE3
:10C6B00051468146404605F0D5FA0146484605F008
:10C6C000C7F939466060404605F0CCFA294607466E
:10C6D000304605F0C7FA0146384605F0B9F9A060C2
:10C6E000BDE8F88F2DE9F04106460D4640684968DF
:10C6F000144605F0AFF9A9688046B06805F0AAF9BC
:10C7000029680746306805F0A5F9C4F80480206060
:10C71000A760BDE8F0812DE9F04106460D460846C8
:10C720007168144605F09EFAB1688046284605F007
:10C7300099FA29460746306805F094FAC4F804804F
:10C740002060A760BDE8F08101380A4B042804D8B6
:10C75000DFE800F00507090B0D00074A08E0074A6B
:10C7600006E0074A04E0074A02E0074A00E0074AF9
:10C770001A607047340000208903010889B8000856
:10C780006506010801BB0008E1BD00081DC10008E5
:10C7900010F80A3C0133DBB20A2B84BF10F8131CDB
:10C7A000044A00F80A3C82BF002322F8113000F846
:10C7B0000A3C7047502F0020334A70B5136C9068C4
:10C7C000194440F68C23081A98429160D060516059
:10C7D00013463BD9127893F9451010468A420BD183
:10C7E000111F082908D893F84610182901D80131DB
:10C7F00003E083F8442002E0002183F8461093F917
:10C8000044402149A24219D191F84740B4B10C31BA
:10C810000024944206DA51F8046F1C4D25F8146088
:10C820000134F6E70C2805D01849002421F81040FF
:10C830000130F7E7164801780131017083F845208F
:10C84000002201211A7083F8471070BD92F847103A
:10C85000C9B140F2DA51A0F2EF248C4208D8117825
:10C860000B2905D80B1D0131117042F8230070BD52
:10C87000002283F84720074B03F13002002143F8E0
:10C88000041F9342FAD170BD54090020502F00209C
:10C89000B400002060090020024A136C01331944DF
:10C8A0001164704754090020024B53F820301B6874
:10C8B0001980704718290020074BA1F57A7153F8A9
:10C8C00020301A681B8959434FF47A7391FBF3F1B6
:10C8D00089B21180704700BF1829002037B504467F
:10C8E00003211E2006226B46F8F71EFB78BB9DF83D
:10C8F00001309DF80000174D43EA002000B205F01A
:10C900005DF9296805F0AEF905F072FB9DF803307A
:10C9100020809DF8020043EA002000B205F04EF9A5
:10C92000A96805F09FF905F063FB9DF80530A0802C
:10C930009DF8040043EA002000B205F03FF9696861
:10C9400005F090F905F054FB6080012000E0002024
:10C9500003B030BD1000002090F83B3210B57BB919
:10C9600090F83A3290F83942A34209D2B0F8401216
:10C9700001229A400A430133A0F84022DBB2F3E7D8
:10C9800010BD1FB50123ADF80830ADF80410002329
:10C9900001A9ADF80A30ADF80C30ADF8062000F072
:10C9A00072FE05B05DF804FB8379DB0748BFB1FA7E
:10C9B00081F1D0F8343148BF49095A681B8909B15F
:10C9C00013617047536170471FB50123ADF80830FC
:10C9D0000023ADF80C30ADF80A30094BADF8041067
:10C9E0001B7801A9012B08BF0323ADF8062008BF5F
:10C9F000ADF80C3000F047FE05B05DF804FB00BF59
:10CA00005009002038B510F80E2C044650F8043CAC
:10CA100052B9012200F80E2C20F80C1C997A1868E3
:10CA20000222BDE83840CFE730F80C2C20F80A1C71
:10CA3000891A89B220F8081C074A10F80F0C002543
:10CA400022F8101004F80E5C1868997A2A46FFF74D
:10CA5000BBFF04F8065C38BD502F0020044B53F890
:10CA600020301BB107289CBF1B681980704700BF8E
:10CA70007C0A0020084A13689B020BD5074B002153
:10CA800019704FF6FE730649086803400B604FF4B7
:10CA900000135360704700BF000002405130002077
:10CAA0006C0002402DE9F047664D2B686649581C22
:10CAB0000A788E4602F0FF060AB10346F6E73746CB
:10CAC0002B60687BAB6895F80C80AA7B39B2202973
:10CAD00000F09C80DFF880C10CEB8103DC789B7850
:10CAE0003CF82110C3F1FF039BB2002B65D04FF03F
:10CAF0003C0CB1FBFCF9C3F1FF0363431B12B9F11A
:10CB0000050F5DD8DFE809F0030B1A293A4AE01A4D
:10CB10004143B1FBFCF0DAB21044C0B251E0B1FBCA
:10CB2000FCF00CFB101189B2DAB2C1F13C01E31A3E
:10CB30004B43B3FBFCFC204694442CE0B1FBFCF0DF
:10CB40000CFB1011E21A89B24A43B2FBFCF25FFA05
:10CB500083F84244D2B2204632E0B1FBFCF90CFB30
:10CB6000191189B2E01AC1F13C014843B0FBFCF055
:10CB70005FFA83F84044C0B2224621E0B1FBFCF8E2
:10CB80000CFB1811D8B289B2E31A01FB03F2B2FB15
:10CB9000FCFC224684445FFA8CF412E0B1FBFCF802
:10CBA0000CFB181189B2D8B2C1F13C01E31A4B4316
:10CBB000B3FBFCF20244D2B203E02246204600E07E
:10CBC00044464FEA042C4CEA004C4CEA020C172372
:10CBD0004FF0010808FA03F806F1170118EA0C0FE4
:10CBE000A1EB0301DFF8748014BF4FF011094FF07F
:10CBF000090989B213F1FF3308F80190E8D2183619
:10CC00000137B6B2BFB2114BA0465FE7AB6001235C
:10CC10008EF8003040F22A33AA730D4AE9800D499C
:10CC200085F80C806873AE80536000238B840B887A
:10CC30009BB243F001030B80136843F001031360C0
:10CC4000BDE8F087B421002051300020C021002031
:10CC50006C00024000040040A2080020150B0020D8
:10CC6000F0B5B1F800E000234EFA03F2D50725D560
:10CC70008E784FEAD30CF40648BFCC7806F00F024A
:10CC800003F0070748BF2243BF0050F82C500F2481
:10CC9000BC4025EA0404BA402243282E40F82C2048
:10CCA00005D1C46801229A4024EA020205E0482E18
:10CCB00004D1C46801229A402243C2600133102B80
:10CCC000D2D1F0BD2DE9F04F1E464FF4147343430B
:10CCD000554D85B005F1100480469146E718A246EF
:10CCE00010B92B44514A03E0012805D1504A2B4486
:10CCF0001A641032C3F844214FF4147303FB08F391
:10CD00004C48EC180AEB030203F59C73343253448D
:10CD10002061E1636262A36200224FF480714FF0F0
:10CD2000010BD4F844310320E1612263E262216205
:10CD3000A263626384F84C2284F848B284F84922E2
:10CD4000A4F85222A4F85422C4F818906075A6756D
:10CD500084F8568258681B8904F5A0724FF0020CC3
:10CD6000ADF80C3003A9102301928DF80E308DF828
:10CD70000FC0CDF800C0FFF773FF236CDDF800C0D3
:10CD8000597B58681B898DF80E1003A9ADF80C303B
:10CD90008DF80FC0FFF764FF59463846FFF704FED1
:10CDA0003220FAF762FD244B019A1B68D2F804B0D6
:10CDB0001A46B2FBF9F1B1F5803F03D3012AF8D945
:10CDC0005208F6E71D4A4FF41474B3FBF2F204FB69
:10CDD00008F8584689B2D2B2FCF7BEF805EB08094C
:10CDE000174B08F512780AEB08040022C9F85832EC
:10CDF00058462146FCF7F8F8D9F8405016F0010FD4
:10CE00000CBF022200222868A97AFFF7BAFD0D4B59
:10CE10002846C9F85C32211D0022FCF7E5F83846A7
:10CE200005B0BDE8F08F00BFB4210020088C0108D8
:10CE3000288C0108B87801083C00002040420F000F
:10CE4000B7AE000819AE00082DE9F7438E46054637
:10CE5000DFF8A092114699F8B0440068164698464B
:10CE60007246631C89F8B034FCF722F82B8901A9BB
:10CE7000ADF8043018238DF80630686802238DF869
:10CE80000730FFF7EDFEAB7A09F2B44724012744DF
:10CE90002A6849460C2B00F2F680DFE813F00D00FB
:10CEA000F400F400F4005100F400F400F4008A00EF
:10CEB000F400F400F400C200138CDFF83CC223F04D
:10CEC00001031B041B0C1384138CB2F804E0108BB9
:10CED000624520F073004FEA00404FEA10409BB2D9
:10CEE0001FFA8EFE40F0700014D00CF5006C624505
:10CEF00010D00CF5406C62450CD00CF5806C62458E
:10CF000008D00CF5806C624504D023F0020343F096
:10CF1000030307E023F00E032EF4407E43F00303E7
:10CF20004EF4807EA2F804E01083A2F834801384CB
:10CF3000138B23F008031B041B0C43F0080336E09B
:10CF4000138CDFF8B4C123F010031B041B0C1384F3
:10CF5000138CB2F804E0108B624520F4E6404FEAEF
:10CF600000404FEA10409BB21FFA8EFE40F4E040B2
:10CF700008D00CF5006C624504D023F0200343F088
:10CF8000300307E023F0E0032EF4406E43F030035B
:10CF90004EF4806EA2F804E01083A2F83880138467
:10CFA000138B23F400631B041B0C43F400631383F3
:10CFB00069E0138CDFF840C123F480731B041B0C61
:10CFC0001384138CB2F804E0908B624520F0730058
:10CFD0004FEA00404FEA10409BB21FFA8EFE40F02D
:10CFE000700008D00CF5006C624504D023F4007387
:10CFF00043F4407307E023F460632EF4405E43F48F
:10D0000040734EF4805EA2F804E09083A2F83C8066
:10D010001384938B23F008031B041B0C43F00803B9
:10D0200030E0138CDFF8D0C023F480531B041B0CBA
:10D030001384108CB2F804E0938B20F4005023F496
:10D04000E6431B0400041B0C000C62451FFA8EFE15
:10D0500043F4E04340F4405003D00CF5006C6245CB
:10D0600003D12EF4804E4EF4804EA2F804E0938358
:10D07000A2F840801084938B23F400631B041B0CE4
:10D0800043F4006393832B7B43B1B2F844306FEADF
:10D0900043436FEA53439BB2A2F8443013889BB2D8
:10D0A00043F001031380AB7A0C2B19D8DFE803F0AF
:10D0B000071818180B1818180F18181813000B1940
:10D0C00002F134000AE00B1902F1380006E00B19F6
:10D0D00002F13C0002E00B1902F14000C3F8B40475
:10D0E00038460C44A4F8BC64C4F8B82403B0BDE8C6
:10D0F000F08300BFB4210020002C0140084BDA6807
:10D10000D10709D4DA68520708D4DB6813F0100F8E
:10D1100014BF03200420704701207047022070478D
:10D1200000200240704701207047704703788B420F
:10D1300086BF024B33F811000020704728270020DB
:10D1400008B50021062207F042FF012008BD08B5FE
:10D150000021062207F03BFF012008BD70B50546FF
:10D16000FAF75CFB324CA369A061C31AB3F5FA5F0E
:10D17000E36182BF002384F8203084F8213094F8E2
:10D1800020302BB9A12D02BF294A012182F821109C
:10D1900094F82110264A31B1D118EDB2013381F84B
:10D1A000225082F8203094F8205094F84330AB425B
:10D1B0003CD11F4B93F84430052B02D0062B03D0F3
:10D1C0002FE0002004F064F994F823301E2B28D1BE
:10D1D00000200246C1B26B1E99421ADA214491F82E
:10D1E00022300821DBB283EA0206F60744BF83F04F
:10D1F0001803C3F3460301F1FF3154BF5B0843F04A
:10D20000800311F0FF01C2F34702ECD101301A464E
:10D21000E0E7234493F822309A4202D1032004F03D
:10D2200037F9002384F8213084F8203070BD00BF26
:10D230002827002010B50446B0F9000002F0B2FE25
:10D24000B4F9020002F0AEFEB4F90400BDE81040EB
:10D2500002F0A8BE10B50446006802F0A3FE6068A4
:10D2600002F0A0FEA068BDE8104002F09BBE2DE9D0
:10D27000F74F0120FAF7A8F9002488B3012C2FD822
:10D280004FF04C0909FB04FA174E06EB0A0808F1A7
:10D290009007BD7815B10134E4B2EEE790F90030A3
:10D2A00090F804E01846114B03228DE82400012178
:10D2B0002A4653F82E30FAF71EFB834660B106F17A
:10D2C0004800504429464A4607F081FE01231C4489
:10D2D000C8F848B0BB70E4B20120FAF75BF9CCE7BC
:10D2E00003B0BDE8F08F00BF28270020D8780108E0
:10D2F0000021222210B5104807F069FE0F4B0022D2
:10D3000019460F480424105C013283F8F40183F8B5
:10D31000F94105200024042A83F8F80183F8FB4131
:10D3200083F8FA0103F10803EBD10123A1F8F631E8
:10D33000522381F8F23110BD461300205411002011
:10D34000F996010870B50646441E14F8011F89B10C
:10D35000094D284607F071FE0028F6D005F10803B4
:10D3600098423FBF054B401BC018A31B38BF80F835
:10D370008831EAE770BD00BFFD9601085411002016
:10D38000031EB8BF2D2210B5B8BF58420C46B8BF17
:10D3900001F8012B0A22FCF763F8002303702046F2
:10D3A00010BD07B51C4B03F1E402C3F8E0201B4A93
:10D3B00092F890215AB1012A14D1032183F8E61082
:10D3C000072183F8E82083F8E7100C2208E0022107
:10D3D00083F8E610032183F8E82083F8E71007229A
:10D3E00083F8E4200E4A0F4B40201A60FAF7ECF85D
:10D3F00070B10122002390F9000040218DE80C005B
:10D40000094A4FF4E133FAF776FA003018BF0120E9
:10D4100003B05DF804FB00BF282700205411002052
:10D42000491201081C000020FD1201080120002102
:10D4300001F0AEBF174AF0B5164692F8E930D2F8BF
:10D44000ECE0032B10D85C1C0EEBC3039D1CE4B274
:10D4500008D09A88D10705D5104203D008E00131E1
:10D46000042907D12346ECE786F8E9300020F0BD17
:10D470009F7800210C2202FB01F3064D05F1F00C10
:10D480001CF803209742EAD12B4485F8E940D3F8F1
:10D49000F400F0BD282700208A6810B50C6A0368E4
:10D4A00014430A6923F4FF4314434A6923F07003C9
:10D4B00014438A691443CA6914434A6A14438A6A42
:10D4C000224313430360CB6843600B6883604B685F
:10D4D000C36010BD4FF6FE73026813400360002363
:10D4E000036043608360C360284B984201D1284A9F
:10D4F00027E0284B984201D1254A2AE0264B984242
:10D5000001D1234A2DE0254B984201D1204A30E039
:10D51000234B984201D11E4A33E0224B984204D15A
:10D520001B4A536843F470032EE01F4B984204D10A
:10D53000174A536843F0706326E01C4B984204D1AD
:10D540001B4A536843F00F031EE01A4B984204D164
:10D55000174A536843F0F00316E0174B984204D182
:10D56000134A536843F470630EE0144B984204D19D
:10D570000F4A536843F4704306E0114B984204D1BC
:10D580000B4A536843F4702353607047080002400D
:10D59000000002401C0002403000024044000240F3
:10D5A000580002406C000240800002400804024023
:10D5B000000402401C0402403004024044040240C3
:10D5C00058040240224A10B5536803F00C03042BA0
:10D5D00003D0082B04D01F4B14E01F4B5B6811E0F5
:10D5E00053685168C3F38343C90303F1020301D4B1
:10D5F0001A4906E0516811F4003F1749496818BFFD
:10D6000049084B4303605368154CC3F30313234489
:10D6100093F820100368CB4043605168C1F30221A6
:10D62000214491F8201023FA01F181605168C1F37F
:10D63000C221214491F82010CB40C3605268C2F34C
:10D640008132224492F83020B3FBF2F3036110BD23
:10D650000010024000127A001C00002000093D006A
:10D66000D878010810B50446FFF748FD012806D117
:10D670001CB1FFF743FD013CF8E7052010BD002C6D
:10D6800008BF052010BD0A88F0B54B888E88B1F818
:10D6900008E0CC88002A3AD1028C43F0010322F042
:10D6A00001021204120C0284058B078CADB225F026
:10D6B000F30545EA0E1189B241EA06027A49BFB282
:10D6C000884212D001F5006188420ED0B0F1804F3F
:10D6D0000BD0A1F59831884207D001F580618842CE
:10D6E00003D001F58061884202D127F0020701E0F2
:10D6F00027F00A071F4302830784038B23F00C03E0
:10D700001B041B0C0383038B9BB21C4344E0042AC1
:10D7100044D1028C22F010021204120C0284018BFC
:10D72000058C21F440721205120D42EA0E325E4958
:10D7300092B242EA06228842ADB292B212D001F50C
:10D74000006188420ED0B0F1804F0BD0A1F5983126
:10D75000884207D001F58061884203D001F58061DD
:10D76000884207D125F0200141EA03139BB243F020
:10D77000100304E025F0A00143F010030B430283E3
:10D780000384038B23F440631B041B0C0383038B70
:10D790009BB243EA0424A4B20483F0BD082A028C9D
:10D7A0003ED122F480721204120C0284828B3E4D10
:10D7B00092B222F0F307018C47EA0E1292B2A8420D
:10D7C00089B242EA060212D005F50065A8420ED0E1
:10D7D000B0F1804F0BD0A5F59835A84207D005F5DC
:10D7E0008065A84203D005F58065A84207D121F4E1
:10D7F000007141EA03239BB243F4807304E021F4F7
:10D80000206143F480730B4382830384838B23F072
:10D810000C031B041B0C8383838B9BB21C4341E0D2
:10D8200022F480521204120C0284858B018C25F4A0
:10D8300040752D052D0D45EA062545EA0E321A4D97
:10D8400089B2A84292B212D005F50065A8420ED066
:10D85000B0F1804F0BD0A5F59835A84207D005F55B
:10D860008065A84203D005F58065A84207D121F460
:10D87000005141EA03339BB243F4805305E047F67D
:10D88000FF5543F480530D402B4382830384838BE5
:10D8900023F440631B041B0C8383838B9BB243EAFA
:10D8A0000424A4B28483F0BD002C0140CA78F0B5F2
:10D8B000D40648BF8C780D8802F00F0348BF23437D
:10D8C00015F0FF0F1DD0016800240126A64006EACE
:10D8D0000507B74211D14FEA840E0F2606FA0EF65D
:10D8E00021EA0601282A03FA0EF641EA060101D1CF
:10D8F000476102E0482A08BF07610134082CE4D1DF
:10D900000160FF2D1FD94168002404F1080701269A
:10D91000BE4006EA0507B74211D14FEA840E0F2632
:10D9200006FA0EF621EA0601282A03FA0EF641EA63
:10D93000060101D1476102E0482A08BF07610134AE
:10D94000082CE2D14160F0BD0F4B1A6842F0010291
:10D950001A6059680D4A0A405A601A6822F08472A7
:10D9600022F480321A601A6822F480221A605A68FF
:10D9700022F4FE025A604FF41F029A60044B4FF0EB
:10D9800000629A60704700BF001002400000FFF87C
:10D9900000ED00E02DE9F8435B4C0368013AC4F860
:10D9A000203183880D46A4F82431072A42D8DFE8C5
:10D9B00002F0040A101822292F35B4F820310B8008
:10D9C000B4F8223113E0B4F822310B80B4F82031DE
:10D9D00005E0B4F820315B420B80B4F822315B42A1
:10D9E00005E0B4F822315B420B80B4F820316B8043
:10D9F000B4F824311DE0B4F820315B420B80B4F858
:10DA0000223112E0B4F822310B80B4F820310CE05E
:10DA1000B4F820310B80B4F8223105E0B4F822319B
:10DA20005B420B80B4F820315B426B80B4F8243148
:10DA30005B42AB80354B1B7A002B62D1B5F90000FD
:10DA400004F0BCF88046B5F9020004F0B7F80746C8
:10DA5000B5F9040004F0B2F8D4F82811064640469F
:10DA600004F000F9D4F834118146384604F0FAF88D
:10DA70000146484603F0EEFFD4F840118146304697
:10DA800004F0F0F80146484603F0E4FF07F0ACFC70
:10DA9000D4F82C112880404604F0E4F8D4F838116A
:10DAA0008146384604F0DEF80146484603F0D2FFCE
:10DAB000D4F844118146304604F0D4F80146484673
:10DAC00003F0C8FF07F090FCD4F83011688040469E
:10DAD00004F0C8F8D4F83C118046384604F0C2F887
:10DAE0000146404603F0B6FFD4F8481107463046D9
:10DAF00004F0B8F80146384603F0ACFF07F074FCB8
:10DB0000A880BDE8F88300BF282700201C00002063
:10DB100044F6FB71084B1A68137803EB431300FBC0
:10DB200003135078C0EB0030B3FBF0F39078B3FBF5
:10DB3000F0F080B2704700BF2C19002008B50A48E9
:10DB40000A2290F84D3100EB4303B3F85C1100F565
:10DB5000B47089B220F8041C00F013F880B2FFF70B
:10DB6000D7FF024B188008BD28270020301900205D
:10DB700003689B68184703685B68184703681B685D
:10DB80001847B0F902302DE9F74F93421CBF00232C
:10DB9000037090F800A004460E469146BAF1000FBB
:10DBA00040F0B480104604F009F88B4904F05AF8AC
:10DBB0008A4904F057F84FF07C5104F053F80746B7
:10DBC000FBF7FCFD05463846FBF76AFE0146284692
:10DBD00004F0FCF80146054604F044F88049834609
:10DBE000284604F03FF8034658461946019303F0CF
:10DBF00031FF4FF07E5103F02DFF01464FF07E5074
:10DC000004F0E4F82946804604F02CF8294604F094
:10DC100029F807460146606003F01CFFE7604FF0FB
:10DC20007E572946A0602761284603F013FF294646
:10DC300004F018F84FF0804103F00AFF0146404617
:10DC400004F010F8019B60611946584603F000FF8C
:10DC5000394603F0FFFE0146404604F003F840F267
:10DC6000DC53A0462746554663651023A4F852307E
:10DC70001823A061A4F850304FF09741D8F8100055
:10DC800003F0F0FF0021824604F08AF928B15046E3
:10DC90004FF07C5103F0DCFE04E050464FF07C5125
:10DCA00003F0D8FE04F006FAC7E90E014FF09741E1
:10DCB000D8F8040003F0D6FF0021824604F070F982
:10DCC00028B150464FF07C5103F0C2FE04E05046AC
:10DCD0004FF07C5103F0BEFE04F0ECF90135032D4A
:10DCE000C7E9080108F1040807F10807C4D1A6F242
:10DCF000DC531B042367E3676367C4F88030A367C2
:10DD0000C4F884300123A4F802902370D4F854900E
:10DD1000B4F95280C9EB0606636A06FA08F6734343
:10DD2000276A4FEAE67B206F07FB0B332667A7FBCA
:10DD30000667E26F1F44636CD4F840C053434FEA58
:10DD4000E27B0CFB0B3ED4F88010C4F88020ACFBC7
:10DD500002237344B61A67EB0307E36AA26A4343DC
:10DD60004FEAE07B02FB0B3EA2FB00237344B61894
:10DD70005F41E36C656F4B436067A06C4FEAE17BEA
:10DD800000FB0B33C4F88410A0FB01011944636B42
:10DD9000361A05FB03F3206B4FEAE57B00FB0B33E0
:10DDA00067EB0107A0FB0501801919447941B4F91B
:10DDB0005020A56703F032FC08F1FF3201239340A5
:10DDC000E067C01841EBE371424603F027FC48448A
:10DDD00003B0BDE8F08F00BF6F12833ADB0F4940FC
:10DDE000F404B53F2DE9F0410024234BE0B293F851
:10DDF00030601F46B0420BD2204A53F8203032F830
:10DE000010101BB10B2801D8DB6898470134ECE7F0
:10DE10001B4B1B685B032CD500242346E2B2B242A5
:10DE200027D257F824204FEA840855689D4218D01D
:10DE30002846FBF7BBF8EFF31283502282F31288D7
:10DE40000D494FF0280EAA8C0EFB001092B2013241
:10DE50008265AA8ADBB292B242F00102AA8283F3FF
:10DE6000118857F8083000221B6801341A802B46AD
:10DE7000D4E7BDE8F08100BF18290020A8100020D9
:10DE8000342E002008B50E4B1B6813F4805F0D4B39
:10DE900014BFD3F8D420D3F8D82093F83010928848
:10DEA0000023D8B2884204D2074820F81320013357
:10DEB000F7E7FFF797FFBDE808403220F9F7D5BC38
:10DEC000342E002018290020A81000200A4B30B55D
:10DED0001A680A4B02F48052D3F8D440D3F8D850D1
:10DEE00000230AB1A18800E0A988054820F8131092
:10DEF00001330C2BF5D130BD342E00201829002021
:10DF0000F22B002070B5124D0024214605F1DD00F2
:10DF1000702285F8DC4007F05AF82146D5F85031D8
:10DF20000B4A0B4493F9020088B11E6802F1DD042C
:10DF30000E5108199C88073184809B797029837160
:10DF400092F8DC3003F1010382F8DC30E6D170BDD9
:10DF500018290020094B1A680E2303FB0020437A7E
:10DF6000FF2B07D0064A12789A4203D9054A32F8A5
:10DF7000130000E0808800B2704700BFEC1C002056
:10DF80000C2800202C2F00202DE9F04F834699B05B
:10DF9000894C94F85471254647B1012F40F05184C3
:10DFA000D4F89871D4F89C61002415E1F9F736FC97
:10DFB0000646C4F85801D4F86001301A03F0FAFD9F
:10DFC0007E4903F04FFE7E4BC4F85C015B6804F5AC
:10DFD000B270C4F86061984704F5B276002800F08A
:10DFE000E580784B30461A783146FFF7D3FCB4F819
:10DFF0006A31002B43D03B46D4F86C01B5F86A2156
:10E000007149B2F5C87F04BF002241F823204FEACE
:10E01000830C36F913E051F80C20674F724441F835
:10E020000C20002126F8131020F813100133032BC5
:10E03000E4D1B7F86A31012B1CD1D7F870314FF415
:10E04000C87EC83393FBFEF20280D7F87421C83231
:10E0500092FBFEF24280D7F878315C4AC83393FBDA
:10E06000FEF312889B1A8380ABF80010ABF8021005
:10E07000FBF70CFFB4F86A31013BA4F86A31544B4A
:10E080001B685B077ED5B4F87C214B4B322A13D139
:10E09000D3F86C211188A3F87E1151889288A3F8D7
:10E0A0008011A3F88221BBF80020A3F88421BBF8DB
:10E0B0000220A3F8862101E0002A41D0D4F86C8127
:10E0C0000020B5F87C314FEA800E322B414B04BF63
:10E0D000002243F8202053F80E1036F91020364F56
:10E0E0000A4443F80E20002326F8103028F8103098
:10E0F000013003281A46E4D1B7F87C31012B1AD13C
:10E100000C2087F8953187F89421F9F74DFBB7F883
:10E110007E31A8F80030B7F88031A8F80230B7F89F
:10E120008231A8F80430B7F88431ABF80030B7F882
:10E130008631ABF80230B4F87C31013BA4F87C3175
:10E1400094F896311C4AEBB1D2F88831322193FB16
:10E15000F1F3D2F86C51002082F896012B80D2F8AE
:10E160008C3193FBF1F36B80D2F89031174A93FB1B
:10E17000F1F312889B1AAB80ABF80000ABF80200F9
:10E18000FBF784FED4F86C21B4F8643111885B1A73
:10E19000A4F864315188B4F866315B1AA4F866318A
:10E1A0009288B4F868319B1AA4F8683194F8543115
:10E1B000013384F85431EBE618290020BD37863549
:10E1C000102C002054300020882A00200A00002053
:10E1D000342E0020A02A0020DFF8DC8208F5B2727D
:10E1E00032F81400B04A08F5D07522F8140000B2D5
:10E1F00003F0E4FC394603F035FDAC4A45F8240051
:10E2000032F9140003F0DAFC314603F02BFD08F577
:10E21000D67545F824000134032CDDD128462A4662
:10E2200008F5DC71FEF75EFA284608F5E27106AAE9
:10E23000FEF758FA06A80246D8F85C11FEF76BFA0A
:10E2400006984FF07C5103F00DFD4FF07C510646CF
:10E25000079803F007FD4FF07C510546089803F03E
:10E2600001FD31460446304603F0FCFC29460746D2
:10E27000284603F0F7FC0146384603F0EBFB214645
:10E280000746204603F0EEFC0146384603F0E2FB69
:10E290004FF07C5103F0E6FC01464FF07E5003F056
:10E2A000D7FBD8F8D491D8F8D831494601930290D9
:10E2B00003F0D8FC01990390204603F0D3FC039AA5
:10E2C0000146104603F0C6FBD8F8DC7103903946CE
:10E2D000284603F0C7FC039A0146104603F0B8FB3A
:10E2E000D8F8D0A103905146304603F0BBFC039A06
:10E2F0000146104603F0AEFB01990590029803F029
:10E30000B1FC39460390304603F0ACFC039A014659
:10E31000104603F09FFB51460390284603F0A2FCF1
:10E32000039A0146104603F095FB494603902046A8
:10E3300003F098FC039A0146104603F089FB494616
:10E340000490284603F08EFC01990390304603F0B8
:10E3500089FC039A0146104603F07AFB3946039084
:10E36000029803F07FFC039A0146104603F072FB0B
:10E3700051460390204603F075FC039A014610466F
:10E3800003F068FB51460390029803F06BFC49468A
:10E390008246304603F066FC0146504603F058FBC7
:10E3A00001990646284603F05DFC0146304603F01D
:10E3B0004FFB39460546204603F054FC01462846EB
:10E3C00003F046FB059BDDF810C0C8F8D431C8F84F
:10E3D000D001C8F8D8C1039A03F1004109A8C8F8D0
:10E3E000DC2102F100420CF1004C09910B92014634
:10E3F0000CAACDF828C0FEF775F92D48D8F8D01131
:10E4000012AAFEF788F90FAE09A8294915AAFEF746
:10E4100031F915A812A93246FEF764F90CA8314665
:10E4200015AAFEF727F93246214815A9FEF75AF931
:10E430001198D8F8E01103F0D1FD1E4B1A7810B1F5
:10E4400042F0080201E022F008021B4C1A70D4F8D6
:10E45000E43104F5F6771B7883B3D4F8E8913846B5
:10E46000494612AAFEF757F9D4F8F88104F5D0709E
:10E47000414615AAFEF74FF912A815A93A46FEF72C
:10E4800031F904F5FE70494612AAFEF744F9304608
:10E49000414615AAFEF73FF912A815A904F5FE7228
:10E4A000FEF720F916E000BF36110020881000208A
:10E4B0000C790108441900201829002004F5D073B4
:10E4C00004F5FE7593E8070087E8070096E8070063
:10E4D00085E80700D4F8A001D4F8A481014603F030
:10E4E000C1FB41460546404603F0BCFB01462846B9
:10E4F00003F0B0FAD4F8A87105463946384603F05F
:10E50000B1FB0146284603F0A5FA9A49074603F0F5
:10E5100065FD994E002520B93846984903F040FD25
:10E5200030B1C4F8C451C4F8C851C4F8CC5112E099
:10E5300006F5E27206F5F67006F5FE71FEF79AF83A
:10E54000D6F85C118E4803F041FC014606F5E270F6
:10E550000246FEF7E0F8B4F80832874D01339BB26B
:10E56000B3F57A7FA4F808324ED1D5F8D001D5F8AA
:10E57000D491014603F076FB49460646484603F02F
:10E5800071FB0146304603F065FAD5F8D88106469E
:10E590004146404603F066FB0146304603F05AFA16
:10E5A000D5F8DC7106463946384603F05BFB014678
:10E5B000304603F04FFA07F055F901464FF07E5010
:10E5C00003F004FCD5F8D411064603F04BFBD5F854
:10E5D000D8118146304603F045FBD5F8DC11804662
:10E5E000304603F03FFB31460746D5F8D00103F033
:10E5F00039FB0023C5F8D001C5F8D491C5F8D881FE
:10E60000C5F8DC71A5F80832D4F8D081D4F8D86107
:10E610004046314603F026FBD4F8D471D4F8DC51DF
:10E6200039460446284603F01DFB0146204603F008
:10E630000FFA014603F00EFA4FF07E51044603F044
:10E64000CDFC50B920464F4903F0AAFCE0B9204662
:10E650004FF07E5103F0C2FC08B14FF07E542046CB
:10E6600003F04EF906F020FF03F09EF90021044666
:10E6700003F0B4FC48B14449204603F0E9F9002115
:10E6800003F0ACFC88B923E0404C04F100493E495A
:10E69000484603F0DDF90021824603F09FFC90B16B
:10E6A0002046002103F09AFC30B12046364903F0A1
:10E6B000CFF94FF0010902E04FF00109504634490B
:10E6C00003F06EFC0FE02046002103F087FC08B148
:10E6D000204600E048462C4903F0BAF92D494FF096
:10E6E000010903F07BFC00B981465FFA89F353B15D
:10E6F00028464146FAF7E1FF014603F0ABF94FF037
:10E70000000A05467DE03946404603F0ABFA29464B
:10E710008146304603F0A6FA0146484603F09AF9CE
:10E72000014603F097F931460190304603F09AFA1A
:10E7300081463946384603F095FA494603F08AF98E
:10E74000014603F087F901464FF07E5003F080F94F
:10E7500000218246019803F019FC20B150460021A7
:10E7600003F014FCC0B951460198FAF7A6FF82469F
:10E7700014E000BFB81E8D3F182900203D0A673FF6
:10E780006F12833A000080BFDB0FC93FDB0FC9BFA8
:10E7900035FA0E3C35FA0EBC4FF0000A29464046C9
:10E7A00003F060FA31468046384603F05BFA0146D2
:10E7B000404603F04FF9014603F04CF9294606465E
:10E7C000284603F04FFA0146484603F043F9014654
:10E7D00003F040F901464FF07E5003F039F9002173
:10E7E0000546304603F0D2FB20B12846002103F055
:10E7F000CDFB28B929463046FAF75FFF054600E011
:10E8000000251549504603F02DFA06F0EDFD134E94
:10E8100011493080204603F025FA06F0E5FD104945
:10E82000708005F1004003F01DFA03F0E1FB80B2B7
:10E830000C4B10F4004F18BF00F5B4701880002383
:10E8400000E00123084A002182F85411002B7FF4D4
:10E850009FAB19B0BDE8F08F4D3D0F442A2E00202C
:10E86000E12E6542441100201829002010B54B8884
:10E87000DC0641BF2F4B14791B6853F8244044BF7A
:10E880002D4B43F820404B889B0641BF294B5479C0
:10E890001B6853F8244044BF274B43F820404B8863
:10E8A0001C070ED5254B0C781B78B3EB141FA1BFAA
:10E8B000204BD4781B6853F82440A4BF1E4B43F868
:10E8C00020404B889B070ED51D4B0C781B78B3EB73
:10E8D000141FDFBF174B54781B6853F82440DCBF6C
:10E8E000154B43F820404B88DC070FD5154C0B78AF
:10E8F000247803F00F03A342DFBF0E4B14781B688C
:10E9000053F82440DCBF0C4B43F820404B885B0796
:10E910000FD50B780C4903F00F0309788B42A1BF88
:10E92000044B92781B6853F82220A4BF024B43F893
:10E93000202010BDE41C0020A20800200721002098
:10E94000052100200421002006210020254A002363
:10E95000F0B515681C461A462348244903700B700D
:10E960002E1976884EB92F5D3FB9037000230A70C7
:10E970004B7007781C461A460CE0360548BF01323A
:10E9800004F1040403F1010348BFD2B2802CDBB2CE
:10E99000E6D1EAE7E0B2B8420CD215F8240001341F
:10E9A00006099E4200F00F00A8BF731C9042A8BF4A
:10E9B000421CEFE78A704B70C2F3470102F001027C
:10E9C0000A444C1E0A490B480A70C3F3470203F07D
:10E9D0000103134404700849501E084A087013705C
:10E9E000F0BD00BFE81C0020FC200020242B0020EC
:10E9F00006210020042100200721002005210020FD
:10EA0000924B2DE9F04FDA68914D1A612A6891B066
:10EA1000DA60904A0295136843F0200313608E4B2E
:10EA20001A78012A0CBF002201221A708B4B1A7827
:10EA3000910740F14D838A490978042940F24883BF
:10EA40008849097801F0040101F0FF0011B922F0B2
:10EA500001021A701B78DB0702D408B1FAF78CF9AF
:10EA60008149CA78531C052293FBF2F202EB820221
:10EA70009A1A7E4BCA701F7892000023DFF810822A
:10EA8000DFF8109258F82310794C91FBF9FE04F14D
:10EA9000080040F823E0774844F8231000FB0E11EB
:10EAA00042F2107091FBF0F004F1100680B226F8EB
:10EAB00013004FF0140C04F114060CFB036C04F16A
:10EAC0003C0A5AF823605CF802504CF80210761B9E
:10EAD000314405264AF8231091FBF6F109FB0E118B
:10EAE0004434012F44F823104FEA830B444605D1E8
:10EAF0000238B0F5797F98BF4BF808100BB90123A5
:10EB0000BCE7594E029BB2461868336DC01A03F039
:10EB100051F8594903F05AF9029B4FF07E511B6896
:10EB20000746336503F03CFA08B94FF07E574B4B6C
:10EB3000CAF854701B78514E13F00103504D12D097
:10EB40000DAA00924F4B0EAA01920CCB94E8030041
:10EB5000FAF728F80D9A6421B2FBF1F20E9B32808D
:10EB600093FBF1F300E033802B809AF858303E4D50
:10EB7000002B35D0696D4FF07E5003F027F9074622
:10EB8000EB6D2068C01A03F019F8394603F06AF8F3
:10EB900003F02EFA2B6E86B2606836B2C01A03F00C
:10EBA0000DF8394B196803F05DF8394603F05AF84F
:10EBB00003F01EFAB5F9662000B28118B5F9642099
:10EBC0000220B31891FBF0F193FBF0F389B29BB2F2
:10EBD000A5F86A10A5F86830A5F86610A5F86430A5
:10EBE00001238AF85830294B61681B88206803F09C
:10EBF00030031D4E264DCAF86010CAF85C00002B89
:10EC000000F0668206F17403009306F17803019325
:10EC1000F26E336FF9F7C6FF6B68306FC01A02F0FF
:10EC2000CDFF194B196803F01DF803F0E1F9F36EFD
:10EC30002A68C6F880009B1AF3670C4B1B78012BDF
:10EC40002AD0022B00F0E68042E200BF340200200E
:10EC5000582E002040190020D21000204419002016
:10EC60004A19002052300020242B0020600F002081
:10EC7000282B0020806967FF00007A44BE1900201D
:10EC8000C0190020D410002028000020081A0020FD
:10EC90004C19002080969800D6F88430D6F8A04011
:10ECA0000293D6F8943004F100400393D6F89830DC
:10ECB000776D059303F09CF98146204603F098F99F
:10ECC000D6F89C30BB4C0493BB4B06901B684FF0AE
:10ECD000000B0793B94E4FEA4B0356F82B80A6F171
:10ECE0001402404632F81B50089302F067FF029965
:10ECF00002F0B8FF03F07CF9401B1FFA80FA2836B7
:10ED000026F81BA00FFA8AFA504602F057FF039923
:10ED100002F0A8FF03F06CF986B20AEB080002F0DB
:10ED20004DFF059902F09EFF394602F09BFF2168D6
:10ED300002F090FE03F05CF9484504DB069B984224
:10ED4000A8BF184600E0484602F038FF206003F0F4
:10ED50004FF9079B304486B2987802F02BFF984910
:10ED600002F080FF01464FF07E5003F02FF8394645
:10ED700002F070FE0146384603F028F809906068FA
:10ED8000D4F808A0C0EB080002F018FF394603F0E1
:10ED90001DF8514602F05CFE099A0146104602F049
:10EDA00061FF0146504602F055FE3135ADB2622D8D
:10EDB00001462061C4F80480A0600ED9049802F0D6
:10EDC00051FF03F015F97F4AB0F5FA6FA8BF4FF471
:10EDD000FA609042B8BF104600E0002040F6B8321A
:10EDE000064436B29642A8BF1646774A089B96421A
:10EDF000B8BF1646754A54F8140B9E52142202FBF3
:10EE00000BF273495050BBF1000F40F061814FF09D
:10EE1000010B5FE7684BB6F8A8401F68736F3D8928
:10EE200002935B089D4228BF1D4623B29D4202DC2F
:10EE30001FFA85F90AE06749706D02F013FF03F0CD
:10EE4000D7F820441FFA80F9A6F8A890DAF878607D
:10EE5000DAF8AC40341B2046F9F7E6FE41F2931392
:10EE60000028D8BF40429842CCBF0020012078B390
:10EE7000204602F0A3FE584902F0F4FEFAF79EFC89
:10EE80000446029802F096FE0146204602F0EAFE91
:10EE900003F0AEF840F6B83380B2AAF8B00000B282
:10EEA0009842A8BF1846484B9842ACBF3018F0189B
:10EEB00048F6A043984203DDA0F50C40A03804E0DA
:10EEC0000028BCBF00F50C40A030CAF8B40001E037
:10EED000CAF8B460DAF8B4300026C3F50C50283014
:10EEE000039302F06BFE3C4902F0BCFE0446FAF7C5
:10EEF000D7FC0F902046FAF761FCDAF8B830DAF860
:10EF0000C4400593DAF8BC300E9004F10040089339
:10EF100003F06EF80490204603F06AF8DAF8C03087
:10EF2000DAF854802A4C09900793730048460A93F4
:10EF300002F044FE0EAB53F8261002F093FEDFF809
:10EF4000A0A005463AF9160002F038FE0146284610
:10EF500002F07EFD03F04CF805B2204BB5F57A7F48
:10EF6000A8BF4FF47A759D42B8BF1D460AF13C0A0E
:10EF7000A8B22AF8160000B202F020FE05998246D7
:10EF800002F070FE03F034F8089983B250460693FD
:10EF900002F068FE414602F065FE216802F05AFD6B
:10EFA00003F026F8049B98421CDB099B9842A8BFFB
:10EFB000184618E09C0F0020640F0020A02B0020B2
:10EFC000DB0FC94030F8FFFF48F4FFFF6E0F002051
:10EFD000C40F00200000C842D302373918FCFFFFDD
:10EFE0008C2B0020049802F0E9FD20608346B8785D
:10EFF00002F0E0FD384902F035FE01464FF07E5048
:10F0000002F0E4FE414602F025FD0146404602F0D2
:10F01000DDFE0B906068D4F808A0281A02F0CEFD3F
:10F02000414602F0D3FE514602F012FDDDF82CC03D
:10F030000146604602F016FE0146504602F00AFD07
:10F04000656001462061A060079802F00BFE02F0A7
:10F05000CFFF069B1434034458469A4602F0C8FF7B
:10F0600040F6B832504400B29042A8BF10461B4A46
:10F070000A9B9042B8BF1046194A1A499852142266
:10F08000724342F801B00EB901264EE73B792BB12D
:10F09000039A642392FBF3F3134A13803B88029A8A
:10F0A000124C9A420DD9D4F8AC30A06FC01AF9F7BF
:10F0B000BBFD42F2107380EAE072A2EBE0729A426A
:10F0C00006DD0B4B01221A70B4F8C820064B1A80DB
:10F0D00011B0BDE8F08F00BFDB0FC94048F4FFFF5F
:10F0E0006E0F00209C0F00205C0F0020242B0020BE
:10F0F000600F002007B5064B06490093064B074AF0
:10F1000001930748074BFAF7AAFA03B05DF804FB2E
:10F11000FE88010835970108D38801083F97010848
:10F1200012970108F288010808B5037833B90C4B2F
:10F130000C481978BDE80840FAF791BA05F0E0FFED
:10F1400002280CD8064B0C221870074B02FB00302B
:10F15000064B06301860FAF7A5FC0548E5E708BD40
:10F16000F02B002046970108FC180020CC1000204E
:10F17000DC8C010808B503783BB90B4B0B4893F8BE
:10F18000AC17BDE80840FAF76ABA05F0B9FF0228E3
:10F1900008D8054B83F8AC07FAF7DEFBFAF7A6FCB4
:10F1A0000348E8E708BD00BF541100204A97010852
:10F1B000DC8C010838B5037803BB214B1B68013395
:10F1C0000F2B07D81F490C2202FB031295681C461F
:10F1D0002DBB00E01C4601340F2C01DD002400E0B3
:10F1E00005D818490C2202FB04129568BDB99C424F
:10F1F000F1D11548BDE83840FAF731BA05F080FF83
:10F200000F28044605D80F4A0C2303FB00239D68F2
:10F210002DB92146BDE838400C48FAF720BA084B12
:10F220001C60F8F7B1FA21462A460948FAF717FA9E
:10F230000C235C43034B185DBDE83840F8F7B4BAC3
:10F240002C00002018790108579701086D970108D4
:10F250008597010873B5037813B9F7F713FE3DE0FE
:10F260001F4901AA05F0ADFF0024014626462546A8
:10F2700099B134B1012C08D1084605F041FF06468A
:10F2800003E0084605F03CFF05461549002001AAA9
:10F2900005F097FF01340146EAE70B2D02D911482A
:10F2A0000C220BE0022C10D1A6F57A73B3F57A7F0D
:10F2B00007D90D484FF47A714FF4FA62F7F75FFD02
:10F2C0000CE00A4B03EB45035E80084B084803EB58
:10F2D00045032946B3F90220FAF7C1F902B070BD1F
:10F2E00047910108208F0108AA940108F02B002003
:10F2F0009C97010838B50D4C05462368834206D11A
:10F30000F8F774F8204600214C2205F060FEE36C0B
:10F31000AB4209D12846F8F769F8BDE838400448FF
:10F3200000214C2205F053BE38BD00BF70270020DD
:10F33000BC270020034B1A68D379591C1344D171A0
:10F34000187A7047E819002010B5FFF7F3FF84B270
:10F35000FFF7F0FF04EB002080B210BD10B5FFF7FF
:10F36000F3FF0446FFF7F0FF04EB004010BD10B5BB
:10F370000446054B21461868FEF700FC034B1B684A
:10F3800098796040987110BDEC190020E8190020B0
:10F3900038B504460D462420FFF7E9FF4D20FFF75E
:10F3A000E6FF002C084C14BF21203E20FFF7DFFFB2
:10F3B0002368002228469A71FFF7D9FF236893F843
:10F3C0004900BDE83840D2E7E81900200146002096
:10F3D000DEE710B50446C0B2FFF7C9FF200ABDE85A
:10F3E0001040C4E710B5044680B2FFF7F2FF200CCE
:10F3F000BDE81040EDE737B5828883680446100603
:10F400000D4641BF29494FF4CC7091F8AC1700FB71
:10F410000133D10542BF26490C20097802F03F0292
:10F4200048BF00FB0133042A12D006D8012A0DD0B0
:10F43000022A2FD193F900102DE0102A0AD0202A99
:10F440000AD0082A26D1B3F9001024E0197822E066
:10F45000198820E019681EE069461868F9F79AFFD4
:10F4600001461448FAF7FBF8F5B1E06802F0A6FB94
:10F470006946F9F78FFF01460F48FAF7F0F820695F
:10F4800002F09CFB6946F9F785FF01460A48FAF746
:10F49000E6F809E000210948FAF7E1F825B1084843
:10F4A000E1682269FAF7DBF803B030BD541100209F
:10F4B000F02B00206090010859900108AF970108D7
:10F4C000AB970108024B0146D869FEF757BB00BF56
:10F4D000F02B002010B5441E14F8011F21B1034B7E
:10F4E000D869FEF74BFBF7E710BD00BFF02B0020FB
:10F4F000F7B52A492A4B08782A4D1C682A4B05EB98
:10F5000080001A88D0F8C010284B29481B78009139
:10F510004FF47A71B4FBF1F1FAF7A1F8254B2648C4
:10F520001968264B0026B1FBF3F1FAF798F8244B43
:10F530001F68F3B205EB8302D2F8D010E9B10124C1
:10F540009C403C4217D0220715D01E4A0B20D25CAB
:10F5500000FB0323134A1C4802EB8303D3F8F0207B
:10F56000FAF77DF8022C06D1184B93F8281011B148
:10F570001748FAF774F80136DBE71648FFF7AAFFD9
:10F58000154B16481A88164B92B219884FF4FB6334
:10F5900003B0BDE8F040FAF762B800BF9019002050
:10F5A000582E002018790108301900203000002062
:10F5B000B29701083C000020F597010840420F0077
:10F5C000401900203800002005980108F02B002089
:10F5D0000D9801085598010866100020119801083F
:10F5E000641000202DE9F0410024804625460F4E8E
:10F5F0004146A759384605F06BFD58B139460C48CD
:10F60000FAF72DF830190021FFF7F5FE0948FFF74A
:10F6100061FF013540F6444314349C42E7D11DB9E3
:10F62000BDE8F041044855E7BDE8F081B87A01082B
:10F63000C990010855980108778F01082DE9F74F07
:10F64000824605F008FD054628B1012819D19AF82F
:10F6500000302A2B15D15948FFF73CFF0024584EA3
:10F660005848A159F9F7FBFF30192946FFF7C3FEA7
:10F670005548FFF72FFF40F6444314349C42EED127
:10F6800098E050463D2105F0D8FC002800F08D8020
:10F6900003461D4613F8012D202AFAD0441C2046AB
:10F6A00005F02EFD81462046F9F7DEFD0746CAEB40
:10F6B00005054FF0000B142404FB0BF4DFF8208148
:10F6C00008F5D073E6580193304605F0C4FC844633
:10F6D000314662465046CDF800C005F0C5FCDDF865
:10F6E00000C0019B002856D1EAB2624553D11D19D2
:10F6F0004444D4F8AC0102F061FA0146384602F005
:10F7000063FC002845D0D4F8B00102F057FA014656
:10F71000384602F04FFC00283BD0B4F8A4319A06DA
:10F7200058BF4F46142202FB0B881C0648BF2748CF
:10F73000D8F8A82142BF90F8AC074FF4CC7404FB72
:10F740000022D80542BF22480C24007803F03F0372
:10F7500048BF04FB0022042B39460BD004D8013BE0
:10F76000012B0CD817700AE0102B05D0202B05D0E8
:10F77000082B04D1118002E0176000E017603146C9
:10F780001448F9F76CFF2846002103B0BDE8F04F9C
:10F7900031E6114805E00BF1010BBBF19D0F8AD159
:10F7A0000E4803B0BDE8F04F94E6504603B0BDE804
:10F7B000F04F17E703B0BDE8F08F00BF4398010892
:10F7C000B87A0108C9900108559801085411002021
:10F7D000F02B00205898010863980108778F0108E2
:10F7E0001879010870B50546284605F034FC064630
:10F7F00058B9194B19485A79194BBDE8704003EBB9
:10F800008203D3F8E01DF9F72ABF2846154932468E
:10F8100005F02AFC60B91448FFF75CFE134C54F85D
:10F82000041F19B11248F9F71AFFF8E7114805E06B
:10F830000024114B53F8241019B91048BDE870404A
:10F8400048E62846324605F00FFC01340028F0D186
:10F85000014B0B4D5C71C7E75411002083980108E0
:10F8600018790108779001088F980108F886010837
:10F870007390010855980108FC860108778F0108EC
:10F88000DC8C010808B50748FFF724FE064BD86951
:10F89000F8F77DF8FEF7F6FAFAF734F8034A044B66
:10F8A000DA6008BDA2980108F02B00200400FA05D8
:10F8B00000ED00E008B50548FFF70CFE00F036F853
:10F8C000FAF74AF8BDE80840DCE700BFAE98010847
:10F8D00008B50448FFF7FEFDFAF73EF8BDE808401A
:10F8E000D0E700BFC49801080E4B1A786C2A15D1D6
:10F8F0005A88B2F5FB6F11D11A79BE2A0ED193F84E
:10F90000D5270020EF2A0BD113F8012B5040064ACF
:10F910009342F9D1B0FA80F0400970470020704757
:10F92000704700BF00F80108D8FF01082DE9F74F24
:10F93000E94C00214FF4FB62204605F048FBE74B01
:10F9400004F539721A60E64B00221A70E54B04F296
:10F95000AE7119606C232370032363714FF48073BD
:10F96000A3604FF41673A4F86431FA23A4F8663147
:10F970004FF4FA73A4F86C31012384F85E3184F8F3
:10F98000693184F86A3184F87C3184F88431052344
:10F9900084F8233240F2DC53A4F8963140F24C4311
:10F9A000A4F8983140F26C73A4F89A3140F27533A0
:10F9B000A4F89C3140F64303A4F89E31234620214D
:10F9C00084F868116E2184F87A110A2184F87B1179
:10F9D0002B2184F87D11212184F87E11232184F8C4
:10F9E0007F114FF4C871A4F88011032ACCBF012104
:10F9F000002102F1010283F8A01114BF1E2175211C
:10FA0000122A83F8A11103F10203EED140F27E41E4
:10FA1000A4F8401140F23A71A4F8421140F27E512C
:10FA2000A4F8481140F2EA5140F2DC50A4F84A111F
:10FA300040F2B4514FF4FA63A4F8C631A4F8CA31C5
:10FA4000A4F8CE31A4F8D231052384F8E031C823DC
:10FA500001264FF47A784FF0320BA4F8E431DFF846
:10FA60007C924FF4C8734FF01E0A1922A4F8E831B3
:10FA7000A4F84601A4F84C11A4F8C481A4F8C881E4
:10FA8000A4F8CC81A4F8D08184F8E26184F8E36121
:10FA900084F8E661A4F84481A4F84EB184F893A1F7
:10FAA00084F8E12100920190A4F8503184F8DF61DC
:10FAB00084F8EC61A4F852B184F8EF61FDF718FC0A
:10FAC000D9F80030009A00254FF00F0E257355210C
:10FAD00083F805E0DA714FF0220E2122D97083F805
:10FAE00006E02D215A744FF00E0E5322597383F8FD
:10FAF00010E0DA7619754FF0350E5A224FF4FA718C
:10FB000083F81AE01A72A3F84E100A2276494FF0D1
:10FB1000780E28279A7483F80AE064224FF0140EB6
:10FB200083F80BA083F80CA01A77DFF8E0C11D70F2
:10FB30005F705F759F709F75DD7583F804B09D736E
:10FB40001D76DD735D765F729E7783F850E0996372
:10FB5000D9636649C3F82CC0C3F830C09962DFF896
:10FB6000B0C16349C3F848C059634FF07F5A614937
:10FB700001984FF04B0CC3F820A0C3F824A083F8E1
:10FB80004CC04FF0000A4FF0460C5964C3F840A037
:10FB900084F8AE2784F8AFC784F8B6E7A4F8B807AE
:10FBA00084F8B0B784F8B15784F8B55784F8B257E1
:10FBB00084F8B35784F8B4571966152183F8681090
:10FBC0004D490420D9664D49009283F85C00A3F8A2
:10FBD0005850A3F85A50A3F8565083F8647083F82D
:10FBE0006570196746494748596783F87860FDF79B
:10FBF000A9FBD9F800300A2218464FF4487183F85F
:10FC0000115183F8125183F8137183F8146183F84A
:10FC10001851A3F8161184F8D621C82284F8D721E8
:10FC2000009AA4F8D88184F8DA51A4F8DC210E22D5
:10FC300002FB05326FF0170482F81941032482F8A1
:10FC40001A416FF02F0482F81B41072482F81C41EF
:10FC50006FF0230482F81D41052482F81E4101350E
:10FC60005A2480F8204180F821416422FF24082D85
:10FC700080F81F2180F822414FF0000100F10E00B2
:10FC8000D5D1C820A3F88A01142083F88C01A3F8E9
:10FC900090211E204FF4967283F88D01A3F89221D3
:10FCA0000120282283F8891183F88E01A3F894217A
:10FCB0000B46094D5A191033C02BC2F810A0F8D1C9
:10FCC00005F529700021402205F081F900230E4E30
:10FCD000EA1899591EE000BF54110020A41000201A
:10FCE000F02B0020CC1000208FC2F53C00006040BB
:10FCF0006666663F0000A0409A99193FF6287C3F4F
:10FD00003D0A773F60A30108C0870108CDCCCC3EF7
:10FD10000000404004330868382B234CC2F8A4028A
:10FD2000D5D104F509700021802205F050F906F1C3
:10FD30003801702204F5097005F03EF9FEF706FE61
:10FD4000D9F8006000230125314604F27C404FF4CD
:10FD5000CC7284F8D43784F8D25784F8D35705F09E
:10FD60002BF904F2146031464FF4CC7205F024F9FB
:10FD70000E4B1B681A68C4F8BA275A68C4F8BE2725
:10FD80009A68C4F8C2271A68C4F8C6275A68C4F823
:10FD9000CA279A680223C4F8CE2784F8D05484F87E
:10FDA000683603B0BDE8F08F54110020CC1000205D
:10FDB00038B5094B93F8D45765B9084C2068F7F764
:10FDC00015FB074B25601B78022B03D1BDE838409B
:10FDD000FDF74DBA38BD00BF54110020382C00206B
:10FDE000352C0020044B93F8D4371BB9034B18680B
:10FDF000F7F7CABD0020704754110020382C0020AE
:10FE000038B505460446204614F8011B21B1034BC2
:10FE10001868FDF7B3FEF6E7401B38BD382C00200C
:10FE20000FB407B504AB53F8042B05490020019328
:10FE3000F9F72AFB03B05DF804EB04B0704700BF8C
:10FE4000ADFF0008024B01461868FDF797BE00BFE2
:10FE5000382C0020F8B5011F06460023083051F861
:10FE6000042F02F120043F2C3AD802F108040F2C91
:10FE700006D80232032A04D9002B08BF012300E070
:10FE800002238142EBD1012B30680ED0022B1AD015
:10FE9000736800F0030003F003039B0043EA0010C3
:10FEA000B36803F00303184317E000F00F0040F0BD
:10FEB0004000FFF7C7FFB068736800F00F0040EA2A
:10FEC0000310C0B209E000F03F0040F08000FFF7EF
:10FED000B9FF3079FFF7B6FF307ABDE8F840B1E7F7
:10FEE00006F10C0734463A46002552F8043DAD00B1
:10FEF00003F18001FF2910D903F50041B1F5803FDE
:10FF000002D245F0010508E003F50003B3F1807F5C
:10FF100034BF45F0020545F00305B242E5D165F076
:10FF20003F00C0B2FFF78EFF05F00303022B2078DD
:10FF300007D0032B0CD0012B13D1FFF783FF607880
:10FF40000FE0FFF77FFF6078FFF77CFFA07808E005
:10FF5000FFF778FF6078FFF775FFA078FFF772FF73
:10FF6000E0780434FFF76EFFBC424FEAA505DBD111
:10FF7000F8BD10B50446C0B2FFF764FFC4F3072014
:10FF8000BDE810405EE710B504467F2C06D964F04A
:10FF90007F00C0B2FFF756FFE409F6E7E0B2BDE824
:10FFA00010404FE7430083EAE070ECE7084649E77A
:10FFB0002DE9F04F94498BB00B7813F0010F03F04B
:10FFC000040200F07C81002A40F086818F48066898
:10FFD00016F0806640F08081980700F1708143F050
:10FFE00004030B708A4B8B4F1A888B4B1A803B682B
:10FFF0001B0340F14581894B80201E70FDF71AFAE2
:020000040801F1
:1000000008B1FFF777F9864C2578012D40F038814B
:10001000844B93F8D21721B193F8D3270AB19142B8
:1000200003D3012283F8D22711E096460846BEF199
:10003000000F06D090FBFEFC0EFB1C0C7046E64643
:10004000F5E791FBF0F192FBF0F283F8D21783F819
:10005000D32793F8D4271AB1724A002182F8D41713
:1000600041F66901704A93F8D497126802EBC20214
:100070008A4284BF40F2E241B2FBF1F26B498CBF8D
:10008000D2B204220A70B9F1000F1FD18020F7F715
:100090009BFA8046D0B18021F7F772FA98F80620D3
:1000A000634B022153F822306070B3F5613F0CBFFF
:1000B0000222002298F900008DE8060080214A46BD
:1000C000F7F719FCDFF85881606008B90023D6E023
:1000D000494608F10800142204F079FF08F12803CA
:1000E000C8F81C3008F1A4034E49C8F8203008F5C0
:1000F0009073C8F824304F4B91F892013A681B88EE
:100100000028A8F89C31C2F3C03318BF012391F82E
:1001100084010593C2F3402C02F40063C2F340084B
:10012000454A04901068C0F38002C0F3C0094879C2
:10013000A0F119077C427C41012814BF2046012010
:10014000039091F8D20791F8D31788422CBF002171
:100150000121069139493A488A460078D1F800B021
:1001600002906F1EFFB2791E132945D8DFE801F017
:100170000C0C0C0C0C0C0C0C0AAEB031333D3F12C5
:10018000121241470399A4E00299B942B4BF002476
:10019000012430E09BF80010022913D1B91E5BF84E
:1001A00021000021CDF824C00893079201F0EEFE53
:1001B00007AA4FF0010492E80C1008B14FF00004B8
:1001C000E4B218E00BEB07014C79003418BF0124AE
:1001D00011E041467DE023B10499481E414241416E
:1001E00000E0194601F0010173E0614671E00599F4
:1001F0006FE006996DE014B10121B9400E43142D52
:1002000020D80135EDB2ACE7523000206810002054
:1002100044110020342E00205E0F00201128002001
:10022000342C002054110020182100204000002010
:10023000D87801088C28002040190020A410002044
:1002400048290020DAF80000254C79301921C4F83B
:10025000A061F7F745FA0023C4F8A831A4F8AC313F
:10026000A4F8AE31C4F8B8311E4BD4F8B4211B68E1
:1002700084F8A401C4F8BC31C4F8B021022323706F
:10028000184B194A1B6892F8E0214FF47A7101FB70
:100290000233164A1360164B1B681A0609D5154B14
:1002A0001B789B0705D5144B1B78042B01D906201E
:1002B00000E005200BB0BDE8F04FF7F775BA5AB96A
:1002C00001200BB0BDE8F04FF7F790BA494600E0C7
:1002D0001146002990D194E70BB0BDE8F08F00BF24
:1002E000342C0020582E002054110020180F00201C
:1002F000342E0020441900204A19002010B5154A58
:100300001378590725D523F004031370124B1B688B
:100310001B0319D5114C2378A3F10802012A0BD82D
:10032000FF200021F7F7CEFC0D4B1B68C4F8BC3151
:10033000FFF758FD0A2306E0012B05D90A2B03D04D
:10034000FFF736FD012323700420BDE81040F7F7C6
:100350002BBA10BD52300020342E0020342C002047
:10036000582E0020064B1B7803F0040303F0FF0017
:100370001BB1044B1888C0F3C01000F00100704797
:1003800052300020081A00202DE9F04F87B0039367
:100390009F4B0026B3F90280B3F90030B8F1000F8B
:1003A000B8BFC8F10008002BB8BF5B429845B8BF82
:1003B00098468346B246B1463446B8F5FA7F029273
:1003C000A8BF4FF4FA7800900196924D67002B88F1
:1003D00013F0030F55D0022C53D08D4BDA5F8E4BA8
:1003E000DB5F03EB4202029B5B429A4203DB029B10
:1003F0009342A8BF1346894AD05F039A1B1A32F969
:10040000140003440193FFF7ADFF019B90B1844AB0
:10041000184612F8049001F0D1FB824901F0D6FC95
:100420000146484600F048FB7E4901F01BFC01F004
:10043000DFFD03469BF8082064215A4392FBF1F24A
:100440009BF81C106FF0040909FB01F94A4504DB15
:1004500001EB81099145A8BF9146734A52F82400E7
:10046000184442F210739842A8BF18466F4B984246
:10047000B8BF18469BF8123042F8240058430313C3
:1004800001932A8802F00303012B01D1022C3CD1F5
:100490005F4B674833F907A0009BA10093F801E088
:1004A000644B50F82460DD5F85EAE573A3EBE573E8
:1004B000B3F5206F1CDC022C14D0502303FB0AF38D
:1004C000042793FBFEF395FBF7F55D1B2E44B6F571
:1004D0007A5F594BA8BF4FF47A569E42ACBF465044
:1004E000435007E08AEAEA73A3EBEA73642BE4DD86
:1004F000002343504E4B7D26CB5893FBF6F6009BD2
:10050000DB7A7343402693FBF6F6910713D5022C52
:1005100011D008FB06F508FB0AF70198C8F5FA7335
:1005200003FB097703FB00534FF4FA7297FBF2F1D8
:1005300093FBF2F508E0D30704D5022C02D0019D0D
:10054000494601E0354651463A4B042733F9143009
:100550003A4A93FBF7F3A25C6FF04F07534393FBC8
:10056000F7F3022C4FEA440C01EB03070FD1384696
:10057000CDF810C001F022FB314B32491E221B681E
:10058000F8F742FE01F034FD0746DDF810C0294BB4
:100590002D4A3CF803103CF902000BB22CF8021073
:1005A0009BF85020181A042390FBF3F082B1CDF889
:1005B00014C0049201F002FB2449214B01EBC40159
:1005C000049A1B68F8F720FE01F012FDDDF814C054
:1005D0001F4B204A1B5D5843202390FBF3F07B19EF
:1005E0001B1A2CF802301C4B404243F824701B4B62
:1005F00043F824501A4B43F82400009B0134013384
:10060000032C00937FF4E1AE07B0BDE8F08F00BF8C
:100610004C110020081A00204C3000202A2E002007
:10062000B47801080000204178210020F0D8FFFFB5
:100630001C2100208810002080C1FFFF80210020A5
:10064000142100200C210020F82D0020342100204E
:10065000882100204C21002054210020602100200E
:100660006C2100202DE9F04F89B00693974B0C4682
:100670001B888146990703924DD540F2E631129BC3
:10068000934AD889B2F900301B1A03F2F3158D4250
:1006900003D8002BB8BF5B4201E04FF4FA73B2F904
:1006A0000220101A40F2E63200F2F311914203D810
:1006B0000028B8BF404201E04FF4FA7099F84C505E
:1006C0003DB39842B8BF1846C0F5FA7001F076FA0B
:1006D000804901F07BFB4FF07E5101F0B9F90646ED
:1006E000642090FBF5F001F069FA0146304601F014
:1006F000B9FA4FF07E5101F0ADF90021074601F043
:100700004FFC30B938464FF07E5101F067FC20B104
:1007100001E0002701E04FF07E57C846E31C049338
:100720000024049B022C1A4612F8013F6A4E0193E2
:1007300004920AD1019DB6F904000A35684301F01C
:100740003DFA664901F042FB74E036F9140001F00D
:1007500035FA8246039801F02DFA5E4901F036FB26
:100760000146504601F07EFA5D4B824633F9140093
:1007700001F024FA0146504601F06CF9039B8246D1
:10078000584201F01BFA0546504629464FEA440BF1
:1007900001F006FC48B9039801F010FA05465046EE
:1007A000294601F01BFC00B955464E4A32F90B00B0
:1007B00001F004FA0146284601F04AF9069B8246F8
:1007C00033F9140001F0FAF90146504601F042F9FC
:1007D000454901F0FBFA8246FFF7C4FD28B1434BBF
:1007E0005146185D00F068F98246384B1B88DA07DD
:1007F00005D55046D9F8441001F034FA1AE0019DAD
:1008000036F90B0014356843029301F0D7F93349E8
:1008100001F0DCFA029B05469B070CD5D9F848107D
:10082000504601F01FFA394601F01CFA01462846ED
:1008300001F010F90546630005932D4B2D4E33F959
:10084000140001F0BBF92C4B996901F00BFA014639
:10085000284601F0FDF8D8F82010824601F002FA8F
:10086000264B0546185D01F0A9F90146284601F01E
:10087000F9F9234901F0AAFA022C019005D1214986
:100880001E223368F8F7C0FC0190336850461946C1
:100890000293DFF87CB001F0E5F9D8F82C1001F0F4
:1008A000E1F9114901F0DEF95BF8241001F0D2F80A
:1008B0001549A500064601F073FB58BB30461349A5
:1008C00001F08CFB38B3114E25E000BF081A002060
:1008D0002C2F00200000FA434C1100200000484259
:1008E0004C3000202A2E002000002041B47801085E
:1008F0008810002014210020F82D0020082100205D
:100900000000C8420C21002000007AC300007A4396
:1009100098210020374E4BF80560DFF804B15046AF
:1009200055F80B1001F094F80299079045F80BA0C8
:100930004FF07E5001F04AFA079B0146184601F03D
:1009400091F999F85020034632B12B49029B01EBF3
:10095000C401F8F759FC0346D8F83810184601F0DE
:1009600081F9264B8246185D01F028F90146504670
:1009700001F078F9224901F029FA2249824601F072
:100980000FFB38B95046204901F028FB20B1DFF8B1
:1009900078A001E0DFF86CA00198314601F05AF828
:1009A000514601F057F804F01FFD184BB0F57A7F5F
:1009B000A8BF4FF47A709842B8BF1846059A144BF6
:1009C0000134D052019801F013FB124B08F10408D6
:1009D0005851304601F00CFB0F4B5851504601F076
:1009E00007FB0E4B032C58517FF49BAE09B0BDE8BA
:1009F000F08F00BF00007AC33421002008210020BE
:100A00000000C842000096C30000964318FCFFFF98
:100A10004C21002054210020602100206C21002066
:100A2000142E0020044B00221A605A60034B00224F
:100A30001A605A60704700BF782100209021002082
:100A400010B50B4C0123E3704FF48060022384F84F
:100A50002030F8F73FFF074A074B926A1B6852782D
:100A6000642101FB0233636123880133238010BDBD
:100A700004300020F82D0020582E00200C4B0D498A
:100A8000DA684378D243C2F30222C2F104029340EF
:100A900002781B01DBB20A4482F80033037801229A
:100AA000580903F01F0302FA03F341F8203070479E
:100AB00000ED00E000E100E02DE9F74FAE4C2378B7
:100AC000013B012B00F253816678864240F04F8152
:100AD000A378022B00F04B81A84B9B5D7600E3705E
:100AE00023791BB1A319B3F9060007E0E36803F10A
:100AF0000043E360A319B3F90600404201F05EF839
:100B00009F4901F063F92369074618039A4D2BD5D5
:100B1000E86801F06DFA8DF80200686901F068FA82
:100B200097498DF80300384601F09CF804F098FCD2
:100B300001F084FA9249ADF80000A86901F092F83A
:100B400004F08EFC01F07AFA8D49ADF80400E869F2
:100B500001F088F804F084FC01F070FA6946ADF801
:100B600006000C20F7F7AEF8D4F81C8000214046B0
:100B7000814D01F00BFA002860D0D5F81880384676
:100B8000414601F02BFA18B1EB68AF616B61DAE016
:100B90004046002101F022FA002800F0D48095F8A8
:100BA00020303BB1022B00F2CE806B6BEF61FA3349
:100BB000AB63C8E0E968384600F04AFF4FF07E5169
:100BC0004FF0010501F000FA00B90546EDB28DB114
:100BD0006C49A06A01F046F8DFF8BC81664F4146D7
:100BE000814601F0DDF910B9C7F8289007E0C7F891
:100BF000288004E0A06A644901F034F8A062236907
:100C00005D4A190311D5116BD3788DF800500B4450
:100C10005A780B208DF80120DA7A69468DF8022087
:100C20005B7D8DF80330F7F74DF80123226B84F8D4
:100C30002030E37813440022DA7282E038464146DD
:100C400001F0AEF900B1EF61D4F81890D4F81CB0FF
:100C50004846594600F0FCFE636BA56B82465D1B5F
:100C60006FEA05084FEAD878B8F1000F0BD14FF0C2
:100C70007E5101F0B3F9002865D03846594601F09D
:100C8000ADF900285FD0484661694FF0010501F0D9
:100C9000A5F900B90546EDB23DB1606A394900F0E9
:100CA000E1FF39496062E06A07E050464FF0804159
:100CB00001F094F928B1E06A324900F0D3FFE06214
:100CC00004E0606A304900F0CDFF60622C49606A40
:100CD00000F0C8FF01F0B2F9D4F830A0E7785FFA6D
:100CE00080F9574487F80190E06A01F0A7F9236979
:100CF000C0B21B0378750ED545EA48058DF8005043
:100D00008DF80190FB7A69468DF803000B208DF871
:100D10000230F6F7D7FF94F82020174B022A0DD1A6
:100D2000002283F820201D6BDA78986A1749154451
:100D300000F098FF01F082F9E87202E0022283F8E5
:100D40002020F8F77BF822790B4B0AB1104A00E01B
:100D5000104A2644DA60B6F9060000F02FFF084971
:100D600001F034F80146E06800F072FE00E0084649
:100D700003B0BDE8F08F00BF242E00209888010842
:100D800000002041EC51783F0AD7833F00007A44AD
:100D90000000A0410000A0C16F12833A2B4BF0B5B8
:100DA0002B4D1E6805F110002F782C46F319597849
:100DB000013501F0040101F0FF0219B18542F3D1C0
:100DC0000020F0BD224D631B022B0ADD1AB102EB9D
:100DD00082025200D2B215F8013B303B1A44D2B223
:100DE000F1E70021AC420AD919B101EB81014900B8
:100DF000C9B215F8013B303B1944C9B2F2E72E2FB6
:100E000016D1013404200023257803EB83037719DE
:100E10007F785B007F079BB244BF303D5B1900F1D8
:100E2000FF3044BF01349BB210F0FF00ECD100E072
:100E3000002308484143642000FB03130620B3FB52
:100E4000F0F3054800FB0230F0BD00BF4400002075
:100E5000602E002040420F008096980000231A4622
:100E600030B510498C1894F83C40BCB12E2C06D1FA
:100E7000013298B18C180444002584F83C500A24AF
:100E80001144634391F83C10A1F13004092C9CBF3C
:100E9000303B5B180E2A03D80132E2E7184630BD1A
:100EA000002030BD242E00200EB40FB5074906AB3C
:100EB0000190074A01A80393F8F7E6FA019B002284
:100EC0001A7004B05DF804EB03B070479D91000800
:100ED0005D9101080028114AB8BF404290FBF2F32F
:100EE00030B50F4C3C2504FB030068430D4D90FBCF
:100EF000F2F22D682D7B25B903EB830303EB83030B
:100F000001E0C3EB031302EB830304FB02020B803B
:100F10004FF47A7392FBF3F24A8030BD80969800CA
:100F2000806967FF34190020022803D0431E58420D
:100F300058417047064B1B681B7823B1054B186856
:100F4000C0F3C0407047044B1878C0F3800070476E
:100F5000400E0020681000205230002010B50A4CCE
:100F60005E280146206805D15D21FCF707FE206858
:100F70003E2105E05D2903D1FCF700FE20683D21FC
:100F8000BDE81040FCF7FABD702E002010B50446F5
:100F9000C0B2FFF7E3FFC4F30720BDE81040DDE770
:100FA000024B5E211868FCF7E9BD00BF702E0020DF
:100FB00038B50546054C5E212068FCF7DFFD20684A
:100FC0002946BDE83840FCF7D9BD00BF702E00208F
:100FD00013B5044601A90068FFF77CFF1320FFF753
:100FE000E7FFBDF90400FFF7D1FF1B20FFF7E0FF8B
:100FF000BDF90600FFF7CAFF2320FFF7D9FF2368DA
:10100000002BB4BF53204E20FFF7C0FF01A960683A
:10101000FFF760FF1220FFF7CBFFBDF90400FFF7D9
:10102000B5FF1A20FFF7C4FFBDF90600FFF7AEFFBA
:101030002220FFF7BDFF6368002BB4BF5720452077
:10104000FFF7A4FF02B010BD674B73B51878FFF728
:101050006BFF664D04462B78834220D0C8B1644BA9
:101060001B68E3B193F9000002230093614B042154
:101070001B6800225B78003318BF012301934FF4F3
:101080001653F6F738FC5C4B186040B101232B7007
:1010900005E0594E3068F6F7A9F934602C70574BCB
:1010A000574D1878FFF740FF2B780446834218D03D
:1010B00088B1544B1B68A3B10022012493F90000AE
:1010C00008214FF4964300940192F6F714FC4E4B1E
:1010D000186028B905E04C4E3068F6F787F934609F
:1010E0002C704A4B4A4D1878FFF71EFF2B780446A8
:1010F00083422E4643D0002838D0464B1A68002A37
:101100003DD0D37992F90000002B4FF00202424CFF
:1011100008BF02230092002254F8233001921021CC
:10112000F6F7E9FB3D4B0546186040B33C4C94F89C
:101130004A30022B0BD094F89620022A01D14C346D
:1011400005E023B1002A04F14C0418BF0024354BFC
:101150001C6044B1204600214C2203F038FF0223DA
:10116000256084F84A300123337008E02B4E306844
:10117000FEF7C0F83068F6F739F934602C702A4B66
:101180002A4D1878FFF7D0FE2B780446834229D0E9
:1011900000B3274B1B682BB3264A93F90000126853
:1011A000032352782021002A0CBF08220922009331
:1011B00001924FF461430022F6F79DFB1E4B18602D
:1011C00080B11E4A012313702B701D4B1A681D4BF2
:1011D0001A6007E0184E3068F6F708F9174B3460CC
:1011E0001C702C7002B070BD480E00202C11002025
:1011F000440E002034190020702E0020490E0020DB
:1012000054190020D8190020C8190020540E0020BD
:10121000DE190020500E0020D8780108E0190020C7
:1012200070270020E4190020600E0020F41900202F
:101230005C0E0020580E0020F8190020FC19002038
:10124000582E0020001A002003788B420AD9064B42
:101250001A78064B53F8210002B1400800F5777068
:1012600080B270470020704710280020742E0020A4
:1012700007299DBF024B03EB8101088E00207047B8
:10128000742E0020034B03EB4101B1F85000C0085D
:10129000704700BF742E002008B5084B03EB810196
:1012A000086F00F087FC064900F0DCFC054900F0FF
:1012B000D1FB00F0C3FE80B208BD00BF742E002039
:1012C0000000203F00005C44024B03EB4101B1F8F9
:1012D000B8007047742E0020024B03EB4101B1F8B7
:1012E000DC007047742E0020024B03EB4101B1F883
:1012F000DC007047742E00200020704710B50446B3
:10130000F6F78CFA41F288310E4BE4B2D3F8F420B0
:10131000C3F8F400821A8A42C3F8F82084BF00227E
:1013200083F8FC2093F8FC2006490F2A134418BFC9
:10133000013283F8FD4012BF81F8FC20012381F8BF
:101340000D3110BD742E002010B50446F6F766FA74
:1013500041F288310E4BD3F81021C3F81001821AE4
:101360008A42C3F8142184BF002283F8182193F81D
:1013700018210749142A134418BF013283F8194170
:1013800012BF81F81821012381F82E3110BD00BF52
:10139000742E002038B50446F6F740FA274A27494C
:1013A000D2F83031C2F83001C31AB3F57A6F84BF76
:1013B000002382F8343192F8343133B9A82C3BD170
:1013C00081F83531A1F8363106E0022B02D181F8DF
:1013D000384101E0242B02D8D11881F8394192F824
:1013E000381101330231DBB249008B42134D82F8D0
:1013F000343118DAB5F83631E0B283EA0020082338
:1014000010F4004F4FEA400018BF80F4815003F100
:10141000FF3318BF80F0010013F0FF0380B2EFD15B
:10142000A2F8360138BD01318B4201BF002385F897
:101430003431012385F8353138BD00BF742E0020CA
:1014400010B50446F6F7EAF940F6AC510F4AD2F867
:101450006031C31A8B42C4BF002382F8643192F812
:101460006431D11881F8654123B90F2C0DD107499A
:10147000C1F860010133DBB2192B044982F86431F1
:101480000CBF0123002381F87E3110BD742E002093
:101490000022134670B5214C1118615C83EA0123C8
:1014A000082113F4004F4FEA430318BF83F481531C
:1014B00001F1FF3118BF83F0010311F0FF019BB26E
:1014C000EFD10132192AE6D100F11902A55C00F131
:1014D0001A02A25C02EB052292B29A421DD1104E72
:1014E00096F87F51CAB2AA4214D2431C03EB4203BE
:1014F000DBB2E25C0133E35C03EB02239BB24FF40B
:10150000AF625343074A1B1303F5487322F81130A7
:101510000131E7E7012386F8803170BD4A270020BA
:10152000742E00202827002030B5114A4300D2F83D
:101530008411CC18257E15B1022D10D00BE00228A5
:1015400005D9032807D10B4B1B68DB0401D5C889DB
:1015500030BD888A30BD1344B3F8B80030BD607E1A
:1015600000EB800000EB800000F2EE2080B230BD86
:10157000742E0020342E002008B5F6F74FF9074BE3
:10158000022283F88C21064AC3F888011268C3F846
:101590009821012283F8B12108BD00BF742E0020DC
:1015A000582E002008B5F6F739F9084B022283F8C7
:1015B0008C21D3F8982100F5B71000F5587002F28D
:1015C000DC52C3F88801C3F8982108BD742E0020AE
:1015D00042F20102034B1B681A420CBF012000209B
:1015E000704700BF342E002008B5F6F717F9044BFA
:1015F00000F5F42000F59070C3F8B40108BD00BFF9
:10160000742E002008B5044B1B7803F00503052B4E
:1016100001D1FCF737FCFEE72C300020D0400B1C3A
:101620001141203A03D49C46134118436346524269
:1016300093401843704700BF81F0004102E000BFB3
:1016400083F0004330B54FEA41044FEA430594EA82
:10165000050F08BF90EA020F1FBF54EA000C55EABD
:10166000020C7FEA645C7FEA655C00F0E2804FEA8E
:101670005454D4EB5555B8BF6D420CDD2C4480EA70
:10168000020281EA030382EA000083EA010180EAA0
:10169000020281EA0303362D88BF30BD11F0004FEE
:1016A0004FEA01314FF4801C4CEA113102D0404224
:1016B00061EB410113F0004F4FEA03334CEA13335F
:1016C00002D0524263EB430394EA050F00F0A78077
:1016D000A4F10104D5F1200E0DDB02FA0EFC22FA72
:1016E00005F2801841F1000103FA0EF2801843FA66
:1016F00005F359410EE0A5F120050EF1200E012A57
:1017000003FA0EFC28BF4CF0020C43FA05F3C01894
:1017100051EBE37101F0004507D54FF0000EDCF10D
:10172000000C7EEB00006EEB0101B1F5801F1BD3B6
:10173000B1F5001F0CD349085FEA30004FEA3C0CBA
:1017400004F101044FEA445212F5800F80F09A80B0
:10175000BCF1004F08BF5FEA500C50F1000041EBB4
:10176000045141EA050130BD5FEA4C0C404141EBB8
:10177000010111F4801FA4F10104E9D191F0000FDF
:1017800004BF01460020B1FA81F308BF2033A3F162
:101790000B03B3F120020CDA0C3208DD02F1140C59
:1017A000C2F10C0201FA0CF021FA02F10CE002F194
:1017B0001402D8BFC2F1200C01FA02F120FA0CFC8D
:1017C000DCBF41EA0C019040E41AA2BF01EB0451D6
:1017D000294330BD6FEA04041F3C1CDA0C340EDCD4
:1017E00004F11404C4F1200220FA04F001FA02F317
:1017F00040EA030021FA04F345EA030130BDC4F1D5
:101800000C04C4F1200220FA02F001FA04F340EAC9
:101810000300294630BD21FA04F0294630BD94F07A
:10182000000F83F4801306BF81F480110134013D61
:101830004EE77FEA645C18BF7FEA655C29D094EAD2
:10184000050F08BF90EA020F05D054EA000C04BF50
:101850001946104630BD91EA030F1EBF002100203B
:1018600030BD5FEA545C05D14000494128BF41F0DA
:10187000004130BD14F580043CBF01F5801130BD3E
:1018800001F0004545F0FE4141F470014FF00000C9
:1018900030BD7FEA645C1ABF194610467FEA655C7A
:1018A0001CBF0B46024650EA013406BF52EA03351C
:1018B00091EA030F41F4002130BD00BF90F0000F0A
:1018C00004BF0021704730B54FF4806404F1320446
:1018D0004FF000054FF0000150E700BF90F0000FFF
:1018E00004BF0021704730B54FF4806404F1320426
:1018F00010F0004548BF40424FF000013EE700BFF6
:1019000042004FEAE2014FEA31014FEA02701FBF85
:1019100012F07F4393F07F4F81F06051704792F057
:10192000000F14BF93F07F4F704730B54FF46074D1
:1019300001F0004521F0004120E700BF50EA01021C
:1019400008BF704730B54FF000050AE050EA0102C9
:1019500008BF704730B511F0004502D5404261EB39
:1019600041014FF4806404F132045FEA915C3FF47A
:10197000DCAE4FF003025FEADC0C18BF03325FEA13
:10198000DC0C18BF033202EBDC02C2F1200300FAC8
:1019900003FC20FA02F001FA03FE40EA0E0021FAED
:1019A00002F11444C1E600BF4FEA4102B2F1E04344
:1019B00024BFB3F5001CDCF1FE5C0DD901F0004C36
:1019C0004FEAC0024CEA5070B2F1004F40EB830086
:1019D00008BF20F00100704711F0804F21D113F1B2
:1019E0003872BCBF01F00040704741F480114FEAEB
:1019F0005252C2F11802C2F1200C10FA0CF320FA74
:101A000002F018BF40F001004FEAC1234FEAD32390
:101A100003FA0CFC40EA0C0023FA02F34FEA4303FA
:101A2000CCE77FEA625307D150EA01331EBF4FF083
:101A3000FE4040F44000704701F0004040F0FE409E
:101A400040F40000704700BF80F0004002E000BF9B
:101A500081F0004142001FBF5FEA410392EA030F99
:101A60007FEA226C7FEA236C6AD04FEA1262D2EBE3
:101A70001363C1BFD218414048404140B8BF5B42E8
:101A8000192B88BF704710F0004F40F4000020F081
:101A90007F4018BF404211F0004F41F4000121F097
:101AA0007F4118BF494292EA030F3FD0A2F10102E1
:101AB00041FA03FC10EB0C00C3F1200301FA03F11F
:101AC00000F0004302D5494260EB4000B0F5000F42
:101AD00013D3B0F1807F06D340084FEA310102F101
:101AE0000102FE2A51D2B1F1004F40EBC25008BFB3
:101AF00020F0010040EA03007047490040EB00007D
:101B000010F4000FA2F10102EDD1B0FA80FCACF1AB
:101B1000080CB2EB0C0200FA0CF0AABF00EBC250AA
:101B200052421843BCBFD0401843704792F0000F98
:101B300081F4000106BF80F400000132013BB5E7EB
:101B40004FEA41037FEA226C18BF7FEA236C21D061
:101B500092EA030F04D092F0000F08BF08467047C6
:101B600090EA010F1CBF0020704712F07F4F04D194
:101B7000400028BF40F00040704712F100723CBFA7
:101B800000F50000704700F0004343F0FE4040F4D1
:101B9000000070477FEA226216BF08467FEA23638F
:101BA0000146420206BF5FEA412390EA010F40F47A
:101BB000800070474FF0000304E000BF10F00043C6
:101BC00048BF40425FEA000C08BF704743F09643AD
:101BD00001464FF000001CE050EA010208BF7047C8
:101BE0004FF000030AE000BF50EA010208BF70474F
:101BF00011F0004302D5404261EB41015FEA010C64
